S0030000FC
S21404000052464C2039373435205472616E73666517
S214040010722054726970204361727269657220534B
S214040020595354454D2056657273696F6E20372EAA
S214040030323B202863292032303039202052464C67
S21204004020456C656374726F6E696373004EC0
S214040100ADB9B3DFC6C8CBCADFAB8D9E918C999AC6
S2140401108DDFAB8D968FDFBC9E8D8D969A8DDFAC72
S214040120A6ACABBAB2DFA99A8D8C969091DFC8D1F3
S214040130CDC4DFD79CD6DFCDCFCFC6DFDFADB9B316
S212040140DFBA939A9C8B8D9091969C8C004E01
S2140402004E5600002F0C48780043487800064EB936
S214040210000041244EB90006A2AA48780044487853
S21404022000064EB9000041244FEF0010287C001051
S214040230582842140839000600104D80660000A4B1
S21404024010140C0000086200008C4880D040303B3C
S21404025000064EFB00020012002000280030003E7C
S214040260004C005A006200704EB9000702504EB9A6
S2140402700006647E60624EB900066808605A4EB98D
S2140402800006D4D260524EB9000564BA4EB90006D0
S214040290657660444EB900056B384EB9000666B8FC
S2140402A060364EB90004033C4EB900066760602809
S2140402B04EB90004070E60204EB9000700BE4EB9C2
S2140402C0000701B260124EB90006A0324EB900060D
S2140402D03F1E600418BC00FF52144EB9000642EEDE
S2140402E0600C4EB90006D4D24EB9000675284EB935
S2140402F000064E924EB90006FB344EB900061A3A72
S2140403004EB9000404DA4EB9000070506000FF26AF
S214040310285F4E5E4E754E5600004EB90000705073
S2140403204EB9000070504EB9000070504EB900002F
S21404033070504EB9000070504E5E4E754E5600001A
S2140403400C390003001049D062120C390003001067
S21404035049D462084A3900102D8A67047001600285
S214040360700013C0001020944A39001049D5670461
S21404037070016002700013C0001020970839000353
S21404038000200001670470016002700013C00010B2
S21404039020910839000400200001670470016002FF
S2140403A0700013C0001020920839000000200001DD
S2140403B0670470016002700013C00010209313F9E4
S2140403C00010471D0010209513F90010471E00105A
S2140403D0209D13F90010471B0010209620390010AA
S2140403E0004290B9001049BC723CB08164124A398C
S2140403F0001049DD670A13FC000100102090600C11
S2140404004239001020904239001049DD4A39001064
S2140404104845670000A4227C00104D950C1100018D
S21404042067160C11000267100C110003670A0C1102
S214040430000667047000600870001039001047104A
S21404044013C0001020990C39000100104D96670E59
S2140404500C39000600104D966704700060087000A2
S21404046010390010471113C00010209A0C390001EF
S21404047000104D97670E0C39000600104D97670460
S21404048070006008700010390010471213C0001086
S214040490209B0C39000100104D98670E0C3900069D
S2140404A000104D9867047000600870001039001042
S2140404B0471313C00010209C4A3900104AAF660840
S2140404C04A3900104AB067084A3900104AB166062D
S2140404D042390010209F4E5E4E754E56000048E787
S2140404E001184AB90010003E6700021C207900106B
S2140404F0003E4E9042790010256042074A390010AB
S2140405002100670408C700004A3900102101670467
S21404051008C700014A3900102102670408C7000210
S2140405204A3900102103670408C700034A3900103B
S2140405302104670408C700044A390010210567042B
S21404054008C70005BE390010263967204878000120
S2140405507000100746802F00487800024EB9000647
S214040560FEE44FEF000C13C700102639287C001059
S214040570263A4A3900104854677042074A39001030
S2140405802106670408C700004A39001021076704DB
S21404059008C700014A3900102108670408C700028A
S2140405A04A3900102109670408C700034A390010B5
S2140405B0210A670408C700044A390010210B67049F
S2140405C008C70005BE146744188708C7000648789D
S2140405D000017000100746802F00487800034EB9CB
S2140405E00006FEE44FEF000C60224A14671E420722
S2140405F04214487800017000100746802F0048789F
S21404060000034EB90006FEE44FEF000C4A39001012
S214040610210C670A08F9000000104D726006423982
S21404062000104D72267C001049A816B90010210D42
S214040630287C001049A04A1367144A94661028B907
S214040640001025AA4A9466387001288060324A133E
S214040650662E4A94672A2039001025AA9094D1B9A8
S2140406600010499C4878000448790010499C487951
S214040670006022904EB90006A24C4FEF000C429444
S2140406804A13670C42390010471E42390010209D59
S21404069042474A390010210E670408C700044A3945
S2140406A00010210F670408C700054A3900102110FE
S2140406B0670408C700064A3900102111670408C7F2
S2140406C0000740C046FC3F0033C000100046287CAC
S2140406D000105816700030077200321402810000B1
S2140406E000F0B08167180254FF0F8F5408B9000257
S2140406F00010000933F900100008004000003039EB
S2140407000010004646C04CDF18804E5E4E754E56AE
S21404071000000C390001001052A266084EB900050C
S21404072037E6600261044E5E4E754E56FFF848E7A3
S2140407300138287C0007E9EA267C0010582A247C25
S214040740001058E21039001061DE0C00001662003A
S21404075028344880D040303B00064EFB0002281E5A
S2140407602816020A0214021E0228176C1BF42734E9
S2140407700232276827E8282627FE282C281628264B
S2140407802826177619042826002E00FC0C390002A9
S21404079000104D95670A4A39001048466700009EC7
S2140407A008390003001061BA671E487900084C62D5
S2140407B0487800E24EB900073660508F13FC000CF0
S2140407C0001061DE600027C44A3900104823671E03
S2140407D0487900084C81487800E24EB90007366034
S2140407E0508F13FC000C001061DE6000279E4878D2
S2140407F000F54EB90006EE6C588F4A806700278CC9
S21404080008F90002001061BA13FC0016001061DE3D
S21404081013FC0001001058EA203CFFFFFEDBD0B9B1
S2140408200010004223C0001049C413FC000100104D
S21404083049DF4EB9000070F260002750487900087E
S2140408404CA9487800E24EB900073660508F13FC76
S214040850000C001061DE600027321039001058EAE0
S2140408600C00000167080C000002670E602A13FCE7
S2140408700002001058EA60002712487800FA4EB9C1
S2140408800006EE6C588F4A806700270013FC0003AE
S214040890001058EA600026F44EB900071992083989
S2140408A00002001061BA660026E24EB9000733F271
S2140408B0287C00104D860C140003670026CE0C140A
S2140408C0000266242F390007E8FA4EB90007384CB0
S2140408D0487900084CBB487800FB4EB900073660E0
S2140408E04FEF000C600026A40C14000166242F3978
S2140408F00007E8FA4EB90007384C487900084CD788
S214040900487800FB4EB9000736604FEF000C6000D5
S214040910267A0C14000466242F390007E8FA4EB928
S2140409200007384C487900084CF1487800FB4EB96B
S214040930000736604FEF000C600026500C140005CC
S214040940660026482F390007E8FA4EB90007384CE7
S214040950487900084D0B487800FB4EB9000736600E
S2140409604FEF000C600026244EB900042F9260005E
S214040970261A4EB90004399E600026104EB90004AB
S214040980490A600026064EB900044DDC600025FCCA
S214040990247C001048451039001061E00600004C25
S2140409A00C0000916200150C024000FFD040303B62
S2140409B000064EFB00021080110E119C120E14FC51
S2140409C014FC128012D41328136813BC1410146475
S2140409D014B014FC14FC14FC14FC14FC14FC14FCDA
S2140409E014FC14FC14FC14FC14FC14FC14FC14FC7E
S2140409F014FC14FC14FC14FC14FC14FC14FC14FC6E
S214040A0014FC14FC14FC14FC14FC14FC14FC14FC5D
S214040A1014FC14FC14FC14FC14FC14FC14FC14FC4D
S214040A2014FC14FC14FC14FC14FC14FC14FC14FC3D
S214040A3014FC14FC14FC14FC14FC14FC14FC14FC2D
S214040A4014FC14FC14FC14FC14FC14FC14FC14FC1D
S214040A500124017001E80238027C02F40338037CA6
S214040A6003C004040DB40E060E4A0DCA14FC044852
S214040A700494050C055C05A00618065C06A006E4AE
S214040A80072814FC14FC14FC14FC14FC076C07B8AC
S214040A900830088008C4093C098009C40A080A4CBE
S214040AA014FC14FC14FC14FC14FC0A900ADC0B540E
S214040AB00BA40BE80C600CA40CE80D2C0D7014FCB5
S214040AC014FC14FC0E8E0EB00ED20F260F6C0F8E76
S214040AD00FB00FD20FF4102A10604A1266122F14A9
S214040AE0487800E24EB900073660508F6000249CB8
S214040AF070001039001052B02F007000103900102A
S214040B004D952F004EB9000461502F390007EA7E38
S214040B102F0B2F390007E9464EB90007401E4FEF4A
S214040B200014600024664A1266122F14487800E205
S214040B304EB900073660508F600024502F390010DD
S214040B4052C42F3900104DAA2F39001052B42F3931
S214040B5000104D9A4EB9000462504FEF00104A3907
S214040B6000104847671C2F390007EA8E2F0B2F39D1
S214040B700007E9564EB90007401E4FEF000C600010
S214040B80240A2F390007EA8A2F0B2F390007E95663
S214040B904EB90007401E4FEF000C600023EE4A12C9
S214040BA066122F14487800E24EB900073660508F5C
S214040BB0600023D82F39001052D82F39001052D491
S214040BC02F3900104DBE2F3900104DBA4EB900040F
S214040BD062962F390007EA922F0B2F390007E96631
S214040BE04EB90007401E4FEF001C6000239E4A12B9
S214040BF066122F14487800E24EB900073660508F0C
S214040C00600023882F39001052F42F3900104DDA73
S214040C104EB9000462EE2F390007EA962F0B2F39DF
S214040C200007E96A4EB90007401E4FEF0014600043
S214040C30235A4A1266122F14487800E24EB9000767
S214040C403660508F600023442F39001053142F3918
S214040C5000104DFA2F39001053042F3900104DEAB6
S214040C604EB9000462504FEF00104A39001048474E
S214040C70671C2F390007EA8E2F0B2F390007E96E01
S214040C804EB90007401E4FEF000C600022FE2F39BD
S214040C900007EA8A2F0B2F390007E96E4EB90007C2
S214040CA0401E4FEF000C600022E24A1266122F1418
S214040CB0487800E24EB900073660508F600022CCB8
S214040CC02F39001053242F3900104E0A4EB9000451
S214040CD063322F390007EA9A2F0B2F390007E97E73
S214040CE04EB90007401E4FEF00146000229E4A12C1
S214040CF066122F14487800E24EB900073660508F0B
S214040D00600022882F39001053342F3900104E1AF1
S214040D104EB9000463762F390007EA9E2F0B2F394D
S214040D200007E9824EB90007401E4FEF001460002A
S214040D30225A4A1266122F14487800E24EB9000767
S214040D403660508F600022442F39001053442F39E8
S214040D5000104E2A4EB9000463BA2F390007EAA2DF
S214040D602F0B2F390007E9864EB90007401E4FEFB8
S214040D700014600022164A1266122F14487800E205
S214040D804EB900073660508F600022002F390010DD
S214040D9053542F3900104E3A4EB9000463DA2F39F3
S214040DA00007EAA62F0B2F390007E98A4EB9000779
S214040DB0401E4FEF0014600021D24A1266122F1410
S214040DC0487800E24EB900073660508F600021BCB8
S214040DD02F39001053642F3900104E4A4EB90004C0
S214040DE063FC2F390007EAAA2F0B2F390007E98E78
S214040DF04EB90007401E4FEF00146000218E4A12C1
S214040E0066122F14487800E24EB900073660508FF9
S214040E106000217870001039001052B12F00700065
S214040E20103900104D962F004EB9000461502F392A
S214040E300007EA822F0B2F390007E94A4EB900074C
S214040E40401E4FEF0014600021424A1266122F140F
S214040E50487800E24EB900073660508F6000212CB7
S214040E602F39001052C82F3900104DAE2F390010FC
S214040E7052B82F3900104D9E4EB9000462504FEF01
S214040E8000104A3900104847671C2F390007EA8EBD
S214040E902F0B2F390007E95A4EB90007401E4FEFB3
S214040EA0000C600020E62F390007EA8A2F0B2F3942
S214040EB00007E95A4EB90007401E4FEF000C6000C9
S214040EC020CA4A1266122F14487800E24EB9000768
S214040ED03660508F600020B42F39001052E02F394E
S214040EE0001052DC2F3900104DC62F3900104DC2A9
S214040EF04EB9000462962F390007EA922F0B2F3959
S214040F000007E9664EB90007401E4FEF001C60005C
S214040F10207A4A1266122F14487800E24EB9000767
S214040F203660508F600020642F39001052F82F3935
S214040F3000104DDE4EB9000462EE2F390007EA9623
S214040F402F0B2F390007E96A4EB90007401E4FEFF2
S214040F500014600020364A1266122F14487800E205
S214040F604EB900073660508F600020202F390010DD
S214040F7053182F3900104DFE2F39001053082F39FF
S214040F8000104DEE4EB9000462504FEF00104A397F
S214040F9000104847671C2F390007EA8E2F0B2F399D
S214040FA00007E9724EB90007401E4FEF000C6000C0
S214040FB01FDA2F390007EA8A2F0B2F390007E97248
S214040FC04EB90007401E4FEF000C60001FBE4A12C9
S214040FD066122F14487800E24EB900073660508F28
S214040FE060001FA82F39001053282F3900104E0E0A
S214040FF04EB9000463322F390007EA9A2F0B2F39B3
S2140410000007E97E4EB90007401E4FEF001460004B
S2140410101F7A4A1266122F14487800E24EB9000767
S2140410203660508F60001F642F39001053382F39F4
S21404103000104E1E4EB9000463762F390007EA9E50
S2140410402F0B2F390007E9824EB90007401E4FEFD9
S214041050001460001F364A1266122F14487800E205
S2140410604EB900073660508F60001F202F390010DD
S21404107053482F3900104E2E4EB9000463BA2F3948
S2140410800007EAA22F0B2F390007E9864EB900079E
S214041090401E4FEF001460001EF24A1266122F1410
S2140410A0487800E24EB900073660508F60001EDCB8
S2140410B02F39001053582F3900104E3E4EB90004F5
S2140410C063DA2F390007EAA62F0B2F390007E98ABF
S2140410D04EB90007401E4FEF001460001EAE4A12C1
S2140410E066122F14487800E24EB900073660508F17
S2140410F060001E982F39001053682F3900104E4E8A
S2140411004EB9000463FC2F390007EAAA2F0B2F39C7
S2140411100007E98E4EB90007401E4FEF001460002A
S2140411201E6A4A1266122F14487800E24EB9000767
S2140411303660508F60001E5470001039001052B292
S2140411402F007000103900104D972F004EB9000480
S21404115061502F390007EA862F0B2F390007E94E16
S2140411604EB90007401E4FEF001460001E1E4A12C0
S21404117066122F14487800E24EB900073660508F86
S21404118060001E082F39001052CC2F3900104DB2C3
S2140411902F39001052BC2F3900104DA24EB900044E
S2140411A062504FEF00104A3900104847671C2F3929
S2140411B00007EA8E2F0B2F390007E95E4EB90007A9
S2140411C0401E4FEF000C60001DC22F390007EA8A4C
S2140411D02F0B2F390007E95E4EB90007401E4FEF6C
S2140411E0000C60001DA64A1266122F14487800E20E
S2140411F04EB900073660508F60001D902F390010DE
S21404120052E82F39001052E42F3900104DCE2F39F2
S21404121000104DCA4EB9000462962F390007EA92B0
S2140412202F0B2F390007E9664EB90007401E4FEF13
S214041230001C60001D564A1266122F14487800E2FD
S2140412404EB900073660508F60001D402F390010DD
S21404125052FC2F3900104DE24EB9000462EE2F39CD
S2140412600007EA962F0B2F390007E96A4EB90007E4
S214041270401E4FEF001460001D124A1266122F140F
S214041280487800E24EB900073660508F60001CFCB8
S2140412902F390010531C2F3900104E022F3900101E
S2140412A0530C2F3900104DF24EB9000462504FEF24
S2140412B000104A3900104847671C2F390007EA8E89
S2140412C02F0B2F390007E9764EB90007401E4FEF63
S2140412D0000C60001CB62F390007EA8A2F0B2F3942
S2140412E00007E9764EB90007401E4FEF000C600079
S2140412F01C9A4A1266122F14487800E24EB9000768
S2140413003660508F60001C842F390010532C2F3900
S21404131000104E124EB9000463322F390007EA9AC1
S2140413202F0B2F390007E97E4EB90007401E4FEFFA
S214041330001460001C564A1266122F14487800E205
S2140413404EB900073660508F60001C402F390010DD
S214041350533C2F3900104E224EB9000463762F39C1
S2140413600007EA9E2F0B2F390007E9824EB90007C3
S214041370401E4FEF001460001C124A1266122F140F
S214041380487800E24EB900073660508F60001BFCB8
S2140413902F390010534C2F3900104E324EB900042A
S2140413A063BA2F390007EAA22F0B2F390007E98604
S2140413B04EB90007401E4FEF001460001BCE4A12C1
S2140413C066122F14487800E24EB900073660508F34
S2140413D060001BB82F390010535C2F3900104E42A2
S2140413E04EB9000463DA2F390007EAA62F0B2F390B
S2140413F00007E98A4EB90007401E4FEF001460004C
S2140414001B8A4A1266122F14487800E24EB9000767
S2140414103660508F60001B742F390010536C2F39C0
S21404142000104E524EB9000463FC2F390007EAAA96
S2140414302F0B2F390007E98E4EB90007401E4FEFD9
S214041440001460001B464A1266122F14487800E205
S2140414504EB900073660508F60001B30700010399C
S214041460001052B32F007000103900104D982F0052
S2140414704EB9000461502F390007EA862F0B2F3926
S2140414800007E9524EB90007401E4FEF00146000F3
S2140414901AFA4A1266122F14487800E24EB9000768
S2140414A03660508F60001AE42F39001052D02F395E
S2140414B000104DB62F39001052C02F3900104DA61B
S2140414C04EB9000462504FEF00104A3900104847E6
S2140414D0671C2F390007EA8E2F0B2F390007E962A5
S2140414E04EB90007401E4FEF000C60001A9E2F39BD
S2140414F00007EA8A2F0B2F390007E9624EB9000766
S214041500401E4FEF000C60001A824A1266122F1417
S214041510487800E24EB900073660508F60001A6CB7
S2140415202F39001052F02F39001052EC2F390010CA
S2140415304DD62F3900104DD24EB9000462962F397D
S2140415400007EA922F0B2F390007E9664EB9000709
S214041550401E4FEF001C60001A324A1266122F1407
S214041560487800E24EB900073660508F60001A1CB7
S2140415702F39001053002F3900104DE64EB90004E1
S21404158062EE2F390007EA962F0B2F390007E96A17
S2140415904EB90007401E4FEF0014600019EE4A12C1
S2140415A066122F14487800E24EB900073660508F52
S2140415B0600019D82F39001053202F3900104E061A
S2140415C02F39001053102F3900104DF64EB9000471
S2140415D062504FEF00104A3900104847671C2F39F5
S2140415E00007EA8E2F0B2F390007E97A4EB9000759
S2140415F0401E4FEF000C600019922F390007EA8A4C
S2140416002F0B2F390007E97A4EB90007401E4FEF1B
S214041610000C600019764A1266122F14487800E20D
S2140416204EB900073660508F600019602F390010DD
S21404163053302F3900104E164EB9000463322F393A
S2140416400007EA9A2F0B2F390007E97E4EB90007E8
S214041650401E4FEF0014600019324A1266122F140F
S214041660487800E24EB900073660508F6000191CB7
S2140416702F39001053402F3900104E264EB900045F
S21404168063762F390007EA9E2F0B2F390007E9826D
S2140416904EB90007401E4FEF0014600018EE4A12C1
S2140416A066122F14487800E24EB900073660508F51
S2140416B0600018D82F39001053502F3900104E36BA
S2140416C04EB9000463BA2F390007EAA22F0B2F394C
S2140416D00007E9864EB90007401E4FEF001460006D
S2140416E018AA4A1266122F14487800E24EB9000768
S2140416F03660508F600018942F39001053602F39CD
S21404170000104E464EB9000463DA2F390007EAA6E5
S2140417102F0B2F390007E98A4EB90007401E4FEFFA
S2140417200014600018664A1266122F14487800E205
S2140417304EB900073660508F600018502F390010DD
S21404174053702F3900104E564EB9000463FC2F39DF
S2140417500007EAAA2F0B2F390007E98E4EB90007B7
S214041760401E4FEF0014600018222F390007EA3A93
S214041770487800E94EB900073660508F6000180CB0
S2140417804A390010484667224EB90005522A2F39B6
S2140417900007EAB22F0B2F390007E9964EB9000767
S2140417A0401E4FEF000C600017E22F14487800E24A
S2140417B04EB900073660508F600017D04A390010C3
S2140417C04846672A4EB90005506408F9000600101A
S2140417D061DF2F390007EADA2F0B2F390007E9BE3D
S2140417E04EB90007401E4FEF000C6000179E2F14E2
S2140417F0487800E24EB900073660508F6000178CB8
S2140418004A3900104846672A4EB9000550A608F91A
S2140418100006001061DF2F390007EADA2F0B2F3994
S2140418200007E9C24EB90007401E4FEF000C6000E7
S214041830175A2F14487800E24EB900073660508FC6
S214041840600017484EB900049EC82F390007EAD630
S2140418502F0B2F390007E9E64EB90007401E4FEF5D
S214041860000C600017264EB9000467282F390007BD
S214041870EC1E2F0B2F390007E9B64EB90007401EA1
S2140418804FEF000C600017044A390010484C6618E5
S2140418904A390010484D66104A390010484E66080A
S2140418A04A390010484F67224EB9000466D42F39CF
S2140418B00007EACA2F0B2F390007E9B24EB9000712
S2140418C0401E4FEF000C600016C22F14487800E24A
S2140418D04EB900073660508F600016B04EB900044B
S2140418E0678E4A3900104846671C2F390007EAD22B
S2140418F02F0B2F390007E9BA4EB90007401E4FEFE9
S214041900000C600016862F390007EACE2F0B2F39FD
S2140419100007E9BA4EB90007401E4FEF000C6000FE
S214041920166A4EB9000464DE2F390007EAB62F0B98
S2140419302F390007E99A4EB90007401E4FEF000CF6
S214041940600016484EB90004655C2F390007EABAF1
S2140419502F0B2F390007E99E4EB90007401E4FEFA4
S214041960000C600016264EB9000465BA2F3900072D
S214041970EABE2F0B2F390007E9A24EB90007401E16
S2140419804FEF000C600016044EB9000466282F3989
S2140419900007EAC22F0B2F390007E9A64EB9000745
S2140419A0401E4FEF000C600015E270003039001046
S2140419B053802F00700030390010472C2F004EB98A
S2140419C0000466822F390007EAC62F0B2F3900075A
S2140419D0E9AA4EB90007401E4FEF0014600015AC8C
S2140419E070003039001053822F0070003039001018
S2140419F0472E2F004EB9000466822F390007EAC628
S214041A002F0B2F390007E9AE4EB90007401E4FEFE3
S214041A100014600015762F390007EC1E487900087C
S214041A204D332F390007E91E4EB90007401E4FEF0D
S214041A30000C600015564A1267084A390010472AF7
S214041A4066122F14487800E24EB900073660508FAD
S214041A506000153848790007ECAA4879001053BE90
S214041A604EB9000780384A4067202F39001053C209
S214041A702F39001053BE487900084D412F0B4EB93C
S214041A80000747704FEF0010601E2F390010259492
S214041A902F3900102590487900084D4C2F0B4EB96D
S214041AA0000747704FEF0010487900084D572F0B7A
S214041AB02F390007EADE4EB90007401E4FEF000C30
S214041AC0600014C84A1267084A390010472A66128A
S214041AD02F14487800E24EB900073660508F600035
S214041AE014AA48790007ECAA4879001053C64EB9E0
S214041AF0000780384A4067202F39001053CA2F3910
S214041B00001053C6487900084D682F0B4EB90007DD
S214041B1047704FEF0010601E2F390010259C2F3998
S214041B2000102598487900084D722F0B4EB900070F
S214041B3047704FEF0010487900084D7C2F0B2F3963
S214041B400007EAE24EB90007401E4FEF000C6000A3
S214041B50143A4A1267084A390010472A66122F14A4
S214041B60487800E24EB900073660508F6000141CB7
S214041B702F39001053CE2F39001025A04EB900047B
S214041B8062EE508F4A3900104847671C48790008AF
S214041B904D8D2F0B2F390007EAE64EB90007401E7D
S214041BA04FEF000C600013E4487900084D982F0BA3
S214041BB02F390007EAE64EB90007401E4FEF000C27
S214041BC0600013C84A1267084A390010472A66128A
S214041BD02F14487800E24EB900073660508F600034
S214041BE013AA2F39001053D22F39001025A44EB94A
S214041BF0000462EE508F4A3900104847671C487943
S214041C0000084DA32F0B2F390007EAEA4EB9000748
S214041C10401E4FEF000C60001372487900084DAE6A
S214041C202F0B2F390007EAEA4EB90007401E4FEF84
S214041C30000C600013564A1266084A390010472AF8
S214041C4066122F14487800E24EB900073660508FAB
S214041C506000133870003039001053BC2F00700039
S214041C60303900104E882F004EB90005513048799F
S214041C7000084DB92F0B2F390007E9DE4EB90007CF
S214041C80401E4FEF0014600013024A1266084A39D9
S214041C900010472A66122F14487800E24EB900074F
S214041CA03660508F600012E470003039001053BA6A
S214041CB02F007000303900104E862F004EB90005F4
S214041CC05130487900084DC32F0B2F390007E9E23D
S214041CD04EB90007401E4FEF0014600012AE4A12C1
S214041CE066084A390010472A66122F14487800E21C
S214041CF04EB900073660508F600012904EB900054A
S214041D0051BA487900084DCD2F0B2F390007E9C684
S214041D104EB90007401E4FEF000C6000126E4A12C8
S214041D2066084A390010472A66122F14487800E2DB
S214041D304EB900073660508F60001250700010399C
S214041D40001053B52F007000103900104E812F007C
S214041D504EB9000550EA487900084DD62F0B2F39A6
S214041D600007E9D64EB90007401E4FEF0014600086
S214041D70121A4A1266084A390010472A66122F14A5
S214041D80487800E24EB900073660508F600011FCB8
S214041D9070001039001053B62F0070001039001070
S214041DA04E822F004EB9000550EA487900084DDEF1
S214041DB02F0B2F390007E9DA4EB90007401E4FEF04
S214041DC00014600011C64A1266084A390010472AF1
S214041DD066122F14487800E24EB900073660508F1A
S214041DE0600011A870001039001053B82F0070005E
S214041DF0103900104E842F004EB9000550EA487979
S214041E0000084DE62F0B2F390007E9D24EB900071C
S214041E10401E4FEF0014600011724A1266084A39D9
S214041E200010472A66122F14487800E24EB90007BD
S214041E303660508F600011542F39001053A22F398A
S214041E4000104E6E4EB900055176487900084DEDE7
S214041E502F0B2F390007E9CA4EB90007401E4FEF73
S214041E600014600011264A1266084A390010472AF0
S214041E7066122F14487800E24EB900073660508F79
S214041E80600011082F39001053A62F3900104E7227
S214041E904EB900055176487900084DFB2F0B2F39B3
S214041EA00007E9CE4EB90007401E4FEF001460004D
S214041EB010DA42A742A7487900084E094EB900072F
S214041EC0401E4FEF000C600010C24EB900045E08BE
S214041ED0600010B81039001061E050000C000008D3
S214041EE0620001764880D040303B00064EFB00027C
S214041EF0014E0134011A00D000B6009C005200388E
S214041F000012487900084E114EB90007384C2F3994
S214041F100007E8FA4EB90007384C508F13FC00FF50
S214041F20001061E060001064487900084E394EB92C
S214041F300007384C588F13FC00FE001061E0600068
S214041F40104A08F90004001061DF487900084E5D65
S214041F504EB90007384C588F08390001001049B4B0
S214041F606710487900084E8E4EB90007384C588FD3
S214041F70600E487900084E9B4EB90007384C588FBF
S214041F8013FC00FD001061E06000100048790008B2
S214041F904EAA4EB90007384C588F13FC00FC0010AC
S214041FA061E060000FE6487900084EC64EB90007A7
S214041FB0384C588F13FC00FB001061E060000FCC17
S214041FC008F90004001061DF487900084EE24EB9B3
S214041FD00007384C588F08390000001049B46710C1
S214041FE0487900084F134EB90007384C588F600ED6
S214041FF0487900084F1D4EB90007384C588F13FC1B
S21404200000FA001061E060000F82487900084F274C
S2140420104EB90007384C588F13FC00F9001061E0E5
S21404202060000F68487900084F3C4EB90007384CEA
S214042030588F13FC00F8001061E060000F4E4879DA
S21404204000084F5E4EB90007384C588F13FC00F753
S214042050001061E060000F344EB90007470C6000C2
S2140420600F2A4EB90007347624804A80660E42A7AB
S2140420704EB9000731A0588F600002C8287C0010B3
S21404208049B2267C001049B820400C100030654840
S2140420900C10003962422F084EB90007708A588F18
S2140420A036804A40631CB054621813FC00100010BB
S2140420B049B54279001049B64EB90007314660006A
S2140420C00282487900084F87487800F54EB9000721
S2140420D03660508F6000026C2E3C00600000205278
S2140420E010100C000041673C0C000044670000A27E
S2140420F00C000045670001040C00004C6700016EEC
S2140421000C000051670001D00C000052670001D299
S2140421100C00003F670002020C000048670001FA4A
S2140421206000020408790001001049B408F90004AC
S214042130001061DF487900084FA24EB9000737A0A7
S214042140588F08390001001049B467104879000810
S2140421504FC34EB90007384C588F600E48790008B4
S2140421604FD04EB90007384C588F4878000148794C
S214042170001049B4487900800DE04EB90006A09ED0
S21404218042A74EB9000731A04FEF0010600001B41B
S2140421904A54634613FC0030001049B542790010D7
S2140421A049B60C54006464043694601E203900104A
S2140421B02562B087660636BC0064600E9087E280AF
S2140421C0722A4EB900077972368033D3001049BAA2
S2140421D04EB9000731466000016A2F390007EA72DB
S2140421E0487800F64EB90007366042A74EB9000795
S2140421F031A04FEF000C6000014A4A54634E13FCB2
S2140422000020001049B54279001049B60C54006409
S214042210640A303CFFFFD05436806020203900101A
S2140422202562B087660636BC006360109087E2803D
S214042230722A4EB9000779725340368033D30010A1
S21404224049BA4EB900073146600000F82F39000736
S214042250EA72487800F64EB90007366042A74EB9CF
S214042260000731A04FEF000C600000D8087900008A
S214042270001049B408F90004001061DF487900082A
S2140422804FDF4EB9000737A0588F083900000010FA
S21404229049B46710487900084FFF4EB90007384C18
S2140422A0588F600E4879000850094EB90007384C1C
S2140422B0588F487800014879001049B4487900805E
S2140422C00DE04EB90006A09E42A74EB9000731A005
S2140422D04FEF0010606C13FC0014001061DE6062A7
S2140422E04A54631613FC0040001049B542790010A6
S2140422F049B64EB90007314660482F390007EA72DE
S214042300487800F64EB90007366042A74EB9000773
S21404231031A04FEF000C602A487800014EB9000740
S21404232031A0588F601C2F390007EA6E48780001E8
S2140423304EB90007366042A74EB9000731A04FEFEA
S214042340000C4EB9000738724EB9000719926000A7
S2140423500C3A4EB90007347624804A80661E2F391C
S2140423600007E9F6487800E34EB900073660508F58
S21404237008B90005001061DF60000B0C103900106E
S21404238061E00600004C0C00009162000AF4024072
S21404239000FFD040303B00064EFB000206F007AAC2
S2140423A0086408F20AE40AE4098009B209E40A089F
S2140423B00A3A0A6A0A8A0AB80AE40AE40AE40AE44E
S2140423C00AE40AE40AE40AE40AE40AE40AE40AE494
S2140423D00AE40AE40AE40AE40AE40AE40AE40AE484
S2140423E00AE40AE40AE40AE40AE40AE40AE40AE474
S2140423F00AE40AE40AE40AE40AE40AE40AE40AE464
S2140424000AE40AE40AE40AE40AE40AE40AE40AE453
S2140424100AE40AE40AE40AE40AE40AE40AE40AE443
S2140424200AE40AE40AE40AE40AE40AE40AE40AE433
S2140424300AE40AE40AE40124012E018C019E01B098
S21404244001EC023A024C025E02700AE406B006D0C0
S21404245006A60AE40282029A02BE02D002E2031E22
S214042460036C037E039003A20AE40AE40AE40AE483
S2140424700AE403B403CC03F0040204140450049ED8
S21404248004B004C204D40AE40AE40AE40AE40AE44B
S21404249004E604FE052205340546058205D005E259
S2140424A005F406060AE40AE40AE406180622062CDC
S2140424B0063E0650065A0664066E0678068A069C8B
S2140424C04EB90004685C600009B80C3900FF0010BF
S2140424D052B0672A70001039001052B02F002F39FE
S2140424E00007E9564879001052C44879001052B4DF
S2140424F04EB900046AC24FEF0010600009847000F1
S214042500103900104D952F002F390007E9564879E9
S214042510001052C44879001052B44EB900046AC27E
S2140425204FEF00106000095A4879001052D44EB993
S21404253000046D04588F600009484879001052F46E
S2140425404EB900046DAE588F600009360CB9FFFF13
S214042550FC1800105324660A23F900104E0A0010D3
S21404256053244879001053242F390007E96E48791C
S214042570001053144879001053044EB900046B8EAF
S2140425804FEF0010600008FA0CB9FFFFFC180010AB
S21404259053046718203900105314D0B9001053049C
S2140425A072024EB9000779202E00601620390010FA
S2140425B04DFAD0B900104DEA72024EB900077920E0
S2140425C02E002F074879001053244EB900046E32AB
S2140425D0508F600008AC4879001053344EB900049C
S2140425E06EFE588F6000089A4879001053444EB91E
S2140425F000046F82588F600008884879001053548E
S2140426004EB900047006588F6000087648790010AA
S21404261053644EB90004708C588F600008642F39D8
S2140426200007E94A4879001052B14EB9000468DA46
S214042630508F6000084C487800012F390007E95A8B
S2140426404879001052C84879001052B84EB90004B0
S2140426506AC24FEF0010600008284879001052DC68
S2140426604EB900046D04588F6000081648790010AF
S21404267052F84EB900046DAE588F600008040CB9C9
S214042680FFFFFC1800105328660A23F900104E0EAC
S214042690001053284879001053282F390007E97290
S2140426A04879001053184879001053084EB90004AE
S2140426B06B8E4FEF0010600007C80CB9FFFFFC18C4
S2140426C0001053086718203900105318D0B90010AA
S2140426D0530872024EB9000779202E00601620397E
S2140426E000104DFED0B900104DEE72024EB9000730
S2140426F079202E002F074879001053284EB900047D
S2140427006E32508F6000077A4879001053384EB9FD
S21404271000046EFE588F600007684879001053481E
S2140427204EB900046F82588F60000756487900102F
S21404273053584EB900047006588F60000744487911
S214042740001053684EB90004708C588F600007322E
S2140427502F390007E94E4879001052B24EB90004EA
S214042760695A508F6000071A487800012F3900070D
S214042770E95E4879001052CC4879001052BC4EB934
S21404278000046AC24FEF0010600006F64879001095
S21404279052E44EB900046D04588F600006E448798C
S2140427A0001052FC4EB900046DAE588F600006D27D
S2140427B00CB9FFFFFC180010532C660A23F900100E
S2140427C04E120010532C48790010532C2F39000752
S2140427D0E97648790010531C48790010530C4EB91A
S2140427E000046B8E4FEF0010600006960CB9FFFFD6
S2140427F0FC180010530C671820390010531CD0B96D
S2140428000010530C72024EB9000779202E00601691
S214042810203900104E02D0B900104DF272024EB9A3
S214042820000779202E002F0748790010532C4EB944
S21404283000046E32508F6000064848790010533CFE
S2140428404EB900046EFE588F6000063648790010B4
S214042850534C4EB900046F82588F600006244879A2
S2140428600010535C4EB900047006588F60000612C0
S21404287048790010536C4EB90004708C588F600071
S21404288006002F390007E9524879001052B34EB9B2
S2140428900004695A508F600005E8487800012F3913
S2140428A00007E9624879001052D04879001052C0F7
S2140428B04EB900046AC24FEF0010600005C44879A0
S2140428C0001052EC4EB900046D04588F600005B237
S2140428D04879001053004EB900046DAE588F60005E
S2140428E005A00CB9FFFFFC1800105330660A23F944
S2140428F000104E16001053304879001053302F390C
S2140429000007E97A487900105320487900105310DC
S2140429104EB900046B8E4FEF0010600005640CB9CE
S214042920FFFFFC18001053106718203900105320BE
S214042930D0B90010531072024EB9000779202E0049
S2140429406016203900104E06D0B900104DF67202FB
S2140429504EB9000779202E002F074879001053300F
S2140429604EB900046E32508F600005164879001088
S21404297053404EB900046EFE588F60000504487933
S214042980001053504EB900046F82588F600004F252
S2140429904879001053604EB900047006588F6000E2
S2140429A004E04879001053704EB90004708C588FB8
S2140429B0600004CE4EB900049F40600004C44EB9C3
S2140429C0000475FA600004BA4879001053744EB9CE
S2140429D00004757C588F600004A84879001053756D
S2140429E04EB900047682588F600004964EB90004EF
S2140429F071966000048C4EB9000471F46000048281
S214042A004EB900047322600004784EB90004743A88
S214042A106000046E4879001053804EB9000474C0F8
S214042A20588F6000045C4879001053824EB9000445
S214042A3074C0588F6000044A4EB90004965A600069
S214042A4004404EB9000557A6600004362F39000727
S214042A50E9BE4879001053964879001053924EB94F
S214042A600005529A4FEF000C600004162F39000739
S214042A70E9C248790010539E48790010539A4EB91B
S214042A800005529A4FEF000C600003F64A39001016
S214042A90472A670000A02F1243EEFFF84EB900073E
S214042AA04EBA588F48790007ECB2486EFFF84EB914
S214042AB0000780384A406D6648790007ECBA486ECD
S214042AC0FFF84EB9000780384A406E5223EEFFF8EE
S214042AD0001053BE23EEFFFC001053C22F39001023
S214042AE053C22F39001053BE4879000850132F0BD9
S214042AF04EB90007477008F90006001061DF2F0B77
S214042B002F390007EADE70001039001061E02F004C
S214042B104EB900073C5E4FEF001C600003642F397B
S214042B200007EA6E487800014EB900073660508FF9
S214042B306000034E2F14487800E24EB90007366052
S214042B40508F6000033C4A390010472A670000A0F3
S214042B502F1243EEFFF84EB900074EBA588F487945
S214042B600007ECC2486EFFF84EB9000780384A40AA
S214042B706D6648790007ECCA486EFFF84EB9000740
S214042B8080384A406E5223EEFFF8001053C623EEF8
S214042B90FFFC001053CA2F39001053CA2F390010F7
S214042BA053C648790008501E2F0B4EB900074770CD
S214042BB008F90006001061DF2F0B2F390007EAE240
S214042BC070001039001061E02F004EB900073C5E1B
S214042BD04FEF001C600002AA2F390007EA6E4878FF
S214042BE000014EB900073660508F600002942F141F
S214042BF0487800E24EB900073660508F60000282C3
S214042C004A390010472A67742F124EB90007708A93
S214042C10588F2E004A3900104847670670DABE807F
S214042C206C0670DFBE806D3E4A876E3A23C700107E
S214042C3053CE4879001053CE4EB90004630E08F9FB
S214042C400006001061DF2F0B2F390007EAE670003C
S214042C501039001061E02F004EB900073C5E4FEFBC
S214042C6000106000021C2F390007EA6E4878000145
S214042C704EB900073660508F600002062F1448785D
S214042C8000E24EB900073660508F600001F44A39FE
S214042C900010472A67742F124EB90007708A588F9F
S214042CA02E004A3900104847670670DABE806C0664
S214042CB070DFBE806D3E4A876E3A23C7001053D23B
S214042CC04879001053D24EB90004630E08F9000682
S214042CD0001061DF2F0B2F390007EAEA7000103965
S214042CE0001061E02F004EB900073C5E4FEF001065
S214042CF06000018E2F390007EA6E487800014EB94D
S214042D0000073660508F600001782F14487800E280
S214042D104EB900073660508F600001664A390010CD
S214042D20472A67182F390007E9DE4879001053BC94
S214042D304EB9000555EC508F600001462F144878B4
S214042D4000E24EB900073660508F600001344A39FD
S214042D500010472A67182F390007E9E2487900105F
S214042D6053BA4EB9000555EC508F600001142F1469
S214042D70487800E24EB900073660508F60000102C2
S214042D804A390010472A670A4EB9000556FA600009
S214042D9000F02F14487800E24EB900073660508FD2
S214042DA0600000DE4A390010472A67182F390007EA
S214042DB0E9D64879001053B54EB9000554E0508F53
S214042DC0600000BE2F14487800E24EB90007366053
S214042DD0508F600000AC4A390010472A67182F3914
S214042DE00007E9DA4879001053B64EB9000554E0F6
S214042DF0508F6000008C2F14487800E24EB900070C
S214042E003660508F607A4A390010472A67084EB9F0
S214042E1000055566606A2F14487800E24EB900072C
S214042E203660508F605A4A390010472A67162F3981
S214042E300007E9CA4879001053A24EB90005567235
S214042E40508F603C2F14487800E24EB90007366075
S214042E50508F602C4A390010472A67162F3900070E
S214042E60E9CE4879001053A64EB900055672508F25
S214042E70600E2F14487800E24EB900073660508F73
S214042E804EB90007387213FC000C001061DE6000B7
S214042E9000FA4A3900104D7366164EB900047BDCFE
S214042EA013C0001061DE4EB90004F338600000DC85
S214042EB04EB900047FEA13C0001061DE4EB9000468
S214042EC0F34A600000C64EB90004DA484EB900045E
S214042ED0D3E24A39001048626762487800014879AC
S214042EE00010485E487900800D484EB90006A09E42
S214042EF04878000148790010485F487900800D4AF8
S214042F004EB90006A09E4878000148790010486033
S214042F10487900800D4C4EB90006A09E4878000102
S214042F20487900104861487900800D4E4EB9000675
S214042F30A09E4FEF003042390010486213FC000C8C
S214042F40001061DE60444EB90004D3E24EB90004BA
S214042F50D89013FC000C001061DE602E4A79001035
S214042F6049B666084EB90004F388601E4EB90004DC
S214042F70F46660164EB900071992600E4EB9000743
S214042F80199260064EB9000719924CDF1C804E5EFB
S214042F904E754E56000048E70F38287C001061E056
S214042FA0267C0010582A247C000738E410140C00F1
S214042FB0006F656C6700086A0C000078650A0C00F0
S214042FC0008262326000097E0C000072651C670095
S214042FD008C20C000074650008FA6700091C0C009F
S214042FE00075660009A66000093C0C0000706700C6
S214042FF00856600008780C0000FD6518670009464E
S2140430000C0000FE670000EE0C0000FF6600097C62
S214043010600000CC0C0000FC660009706000023EF4
S2140430200C00005E6558670002BA0C000066652E48
S214043030670005020C0000696518670006480C0066
S214043040006A670006B00C00006B6600093E60006C
S21404305007AA0C0000676700054C600005B80C0062
S2140430600060650002EE6700035A0C00006167000A
S21404307003E40C00006566000912600004480C00B6
S21404308000586526670001060C00005B65106700A3
S21404309001740C00005C67000192600001D60C000D
S2140430A00059660008E6600001260C000055650E0F
S2140430B067680C00005667000088600000AA4A0093
S2140430C0660008C8600000024879000850284EB917
S2140430D00007384C588F18BC00FF600008BA4879BF
S2140430E0000850724EB90007384C588F18BC00FEC2
S2140430F0600008A4487800554EB90004D0B41E00F9
S214043100700010072F004879000850BC4878005516
S2140431104E924FEF00106000087E487800564EB975
S2140431200004D0B41E00700010072F004879000871
S21404313050CC487800564E924FEF00106000085866
S214043140487800574EB90004D0B41E00700010072B
S2140431502F004879000850D6487800574E924FEF13
S214043160001060000832487800584EB90004D0B405
S2140431701E00700010072F004879000850E44878B5
S21404318000584E924FEF00106000080C4878005923
S2140431904EB90004D0B41E00700010072F00487902
S2140431A0000850F3487800594E924FEF00100C393F
S2140431B0000300104D95660007DE4EB9000734265E
S2140431C04A00660007D218BC005B600007CA48784D
S2140431D0005B4EB90004D0B41E00700010072F0028
S2140431E04879000850FF4878005B4E924FEF001075
S2140431F04EB9000734264A006600079C18BC005CDB
S214043200600007944878005C4EB90004D0B41E00F1
S214043210700010072F0048790008510F4878005CAA
S2140432204E924FEF00106000076E4878005D4EB96E
S2140432300004D0B41E0008F90006001061DF700018
S21404324010072F0048790008511E4878005D4E92FA
S2140432504FEF001018BC00FC6000073C48790008DB
S214043260512C4EB90007384C588F18BC005D6000CE
S21404327007264A39001020806704704160027049AE
S21404328028004A39001020826704704160027049A1
S2140432902A004A390010208467047041600270498D
S2140432A02C004A3900102086670470416002704979
S2140432B02E002F072F062F052F042F390007E9426B
S2140432C02F0B4EB9000747702F0B4879000851742E
S2140432D04878005E4EB9000741664FEF0024600050
S2140432E006B64A39001020816704704160027049AE
S2140432F028004A3900102083670470416002704930
S2140433002A004A390010208567047041600270491B
S2140433102C004A3900102087670470416002704907
S2140433202E002F072F062F052F042F390007E942FA
S2140433302F0B4EB9000747702F0B487900085183AE
S2140433404878005F4EB9000741664FEF00246000DE
S21404335006464A39001020886704704160027049A6
S21404336028004A390010208A6704704160027049B8
S2140433702A004A390010208C6704704160027049A4
S2140433802C004A390010208E670470416002704990
S2140433902E002F072F062F052F042F390007E9428A
S2140433A02F0B4EB9000747702F0B4879000851922F
S2140433B0487800604EB9000741664FEF002460006D
S2140433C005D64A39001020896704704160027049A6
S2140433D028004A390010208B670470416002704947
S2140433E02A004A390010208D670470416002704933
S2140433F02C004A390010208F67047041600270491F
S2140434002E002F072F062F052F042F390007E94219
S2140434102F0B4EB90007477008F90006001061DF4D
S2140434202F0B4879000851A3487800614EB900076D
S21404343041664FEF00244A39001048466700055895
S2140434404EB9000734264A006600054C18BC006BCB
S214043450600005444A390010201767047041600272
S214043460704928004A390010201F67047041600222
S21404347070492A004A390010202767047041600208
S21404348070492C004A390010202F670470416002EE
S21404349070492E002F072F062F052F042F390007FB
S2140434A0E9422F0B4EB9000747702F0B48790008E6
S2140434B051B4487800654EB9000741664FEF0024C2
S2140434C0600004D44A390010201667047041600274
S2140434D0704928004A390010201E670470416002B3
S2140434E070492A004A390010202667047041600299
S2140434F070492C004A390010202E6704704160027F
S21404350070492E002F072F062F052F042F3900078A
S214043510E9422F0B4EB9000747702F0B4879000875
S21404352051C4487800664EB9000741664FEF002440
S214043530600004644A390010201267047041600277
S214043540704928004A390010201A67047041600246
S21404355070492A004A39001020226704704160022C
S21404356070492C004A390010202A67047041600212
S21404357070492E002F072F062F052F042F3900071A
S214043580E9422F0B4EB9000747702F0B4879000805
S21404359051CD487800674EB9000741664FEF0024C6
S2140435A0600003F44A390010201467047041600276
S2140435B0704928004A390010201C670470416002D4
S2140435C070492A004A3900102024670470416002BA
S2140435D070492C004A390010202C670470416002A0
S2140435E070492E002F072F062F052F042F390007AA
S2140435F0E9422F0B4EB9000747702F0B4879000895
S21404360051DE487800684EB9000741664FEF002443
S214043610600003844A390010201367047041600276
S214043620704928004A390010201B67047041600264
S21404363070492A004A39001020236704704160024A
S21404364070492C004A390010202B67047041600230
S21404365070492E002F072F062F052F042F39000739
S214043660E9422F0B4EB9000747702F0B4879000824
S21404367051EF487800694EB9000741664FEF0024C1
S214043680600003144A390010201567047041600274
S214043690704928004A390010201D670470416002F2
S2140436A070492A004A3900102025670470416002D8
S2140436B070492C004A390010202D670470416002BE
S2140436C070492E002F072F062F052F042F390007C9
S2140436D0E9422F0B4EB9000747702F0B48790008B4
S2140436E051FF4878006A4EB9000741664FEF002440
S2140436F0600002A40C39000100104D9567220C39B5
S214043700000200104D9567180C39000300104D9503
S214043710670E0C39000600104D9567047044600E61
S2140437204A39001047106704704160027049280047
S2140437300C39000100104D96670E0C390006001077
S2140437404D9667047044600E4A39001047116704AA
S2140437507041600270492A000C39000100104D9730
S214043760670E0C39000600104D9767047044600E0F
S2140437704A390010471267047041600270492C00F1
S2140437800C39000100104D98670E0C390006001025
S2140437904D9867047044600E4A3900104713670456
S2140437A07041600270492E002F072F062F052F0444
S2140437B02F390007E9422F0B4EB90007477008F966
S2140437C00006001061DF2F0B48790008520F487876
S2140437D0006B4EB9000741664FEF00244A390010CB
S2140437E04845670001B24EB9000734264A00660011
S2140437F001A618BC00756000019E4878006F4EB99B
S2140438000004D0B41E00700010072F00487900088A
S214043810521A4878006F4E924FEF001060000178FD
S214043820487800704EB90004D0B41E00700010072B
S2140438302F0048790008522B487800704E924FEFBC
S214043840001060000152487800714EB90004D0B4EC
S2140438501E00700010072F0048790008523C487874
S21404386000714E924FEF00106000012C48780072F1
S2140438704EB90004D0B41E00700010072F0048791B
S21404388000085249487800724E924FEF00106000CC
S2140438900106487800734EB90004D0B41E007000C8
S2140438A010072F00487900085256487800734E9245
S2140438B04FEF00104A3900104851660000DA4EB93E
S2140438C0000734264A00660000CE18BC0074600068
S2140438D000C6487800744EB90004D0B41E007000C8
S2140438E010072F00487900085263487800744E92F7
S2140438F04FEF0010600000A0487800754EB9000431
S214043900D0B41E0008F90006001061DF700010072E
S2140439102F0048790008526B487800754E924FEF96
S214043920001060722F390007E8FA4EB90007384CC9
S2140439304879000852774EB90007384C508F18BCA7
S21404394000FD60520C1400FD660618BC0078600288
S2140439505214700010142F004EB90004D0B4588FBF
S2140439601E000C0700FF672E700010142F004EB9BF
S2140439700004BE28700010072F002F0B70001014D0
S2140439802F004E924FEF0010600C42A742A742A7AA
S2140439904E924FEF000C4CDF1CF04E5E4E754E56AA
S2140439A0FFD848E73F38287C001061E0267C0007F3
S2140439B0ECA2247C0010582A1014060000740C0094
S2140439C0007462000F2E4880D040303B00064EFB49
S2140439D000020170019001EA024E034203C6041E6F
S2140439E004BA04E805160544057205CE0F20062C15
S2140439F0062C062C062C062C062C062C062C073227
S214043A0007320732073207320732073207DA09DE8F
S214043A100A5E0ADE0B560BE80D420E1E0F200F2020
S214043A200F200F200F200F200F200F200F200F2015
S214043A300F200F200F200F200F200F200F200F2005
S214043A400F200F200F200F200F200F200F200F20F5
S214043A500F200F200F200F200F200F200F200F20E5
S214043A600F200F200F200F200F200F200F200F20D5
S214043A700F200F200F200F200F200F200F200F20C5
S214043A800F200F200F200F200F200F200F200F20B5
S214043A900F200F200F200F200F200F200F200F20A5
S214043AA00F200F200F200F200F200F200F200F2095
S214043AB00F2006DC05AC0116010000EA4879000870
S214043AC0528C4EB90007384C588F18BC00FF600063
S214043AD00E324879000852CF4EB90007384C588F3A
S214043AE018BC00FE60000E1C700010390010471849
S214043AF0E2802E00083900000010471867162F07CA
S214043B0048790008531E2F0A4EB9000747704FEF36
S214043B10000C60142F074879000853262F0A4EB964
S214043B20000747704FEF000C2F0A48790008532E01
S214043B304878008C4EB9000741664FEF000C6000D1
S214043B400DC24EB900047A7E2F0A48790008533C09
S214043B504878008D4EB9000741664FEF000C6000B0
S214043B600DA27000103900104719E2802E000839A3
S214043B7000000010471967162F0748790008534BB2
S214043B802F0A4EB9000747704FEF000C60142F073A
S214043B904879000853532F0A4EB9000747704FEF71
S214043BA0000C2F0A48790008535B4878008E4EB9FB
S214043BB0000741664FEF000C60000D487000103996
S214043BC0001049B02F0070001039001049AE2F00C5
S214043BD070001039001049AF2F0070001039001023
S214043BE049AB2F0070001039001049AC2F0070004C
S214043BF01039001049AD2F004879000853692F0A80
S214043C004EB9000747702F0A48790008538748784A
S214043C10008F4EB9000741664FEF002C60000CE49D
S214043C202E390010499C4A39001049A8670E2039DD
S214043C30001025AA90B9001049A0DE802007223C77
S214043C400A4CB8004EB9000779722800C1414EB933
S214043C5000078C96C1419E812007223C006DDD0042
S214043C604EB9000779722C00C1414EB900078C96F4
S214043C70C1419E812007223C0001D4C04EB90007F2
S214043C8079722600C1414EB900078C96C1419E81C7
S214043C902007223C000007D04EB9000779722A009C
S214043CA020072D40FFD82005C1414EB900078C9649
S214043CB0C14193AEFFD8202EFFD872024EB900073A
S214043CC0792024004A8467182F062F0448790008B0
S214043CD053972F0A4EB9000747704FEF0010601A2B
S214043CE02F022F052F032F064879000853A92F0A01
S214043CF04EB9000747704FEF00182F0A487900089E
S214043D0053BD487800904EB9000741664FEF000C4B
S214043D1060000BF0486EFFDD4EB9000703A4700088
S214043D20102EFFE32F007000102EFFE12F0070000E
S214043D30102EFFE22F007000102EFFDE2F00700002
S214043D40102EFFDF2F007000102EFFE02F004879A2
S214043D50000853CD2F0A4EB90007477008F900062D
S214043D60001061DF2F0A4879000853EB4878009169
S214043D704EB9000741664FEF00304A3900104846F6
S214043D8066000B804EB9000734264A0066000B74A2
S214043D9018BC00FD60000B6C0CB9FFFFFFFF0010A1
S214043DA0480666122F390007E90A2F0A4EB90000A2
S214043DB071C2508F60182F390010480648790008E1
S214043DC053F82F0A4EB9000747704FEF000C08F956
S214043DD00006001061DF2F0A4879000853FC487873
S214043DE000924EB9000741664FEF000C60000B14BA
S214043DF04AB90010480666122F390007E90A2F0A46
S214043E004EB9000071C2508F60684879001047F6BA
S214043E104EB900077D964A00661248790008540693
S214043E202F0A4EB900074770508F6046487900073E
S214043E30ECD24879001047F64EB9000780384A405D
S214043E406F1248790008540C2F0A4EB9000071C24C
S214043E50508F601E2F39001047FA2F39001047F68E
S214043E604879000854162F0A4EB9000747704FEFDA
S214043E7000102F0A48790008541C487800934EB95D
S214043E80000741664FEF000C60000A782F390010D7
S214043E90472648790008542B2F0A4EB90007477066
S214043EA02F0A487900085431487800944EB9000720
S214043EB041664FEF001860000A4A2F39001049582F
S214043EC048790008543D2F0A4EB9000747702F0A58
S214043ED0487900085443487800954EB9000741666F
S214043EE04FEF001860000A1C2F390010495C48790F
S214043EF0000854502F0A4EB9000747702F0A487915
S214043F0000085456487800964EB9000741664FEFAD
S214043F100018600009EE2F3900104960487900083F
S214043F2054632F0A4EB9000747702F0A48790008D1
S214043F305469487800974EB9000741664FEF001859
S214043F40600009C02F390010496448790008547B82
S214043F502F0A4EB90007477008F90006001061DF03
S214043F602F0A487900085481487800984EB900070B
S214043F7041664FEF001818BC00FD600009862F3913
S214043F800007E8FA4EB90007384C487900085493FD
S214043F904EB90007384C508F18BC0098600009646E
S214043FA04A390010200867047041600270492E00E8
S214043FB02F39001048642F072F390007E9362F0AD7
S214043FC04EB9000747702F390007EB222F39000738
S214043FD0EB922F390007EB1E4879001058CC4EB9E7
S214043FE0000747702F0A4879001058CC4878009A82
S214043FF04EB9000741664FEF002C600009067000BA
S21404400010140680FFFFFF6606800007EB4A204078
S2140440101C10700010060680001057D620404A1068
S21404402067047041600270492E0070001014068008
S214044030FFFFFF66E58806800007EB7222402051EA
S2140440402F102F072F390007E9362F0A4EB900071D
S2140440504770700010140680FFFFFF66E588068030
S2140440600007EB2220402F102F390007EB962F393C
S2140440700007EB1E4879001058CC4EB9000747706D
S2140440802F0A4879001058CC7008D0147200120019
S21404409020012F004EB9000741664FEF002C0C1488
S2140440A000A96600085E18BC00FC600008562F399C
S2140440B00007E8FA4EB90007384C588F4A39001002
S2140440C0484667104879000854DB4EB90007384C58
S2140440D0588F600E4879000855254EB90007384CAD
S2140440E0588F4A390010484667124EB900073426DE
S2140440F04A00660818BC00AE6000080818BC00A990
S214044100600008005214700010140680FFFFFF5E63
S21404411006800007EB4220401C1070001006068044
S2140441200010200020404A10670470416002704965
S2140441302E00700010140680FFFFFF5EE5880680E0
S2140441400007EB52224020512F102F072F3900076B
S214044150E9362F0A4EB9000747707000101406801F
S214044160FFFFFF5EE58806800007EB2220402F1045
S2140441702F390007EB922F390007EB1E4879001001
S21404418058CC4EB9000747702F0A4879001058CC0F
S214044190103C00F8D0147200120020012F004EB913
S2140441A0000741664FEF002C60000758287C00107B
S2140441B04D95267C0007E90E0C14000167120C14BA
S2140441C00002670C0C14000367060C140006663421
S2140441D00CB9FFFFFC1900104700660E2F132F0AB8
S2140441E04EB9000071C2508F602A2F390010470064
S2140441F04879000855602F0A4EB9000747704FEFFC
S214044200000C60102F390007E90A2F0A4EB9000087
S21404421071C2508F2F390007E90648790010582DCF
S2140442204EB9000071C2508F0C39000100104D9633
S214044230670A0C39000600104D96663C0CB9FFFF61
S214044240FC190010470466122F13487900105835DD
S2140442504EB9000071C2508F60322F3900104704E7
S2140442604879000855644879001058354EB9000757
S21404427047704FEF000C60142F390007E90A48799D
S214044280001058354EB9000071C2508F2F39000700
S214044290E9064879001058384EB9000071C2508FAC
S2140442A00C39000100104D97670A0C3900060010FF
S2140442B04D97663C0CB9FFFFFC19001047086612C0
S2140442C02F134879001058404EB9000071C2508F21
S2140442D060322F3900104708487900085568487935
S2140442E0001058404EB9000747704FEF000C60149A
S2140442F02F390007E90A4879001058404EB90000E3
S21404430071C2508F2F390007E906487900105843C8
S2140443104EB9000071C2508F0C39000100104D9840
S214044320670A0C39000600104D98663C0CB9FFFF6E
S214044330FC190010470C66122F1348790010584BCE
S2140443404EB9000071C2508F60322F390010470CEE
S21404435048790008556C48790010584B4EB9000748
S21404436047704FEF000C60142F390007E90A4879AC
S2140443700010584B4EB9000071C2508F487900089F
S214044380557048790010584E4EB9000071C208F9AD
S2140443900006001061DF2F0A487900085575487832
S2140443A000AA4EB9000741664FEF0014600005549A
S2140443B008390000001046EC67047041600270493A
S2140443C02A0008390000001046ED670470416002B8
S2140443D07049280008390000001046EE6704704152
S2140443E0600270492C0008390000001046EF67048C
S2140443F07041600270492E002F072F062F042F05E8
S2140444002F390007E93A2F0A4EB90007477008F912
S2140444100006001061DF2F0A4879000855854878A1
S21404442000AB4EB9000741664FEF0024600004D489
S21404443008390001001046EC6704704960027041B8
S2140444402A0008390001001046ED6704704960022E
S2140444507041280008390001001046EE67047049D0
S214044460600270412C0008390001001046EF670412
S2140444707049600270412E002F072F062F042F0567
S2140444802F390007E93A2F0A4EB90007477008F992
S2140444900006001061DF2F0A487900085591487815
S2140444A000AC4EB9000741664FEF00246000045488
S2140444B04A390010201067047041600270492A00CF
S2140444C04A390010201867047041600270492800B9
S2140444D04A390010202067047041600270492C009D
S2140444E04A390010202867047041600270492E0083
S2140444F02F072F062F042F052F390007E93A2F0A16
S2140445004EB90007477008F90006001061DF2F0A4D
S21404451048790008559C487800AD4EB900074166B6
S2140445204FEF0024600003DC4A39001020116704B2
S2140445307041600270492A004A3900102019670445
S21404454070416002704928004A390010202167042F
S2140445507041600270492C004A3900102029670413
S2140445607041600270492E002F072F062F042F0576
S2140445702F390007E93A2F0A4EB90007477008F9A1
S2140445800006001061DF2F0A4879000855A948780C
S21404459000AE4EB9000741664FEF00244A390010BA
S2140445A048466600035E4EB9000734264A00660095
S2140445B0035218BC00B06000034A287C0007ECA62F
S2140445C008390000001046F167160839000000108C
S2140445D046F6670820790007EC9E600220536002C6
S2140445E020542D48FFFC08390001001046F16716D8
S2140445F008390001001046F6670820790007EC9E8B
S21404460060022053600220542D48FFF80839000247
S214044610001046F1671608390002001046F66708CF
S21404462020790007EC9E60022053600220542D4837
S214044630FFF408390003001046F167160839000332
S214044640001046F6670820790007EC9E60022053A7
S214044650600220542D48FFF008390004001046F18B
S214044660671608390004001046F767082079000723
S214044670EC9E60022053600220542D48FFEC08395B
S2140446800005001046F1671608390005001046F7C5
S214044690670820790007EC9E6002205360022054CD
S2140446A02D48FFE808390006001046F16716083959
S2140446B00006001046F7670820790007EC9E6002A3
S2140446C02053600220542D48FFE42F082F2EFFE8C5
S2140446D02F2EFFEC2F2EFFF02F2EFFF42F2EFFF899
S2140446E02F2EFFFC2F390007E93E2F0A4EB900078C
S2140446F0477008F90006001061DF2F0A48790008A1
S21404470055B5487800AF4EB9000741664FEF003004
S214044710600001F0287C001046F0081400006708CA
S21404472020790007EC9E600220532D48FFFC0814F5
S2140447300001670820790007EC9E600220532D488C
S214044740FFF808140002670820790007EC9E600250
S21404475020532D48FFF40814000367082079000747
S214044760EC9E600220532D48FFF0081400046708EE
S21404477020790007EC9E600220532D48FFEC0814B5
S2140447800005670820790007EC9E600220532D4838
S214044790FFE808140006670820790007EC9E60020C
S2140447A020532D48FFE42F082F2EFFE82F2EFFEC72
S2140447B02F2EFFF02F2EFFF42F2EFFF82F2EFFFCA8
S2140447C02F390007E93E2F0A4EB90007477008F94B
S2140447D00006001061DF2F0A4879000855C14878A2
S2140447E000B04EB9000741664FEF00306000011478
S2140447F04A390010472A670000E8264A287900103C
S21404480047C27E002C3C001047366042202C000233
S214044810E2882F007000102C00072F00424010146E
S2140448207200320020012F004879000855CD2F0B66
S2140448304EB9000747704FEF001447EB000B49ECE6
S214044840FFF2B9C66406287C001047B45287700588
S214044850BE806DB808F90006001061DF2F0A48799B
S214044860000855DF487800C74EB9000741664FEF89
S214044870000C264A7E006042202C0002E2882F00AC
S2140448807000102C00072F004240101472003200F3
S21404489020012F004879000855EB2F0B4EB900076E
S2140448A047704FEF001447EB000B49ECFFF2B9C614
S2140448B06406287C001047B452877005BE806DB825
S2140448C008F90006001061DF2F0A2F390007E8FAFE
S2140448D0487800C84EB9000741664FEF000C6022C6
S2140448E042A742A742A74EB9000741664FEF000C05
S2140448F0601042A742A742A74EB9000741664FEF91
S214044900000C4CDF1CFC4E5E4E754E56000048E70D
S2140449100038287C0010582A267C001061DF247C8E
S214044920001061E010120C00004C653C6700021C8D
S2140449300C0000506522670003140C00005265004A
S2140449400350670003A00C000053670004160C0015
S21404495000FF6600047060520C00004E6500021AE8
S21404496067000262600002A20C000048651467003B
S21404497000A00C00004A650000BA67000128600029
S21404498001960C000046626667424A0066000436DA
S214044990600000024879000855FD4EB90007384CFF
S2140449A0588F14BC00FF6000042C08D30006487916
S2140449B00004002E487900085611487800464EB97F
S2140449C0000741664FEF000C6000040A08D3000697
S2140449D048790000402C48790008561D487800475E
S2140449E04EB9000741664FEF000C600003E808D399
S2140449F0000648790007E88C487900085625487868
S214044A0000484EB9000741664FEF000C600003C62D
S214044A1008D300064879000074E448790008563143
S214044A20487800494EB9000741664FEF000C600015
S214044A3003A4487800302F390007F0322F390007D6
S214044A40F02E48790008563B4EB9000051844FEFCB
S214044A5000100C4000016618487800302F39000713
S214044A60F02E2F0C4EB9000752F44FEF000C6016D0
S214044A7048780030487900078E3A2F0C4EB9000764
S214044A8052F44FEF000C08D300062F0C48790008A8
S214044A9056454878004A4EB9000741664FEF000C69
S214044AA060000332487800302F390007F0422F396F
S214044AB00007F03E4879000856524EB9000051846B
S214044AC04FEF00100C4000016618487800302F396C
S214044AD00007F03E2F0C4EB9000752F44FEF000CBF
S214044AE0601648780030487900078E3A2F0C4EB985
S214044AF0000752F44FEF000C08D300062F0C487939
S214044B00000856584878004B4EB9000741664FEFE8
S214044B10000C600002C04A39001048546708287C1C
S214044B20000856676006287C0008567108D30006FD
S214044B302F0C48790008567F4878004C4EB9000779
S214044B4041664FEF000C6000028C70003039001094
S214044B50472C2F004EB90004D2B408D300062F0CFD
S214044B6048790008568E4878004D4EB900074166CD
S214044B704FEF00106000025E700030390010472EC0
S214044B802F004EB90004D2B408D300062F0C48797F
S214044B900008569C4878004E4EB9000741664FEF11
S214044BA000104A390010484667124EB900073426EA
S214044BB04A00660814BC00526000021A14BC004E78
S214044BC0600002124A390010484C67184A3900102F
S214044BD04847670828790007E92E600E28790007F9
S214044BE0E92A600628790007E93208D300062F0C64
S214044BF02F390007E9464878004F4EB9000741664A
S214044C004FEF000C600001CE4A390010484D67187B
S214044C104A3900104847670828790007E92E600ECD
S214044C2028790007E92A600628790007E93208D3BC
S214044C3000062F0C2F390007E94A487800504EB971
S214044C40000741664FEF000C6000018A4A390010E5
S214044C50484E67184A3900104847670828790007FD
S214044C60E92E600E28790007E92A600628790007ED
S214044C70E93208D300062F0C2F390007E94E48788E
S214044C8000514EB9000741664FEF000C6000014624
S214044C904A390010484F67184A39001048476708D1
S214044CA028790007E92E600E28790007E92A6006AD
S214044CB028790007E93208D300062F0C2F3900079D
S214044CC0E952487800524EB9000741664FEF000C8F
S214044CD04EB9000734264A00660000FA14BC005495
S214044CE0600000F21039001048210C00000C672008
S214044CF00C00000967220C00000A67240C00000B55
S214044D0067260C00000867280C00000F672A60302E
S214044D10287C000856AB602E287C000856C1602606
S214044D20287C000856DE601E287C000856FF6016A5
S214044D30287C00085718600E287C00085732600646
S214044D40287C0008574D08D300062F0C4879000825
S214044D505764487800534EB9000741664FEF000C7D
S214044D6060724AB900104806672E203C000001F421
S214044D70D0B900104806223C000003E84EB90007EC
S214044D8079722F004879000857712F0C4EB9000726
S214044D9047704FEF000C60104879000857812F0CBD
S214044DA04EB9000071C2508F08D300062F0C487904
S214044DB00008578A487800544EB9000741664FEFFA
S214044DC0000C601042A742A742A74EB900074166EE
S214044DD04FEF000C4CDF1C004E5E4E754E56000026
S214044DE048E70138287C001061DF267C0010582A2A
S214044DF0247C001061E010120600004C0C000091A8
S214044E0062000FEE024000FFD040303B00064EFB2F
S214044E1000020D6E0DDC0E080E340FDE0FDE0E964D
S214044E200ECA0EEA0F1E0F520F840FB20FDE0FDEED
S214044E300FDE0FDE0FDE0FDE0FDE0FDE0FDE0FDE01
S214044E400FDE0FDE0FDE0E340FDE0FDE0FDE0FDE9C
S214044E500FDE0FDE0FDE0FDE0FDE0FDE0FDE0FDEE1
S214044E600FDE0FDE0FDE0FDE0FDE0FDE0FDE0FDED1
S214044E700FDE0FDE0FDE0FDE0FDE0FDE0FDE0FDEC1
S214044E800FDE0FDE0FDE0FDE0FDE0FDE0FDE0FDEB1
S214044E900FDE0FDE0FDE0FDE0FDE0FDE0FDE0FDEA1
S214044EA00FDE0FDE0FDE0166013A012401D2020E88
S214044EB00246027202AE02DA03060332035E038E71
S214044EC00A660A8A0AAE0AD60B1A04060442047A4A
S214044ED004A604E2050E053A0566059205C20FDE31
S214044EE00FDE0FDE0FDE0FDE063A067606AE06DAB5
S214044EF007160742076E079A07C607F60FDE0FDE89
S214044F000FDE0FDE0FDE086E08AA08E2090E094A55
S214044F10097609A209CE09FA0A440FDE0FDE0FDE6F
S214044F200B3A0B5A0BB40BD40BF40C140C340C5471
S214044F300C880CBC0CDE4879000857944EB9000760
S214044F40384C588F14BC00FF60000EB642A74EB90A
S214044F5000073B08588F4A3900104846670A4EB97E
S214044F60000734264A00670814BC00FE60000E9250
S214044F7014BC003760000E8A70001039001052B05E
S214044F802F007000103900104D952F004EB9000404
S214044F90615008D400062F0B2F390007E9464878DD
S214044FA000014EB900073C5E70001039001052B084
S214044FB02F007000103900104D952F004EB90004D4
S214044FC062344FEF001C7E001E004A8766000E32D5
S214044FD04EB9000734264A0066000E2614BC000AA2
S214044FE060000E1E2F39001052C42F3900104DAA2F
S214044FF02F39001052B42F3900104D9A4EB90004C0
S214045000625008D400062F0B2F390007E95648785B
S21404501000024EB900073C5E4FEF001C60000DE234
S2140450202F39001052D82F39001052D42F390010BF
S2140450304DBE2F3900104DBA4EB9000462962F0BA0
S2140450402F390007E966487800034EB900073C5E2E
S2140450504FEF001C60000DAA2F39001052F42F39B0
S21404506000104DDA4EB9000462EE2F0B2F390007FC
S214045070E96A487800044EB900073C5E4FEF001416
S21404508060000D7E2F39001053142F3900104DFA8E
S2140450902F39001053042F3900104DEA4EB900047E
S2140450A0625008D400062F0B2F390007E96E4878A3
S2140450B000054EB900073C5E4FEF001C60000D4231
S2140450C02F39001053242F3900104E0A4EB900040D
S2140450D063322F0B2F390007E97E487800064EB955
S2140450E000073C5E4FEF001460000D162F390010C9
S2140450F053342F3900104E1A4EB9000463762F0B22
S2140451002F390007E982487800074EB900073C5E4D
S2140451104FEF001460000CEA2F39001053442F3967
S21404512000104E2A4EB9000463BA2F0B2F3900071D
S214045130E986487800084EB900073C5E4FEF001435
S21404514060000CBE2F39001053542F3900104E3A0D
S2140451504EB9000463DA2F0B2F390007E98A487822
S21404516000094EB900073C5E4FEF001460000C9235
S2140451702F39001053642F3900104E4A4EB90004DC
S21404518063FC08D400062F0B2F390007E98E4878F5
S214045190000A4EB900073C5E4FEF001460000C6234
S2140451A02F390007E8FA4EB90007384C700010395A
S2140451B0001052B12F007000103900104D962F00C9
S2140451C04EB90004615008D400062F0B2F3900078F
S2140451D0E94A487800104EB900073C5E7000103962
S2140451E0001052B12F007000103900104D962F0099
S2140451F04EB9000462344FEF00207E001E004A873A
S21404520066000BFE4EB9000734264A0066000BF211
S21404521014BC001960000BEA2F39001052C82F394D
S21404522000104DAE2F39001052B82F3900104D9E85
S2140452304EB90004625008D400062F0B2F3900071D
S214045240E95A487800114EB900073C5E4FEF001C3F
S21404525060000BAE2F39001052E02F39001052DCDC
S2140452602F3900104DC62F3900104DC24EB9000418
S21404527062962F0B2F390007E966487800124EB95C
S21404528000073C5E4FEF001C60000B762F390010C1
S21404529052F82F3900104DDE4EB9000462EE2F0B83
S2140452A02F390007E96A487800134EB900073C5EB8
S2140452B04FEF001460000B4A2F39001053182F3993
S2140452C000104DFE2F39001053082F3900104DEEF4
S2140452D04EB90004625008D400062F0B2F3900077D
S2140452E0E972487800144EB900073C5E4FEF001C84
S2140452F060000B0E2F39001053282F3900104E0E65
S2140453004EB9000463322F0B2F390007E97E487824
S21404531000154EB900073C5E4FEF001460000AE229
S2140453202F39001053382F3900104E1E4EB9000482
S21404533063762F0B2F390007E982487800164EB99A
S21404534000073C5E4FEF001460000AB62F390010C9
S21404535053482F3900104E2E4EB9000463BA2F0B53
S2140453602F390007E986487800174EB900073C5ED7
S2140453704FEF001460000A8A2F39001053582F3953
S21404538000104E3E4EB9000463DA2F0B2F39000787
S214045390E98A487800184EB900073C5E4FEF0014BF
S2140453A060000A5E2F39001053682F3900104E4EE5
S2140453B04EB9000463FC08D400062F0B2F390007EF
S2140453C0E98E487800194EB900073C5E4FEF00148A
S2140453D060000A2E2F390007E8FA4EB90007384C49
S2140453E070001039001052B22F00700010390010EF
S2140453F04D972F004EB90004615008D400062F0BB9
S2140454002F390007E94E4878001F4EB900073C5E66
S21404541070001039001052B22F00700010390010BE
S2140454204D972F004EB9000462344FEF00207E00E3
S2140454301E004A87660009CA4EB9000734264A0089
S214045440660009BE14BC0028600009B62F39001097
S21404545052CC2F3900104DB22F39001052BC2F39C0
S21404546000104DA24EB90004625008D400062F0B5B
S2140454702F390007E95E487800204EB900073C5EE5
S2140454804FEF001C6000097A2F39001052E82F39BC
S214045490001052E42F3900104DCE2F3900104DCA9B
S2140454A04EB9000462962F0B2F390007E966487838
S2140454B000214EB900073C5E4FEF001C6000094215
S2140454C02F39001052FC2F3900104DE24EB900045B
S2140454D062EE2F0B2F390007E96A487800224EB98E
S2140454E000073C5E4FEF0014600009162F390010C9
S2140454F0531C2F3900104E022F390010530C2F392D
S21404550000104DF24EB90004625008D400062F0B6A
S2140455102F390007E976487800234EB900073C5E29
S2140455204FEF001C600008DA2F390010532C2F3977
S21404553000104E124EB9000463322F0B2F390007A9
S214045540E97E487800244EB900073C5E4FEF00140D
S214045550600008AE2F390010533C2F3900104E223D
S2140455604EB9000463762F0B2F390007E98248787A
S21404557000254EB900073C5E4FEF00146000088219
S2140455802F390010534C2F3900104E324EB90004F8
S21404559063BA2F0B2F390007E986487800264EB9E0
S2140455A000073C5E4FEF0014600008562F390010C9
S2140455B0535C2F3900104E424EB9000463DA2F0BA9
S2140455C02F390007E98A487800274EB900073C5E61
S2140455D04FEF00146000082A2F390010536C2F393F
S2140455E000104E524EB9000463FC08D400062F0B7C
S2140455F02F390007E98E487800284EB900073C5E2C
S2140456004FEF0014600007FA2F390007E8FA4EB986
S2140456100007384C70001039001052B32F00700089
S214045620103900104D982F004EB90004615008D46C
S21404563000062F0B2F390007E9524878002E4EB982
S21404564000073C5E70001039001052B32F00700043
S214045650103900104D982F004EB9000462344FEFF5
S21404566000207E001E004A87660007964EB9000793
S21404567034264A006600078A14BC000F60000782BE
S2140456802F39001052D02F3900104DB62F39001084
S21404569052C02F3900104DA64EB90004625008D4EB
S2140456A000062F0B2F390007E9624878002F4EB901
S2140456B000073C5E4FEF001C600007462F390010C1
S2140456C052F02F39001052EC2F3900104DD62F39D6
S2140456D000104DD24EB9000462962F0B2F390007E6
S2140456E0E966487800304EB900073C5E4FEF001C70
S2140456F06000070E2F39001053002F3900104DE6B6
S2140457004EB9000462EE2F0B2F390007E96A487879
S21404571000314EB900073C5E4FEF0014600006E20D
S2140457202F39001053202F3900104E062F39001041
S21404573053102F3900104DF64EB90004625008D4A9
S21404574000062F0B2F390007E97A487800324EB945
S21404575000073C5E4FEF001C600006A62F390010C1
S21404576053302F3900104E164EB9000463322F0BF7
S2140457702F390007E97E487800334EB900073C5EAF
S2140457804FEF00146000067A2F39001053402F396B
S21404579000104E264EB9000463762F0B2F390007EF
S2140457A0E982487800344EB900073C5E4FEF001497
S2140457B06000064E2F39001053502F3900104E3615
S2140457C04EB9000463BA2F0B2F390007E9864878D0
S2140457D000354EB900073C5E4FEF00146000062209
S2140457E02F39001053602F3900104E464EB900046E
S2140457F063DA2F0B2F390007E98A487800364EB94A
S21404580000073C5E4FEF0014600005F62F390010C9
S21404581053702F3900104E564EB9000463FC08D45A
S21404582000062F0B2F390007E98E487800374EB94B
S21404583000073C5E4FEF00144A39001048466600E5
S21404584005C04EB9000734264A00660005B414BCE9
S214045850000F600005AC08D400064879000857EA33
S2140458604879000857DC4878000B4EB900073C5EC0
S2140458704FEF000C6000058A4EB90005506408D44A
S21404588000062F0B2F390007E9BE4878000C4EB9E6
S21404589000073C5E4FEF000C600005664EB900053D
S2140458A050A608D400062F0B2F390007E9C2487803
S2140458B0000D4EB900073C5E4FEF000C6000054239
S2140458C04EB90005522A08D400062F0B2F390007BC
S2140458D0E9964878000E4EB900073C5E4FEF000C80
S2140458E014BC000F6000051A7000103900104E76C4
S2140458F0D08006800007F1602040301048C02F009A
S2140459004879000857F22F0B4EB90007477008D4A1
S21404591000062F0B4879000857F54878000F4EB953
S21404592000073C5E4FEF0018600004D64EB9000432
S2140459309EC82F0B2F390007E9E64878003B4EB97E
S21404594000073C5E4FEF000C600004B64EB900043E
S21404595067282F0B2F390007E9B64878003C4EB964
S21404596000073C5E4FEF000C600004964A390010B6
S214045970484567204A390010484C66224A390010C8
S214045980484D661A4A390010484E66124A390010C5
S214045990484F660A4EB9000734264A0067204EB9B7
S2140459A0000466D42F0B2F390007E9B24878003D6F
S2140459B04EB900073C5E4FEF000C6000044414BC74
S2140459C0003D6000043C4EB90004678E2F0B2F394F
S2140459D00007E9BA4878003E4EB900073C5E4FEF30
S2140459E0000C6000041C4EB9000464DE2F0B2F3933
S2140459F00007E99A4878003F4EB900073C5E4FEF2F
S214045A00000C600003FC4EB90004655C2F0B2F39B4
S214045A100007E99E487800404EB900073C5E4FEF09
S214045A20000C600003DC4EB9000465BA2F0B2F3956
S214045A300007E9A2487800414EB900073C5E4FEFE4
S214045A40000C600003BC4EB9000466282F0B2F39E7
S214045A500007E9A6487800424EB900073C5E4FEFBF
S214045A60000C6000039C70003039001053802F0037
S214045A70700030390010472C2F004EB9000466829F
S214045A802F0B2F390007E9AA487800434EB90007C0
S214045A903C5E4FEF0014600003687000303900105D
S214045AA053822F00700030390010472E2F004EB955
S214045AB0000466822F0B2F390007E9AE48780044AD
S214045AC04EB900073C5E4FEF00146000033408D460
S214045AD000062F390007E8FA2F390007E91E487830
S214045AE000454EB900073C5E4FEF000C6000031201
S214045AF04A390010484666084A390010472A660A9A
S214045B004EB9000734264A00676E48790007ECDA77
S214045B104879001053BE4EB9000780384A406720C3
S214045B202F39001053C22F39001053BE487900088D
S214045B3058042F0B4EB9000747704FEF0010601E35
S214045B402F39001025942F39001025904879000825
S214045B50580F2F0B4EB9000747704FEF00102F0B4E
S214045B602F390007EADE487800B44EB900073C5ED9
S214045B704FEF000C6000028A14BC00CE6000028264
S214045B8048790007ECDA4879001053C64EB9000786
S214045B9080384A4067202F39001053CA2F39001026
S214045BA053C648790008581A2F0B4EB90007477099
S214045BB04FEF0010601E2F390010259C2F3900105F
S214045BC025984879000858242F0B4EB900074770CB
S214045BD04FEF00102F0B2F390007EAE2487800B584
S214045BE04EB900073C5E4FEF000C600002142F39DC
S214045BF0001053CE2F39001025A04EB9000462EED3
S214045C002F0B2F390007EAE6487800B64EB900078E
S214045C103C5E4FEF0014600001E82F39001053D2A9
S214045C202F39001025A44EB9000462EE2F0B2F392D
S214045C300007EAEA487800B74EB900073C5E4FEF23
S214045C400014600001BC4A390010484667084A3907
S214045C500010472A660A4EB9000734264A006734FD
S214045C6070003039001053BC2F007000303900101B
S214045C704E882F004EB9000551302F0B2F390007E0
S214045C80E9DE487800BA4EB900073C5E4FEF0014D0
S214045C906000016E42A742A742A74EB900073C5EC9
S214045CA04FEF000C6000015A70003039001053BAF0
S214045CB02F007000303900104E862F004EB90005B4
S214045CC051302F0B2F390007E9E2487800BB4EB954
S214045CD000073C5E4FEF0014600001264EB9000535
S214045CE051BA2F0B2F390007E9C6487800BC4EB9C5
S214045CF000073C5E4FEF000C600001067000103990
S214045D00001053B52F007000103900104E812F007C
S214045D104EB9000550EA2F0B2F390007E9D648780C
S214045D2000BD4EB900073C5E4FEF0014600000D281
S214045D3070001039001053B62F0070001039001090
S214045D404E822F004EB9000550EA2F0B2F3900075C
S214045D50E9DA487800BE4EB900073C5E4FEF0014FF
S214045D606000009E70001039001053B82F007000B9
S214045D70103900104E842F004EB9000550EA2F0B40
S214045D802F390007E9D2487800BF4EB900073C5EB9
S214045D904FEF0014606A2F39001053A22F390010F9
S214045DA04E6E4EB90005517608D400062F0B2F39D7
S214045DB00007E9CA487800C04EB900073C5E4FEFBA
S214045DC00014603C2F39001053A62F3900104E7271
S214045DD04EB90005517608D400062F0B2F3900075C
S214045DE0E9CE487800C14EB900073C5E4FEF001478
S214045DF042A742A742A74EB900073C5E4FEF000CED
S214045E004CDF1C804E5E4E754E56000048E7003848
S214045E10287C0010582A267C001061E0247C0007A9
S214045E203EE0101356000C0000666200031648801D
S214045E30D040303B00064EFB0002014C01940308A0
S214045E4000CE00FC010A011E012E018001C001D013
S214045E5002080218022C023C024C025C026A027817
S214045E6002B602C403080308030803080308030869
S214045E7003080308030803080308030803080308C1
S214045E8003080308030803080308030803080308B1
S214045E9003080308030803080308030803080308A1
S214045EA00308030803080308030803080308030891
S214045EB00308030803080308030803080308030881
S214045EC00308030803080308030803080308030871
S214045ED00308030803080308030803080308030861
S214045EE00308030803080308030803080308030851
S214045EF00308030803080308030803080308030841
S214045F00030802FC02F002D248790008582E4EB963
S214045F100007384C2F390007E8FA4EB90007384C0A
S214045F20508F4A39001048456704700160027003B8
S214045F301680600002142F390007E9124E92588F1B
S214045F40600002064EB9000477102F0C4E92588F4C
S214045F5016BC0004600001F24EB9000559202F0C4F
S214045F604E92588F600001E24EB9000478EE2F0C72
S214045F704E92588F4A3900104846670001CC16BC2A
S214045F8000FD600001C42F390010491C2F39001091
S214045F9049182F39001049144879000858482F0C1E
S214045FA04EB9000747702F0C4EB90007384C4FEF18
S214045FB0001816BC0005600001904EB9000477D0A6
S214045FC02F0C4E92588F16BC00FE6000017C2F39B1
S214045FD00007E8FA4EB90007384C588F4A390010C3
S214045FE04845670E4879000858854EB90007384C6E
S214045FF0588F16BC0006600001504EB90004795C48
S2140460002F0C4E92588F600001404EB9000479ACB4
S2140460102F0C4E92588F4A390010484666140C3995
S214046020000200104D95670A0C39000300104D95C8
S214046030660816BC00086000011016BC000F60005D
S21404604001084EB9000479FC2F0C4E92588F60005C
S21404605000F84EB900047B3C48790010587B4E92F9
S214046060588F600000E44EB900047B702F0C4E92EB
S214046070588F600000D44EB900047B942F0C4E92C7
S214046080588F600000C44EB900047BB82F0C4E92A3
S214046090588F600000B42F390007E9164E92588FC7
S2140460A0600000A62F390007E91A4E92588F600048
S2140460B000982F390007E91E4E92588F4A3900106F
S2140460C04845670616BC0063607E0C39000B00105A
S2140460D04821660616BC0010606E0C3900090010D4
S2140460E04821660616BC0011605E16BC0063605844
S2140460F04EB900055AA42F0C4E92588F604A4EB9DA
S21404610000055A562F0C4E92588F603C4A390010A0
S214046110472A670E4EB9000561562F0C4E92588FCB
S214046120602642A74E92588F601E48790008589001
S2140461304E92588F60124879000858A54E92588F90
S214046140600642A74E92588F4CDF1C004E5E4E757A
S2140461504E56FFFE7000102E000F2F007000102EFB
S214046160000B2F00610000CE1D40FFFF486EFFFFAE
S21404617061084FEF000C4E5E4E754E5600002F0C15
S214046180287C0010582A206E000810100C0000010D
S21404619067200C000003672C0C00000467380C0012
S2140461A0000567440C00000267500C000006675C9C
S2140461B0606C4879000859382F0C4EB9000071C23B
S2140461C0508F606A48790008593F2F0C4EB900007A
S2140461D071C2508F605848790008594A2F0C4EB93E
S2140461E0000071C2508F60464879000859542F0C3D
S2140461F04EB9000071C2508F603448790008595C6B
S2140462002F0C4EB9000071C2508F602248790008E6
S21404621059622F0C4EB9000071C2508F6010487935
S2140462200008596F2F0C4EB9000071C2508F285FBA
S2140462304E5E4E754E5600000C2E00FF000F67068D
S214046240122E000F6004122E000B10014E5E4E75C7
S2140462504E5600000CAEFFFFFC18000C66062D6EB2
S2140462600008000C0CAEFFFFFC18001466062D6E2A
S214046270001000142F2E00142F2E000C487900084E
S214046280597B48790010582A4EB9000747704FEFDB
S21404629000104E5E4E754E56000048790007ECF628
S2140462A0486E00104EB9000780384A40660C2D6EC2
S2140462B0000800102D6E000C0014486E00106106D5
S2140462C0588F4E5E4E754E560000206E00082F28DE
S2140462D000042F1048790008598A48790010582A73
S2140462E04EB9000747704FEF00104E5E4E754E567F
S2140462F000000CAEFFFFFC18000C66062D6E0008AE
S214046300000C486E000C6106588F4E5E4E754E5655
S2140463100000206E00082F10487900085995487927
S2140463200010582A4EB9000747704FEF000C4E5E17
S2140463304E754E5600000CAEFFFFFC18000C6606A9
S2140463402D6E0008000C486E000C6106588F4E5ED9
S2140463504E754E560000206E00082F10487900082F
S214046360599B48790010582A4EB9000747704FEFDA
S214046370000C4E5E4E754E5600000CAEFFFFFC1829
S214046380000C66062D6E0008000C486E000C6106B4
S214046390588F4E5E4E754E560000206E00082F1025
S2140463A04879000859A148790010582A4EB90007C0
S2140463B047704FEF000C4E5E4E754E5600000CAE06
S2140463C0FFFFFC18000C66062D6E0008000C486ED5
S2140463D0000C61C2588F4E5E4E754E5600000CAED1
S2140463E0FFFFFC18000C66062D6E0008000C486EB5
S2140463F0000C6100FF1A588F4E5E4E754E56000014
S2140464000CAEFFFFFC18000C66062D6E0008000C90
S214046410486E000C6106588F4E5E4E754E56000050
S214046420206E00082F104879000859A848790010F3
S214046430582A4EB9000747704FEF000C4E5E4E7553
S2140464404E56FFFE0C2E00FF000F67081D6E000F51
S214046450FFFF60061D6E000BFFFF486EFFFF610620
S214046460588F4E5E4E754E560000206E0008101073
S2140464700C000003670E0C000038671E0C0000407A
S214046480672E60424879000859AE48790010582AA9
S2140464904EB9000071C2508F60404879000859B266
S2140464A048790010582A4EB9000071C2508F602AED
S2140464B04879000859B648790010582A4EB90000A1
S2140464C071C2508F60144879000859BA4879001090
S2140464D0582A4EB9000071C2508F4E5E4E754E5605
S2140464E0FFF40C79FFFF0010537C670E7000303900
S2140464F00010537C2D40FFFC6032486EFFF54EB909
S214046500000703A4588F7000102EFFFB2D40FFFCDD
S214046510725EB0816D0C06800000076C2D40FFFC97
S214046520600A0680000007D02D40FFFC486EFFFC82
S2140465306106588F4E5E4E754E560000206E00085B
S2140465402F104879000859C248790010582A4EB9C5
S214046550000747704FEF000C4E5E4E754E56FFF820
S21404656048E703000C3900FF0010537967127C00DB
S2140465701C39001053797E001E390010537A6018B7
S214046580486EFFF94EB9000703A4588F7C001C2EF2
S214046590FFFD7E001E2EFFFE2F062F0748790008FB
S2140465A059C748790010582A4EB9000747704FEF6C
S2140465B000104CDF00C04E5E4E754E56FFF848E79E
S2140465C007000C3900FF00105376671A7A001A3950
S2140465D0001053767C001C39001053777E001E3959
S2140465E000105378601E486EFFF94EB9000703A4E6
S2140465F0588F7A001A2EFFFA7C001C2EFFFB7E00B2
S2140466001E2EFFFC2F052F062F074879000859D1A8
S21404661048790010582A4EB9000747704FEF001407
S2140466204CDF00E04E5E4E754E56FFFE0C390055AC
S2140466300010537E670A1D790010537EFFFF600822
S2140466401D79001047EEFFFF486EFFFF6106588F66
S2140466504E5E4E754E56FFFC206E000810104880A5
S21404666048C02D40FFFC2F004879000859E04879BF
S2140466700010582A4EB9000747704FEF000C4E5EC4
S2140466804E754E56FFFC0C6EFFFF000E670C700036
S214046690302E000E2D40FFFC600A7000302E000ADB
S2140466A02D40FFFC486EFFFC6106588F4E5E4E750B
S2140466B04E560000206E00082F104879000859E353
S2140466C048790010582A4EB9000747704FEF000C5F
S2140466D04E5E4E754E56FFFE0C3900FF0010537486
S2140466E0670A1D7900105374FFFF60081D790010B7
S2140466F04E5DFFFF486EFFFF6106588F4E5E4E7577
S2140467004E560000206E0008700010102F004879C6
S214046710000859E648790010582A4EB90007477011
S2140467204FEF000C4E5E4E754E56FFFE0C3900FFC2
S21404673000105384670A1D7900105384FFFF600815
S2140467401D7900104854FFFF486EFFFF6106588FFE
S2140467504E5E4E754E560000206E00084A106716B0
S2140467602F390007E8FE48790010582A4EB9000071
S21404677071C2508F60142F390007E902487900105F
S214046780582A4EB9000071C2508F4E5E4E754E5652
S214046790FFFE0C3900FF00105375670A1D790010C0
S2140467A05375FFFF60081D790010471AFFFF486EF7
S2140467B0FFFF6106588F4E5E4E754E560000206EE3
S2140467C0000870001010E2802F004879000859E98C
S2140467D048790010582A4EB9000747704FEF000C4E
S2140467E04E5E4E754E5600002F0C286E00082F394C
S2140467F0001058E24EB9000074CC588F4A806606E2
S21404680018BC00FE605008F90006001061DF20790D
S214046810001058E210100C000053671A0C00004DCC
S214046820671A0C000036671A0C00004E671A0C0034
S21404683000506718601C18BC0001601A18BC0002DF
S214046840601418BC0003600E4214600A18BC0006EC
S214046850600418BC00FF285F4E5E4E754E56FFFE61
S214046860486EFFFF6100FF7E588F0C2E00FEFFFF70
S214046870676408F90006001061DF102EFFFF0C00A5
S214046880000363060C000006663A13EEFFFF0010D2
S21404689052B070001039001052B02F002F00610063
S2140468A0F8B048790010582A2F390007E9467000D6
S2140468B01039001061E02F004EB900073C5E4FEF20
S2140468C0001460122F390007E9FA487800C94EB957
S2140468D000073660508F4E5E4E754E56FFFE2F0CE8
S2140468E0286E0008486EFFFF6100FEFA588F0C2ED3
S2140468F000FEFFFF675E08F90006001061DF102E39
S214046900FFFF0C000001630A0C00000666346000FA
S214046910000218AEFFFF700010142F002F00610055
S214046920F83048790010582A2F2E000C70001039C1
S214046930001061E02F004EB900073C5E4FEF0014D4
S21404694060122F390007E9FA487800C94EB90007E3
S2140469503660508F285F4E5E4E754E56FFFE2F0CE7
S214046960286E0008486EFFFF6100FE7A588F0C2ED2
S21404697000FEFFFF675E08F90006001061DF102EB8
S214046980FFFF0C000001630A0C000006663460007A
S214046990000218AEFFFF700010142F002F006100D5
S2140469A0F7B048790010582A2F2E000C70001039C2
S2140469B0001061E02F004EB900073C5E4FEF001454
S2140469C060122F390007E9FA487800C94EB9000763
S2140469D03660508F285F4E5E4E754E56000048E770
S2140469E00338246E000C2679001058E24878002CF0
S2140469F02F0B4EB900077A04508F2840200C6702EC
S214046A00528C200B6704200C661E2F390007E9FE03
S214046A10487800CA4EB900073660508F4292206EFE
S214046A2000084290600000942F0B4EB90007708A4D
S214046A302C002F0C4EB90007708A508F2E000C863F
S214046A400000012C6D300C870000012D6D280C868B
S214046A5000000F9F6E200C8700000FA06E184A39A6
S214046A6000104847662C0C8600000D476E080C87FD
S214046A7000000D486F1C2F390007E9FE487800CA4D
S214046A804EB900073660508F4292206E000842903E
S214046A906028BE866E1C2F390007EA02487800CAB2
S214046AA04EB900073660508F4292206E000842901E
S214046AB06008206E0008208624874CDF1CC04E5ECB
S214046AC04E754E56FFF82F39001058E24EB90000A6
S214046AD074CC588F4A80670000B2486EFFF8486E40
S214046AE0FFFC6100FEF6508F4AAEFFFC6700009C78
S214046AF00C2E0002001767080C2E000300176640D1
S214046B00202EFFFCD0AEFFF872024EB900077920A3
S214046B10222EFFF892AEFFFCD281B0816C22487917
S214046B20000859EF487800F84EB9000736602F3948
S214046B300007ECEE4EB90007384C4FEF000C604AE5
S214046B40206E000820AEFFFC206E000C20AEFFF87E
S214046B502F2EFFF82F2EFFF82F2EFFFC2F2EFFFCD4
S214046B606100F6EE08F90006001061DF48790010AF
S214046B70582A2F2E001070001039001061E02F00E4
S214046B804EB900073C5E4FEF001C4E5E4E754E56E7
S214046B90FFE048E70138286E00142F39001058E249
S214046BA04EB9000074CC588F4A806700015045EEF9
S214046BB0FFFC486EFFF82F0A6100FE20508F4A92B1
S214046BC06700013A267C0010582A202EFFF8486EEB
S214046BD0FFF04EB90007597A2012486EFFE84EB906
S214046BE00007597A48790007ECFE486EFFE8486EBD
S214046BF0FFE04EB900078170486EFFE0486EFFF074
S214046C004EB9000780384A406F5A2012486EFFF08B
S214046C104EB90007597A48790007ECFE486EFFF033
S214046C20486EFFE84EB900078170486EFFE84EB91B
S214046C3000077C682F00487900085A182F0B4EB9B5
S214046C40000747702F0B487800F94EB900073660E6
S214046C502F390007ECF24EB90007384C4FEF0018F6
S214046C606000009A2012D0AEFFF872024EB90007F8
S214046C7079202E002012D0AEFFF84EB900077920F6
S214046C802214D281B0816C34200772024EB90007F8
S214046C90792028802F00487900085A3E2F0B4EB9D9
S214046CA0000747702F0B4EB90007384C2F390007E2
S214046CB0ECEE4EB90007384C4FEF0014206E000877
S214046CC02092206E000C20AEFFF82F2EFFF82F2EF9
S214046CD0FFF82F122F126100F57808F9000600104D
S214046CE061DF2F0B2F2E001070001039001061E0AA
S214046CF02F004EB900073C5E4FEF001C4CDF1C8093
S214046D004E5E4E754E56FFF82F0C286E00082F392F
S214046D10001058E24EB9000074CC588F4A806700C1
S214046D2000882F39001058E243EEFFF84EB90007EA
S214046D304EBA588F48790007ED06486EFFF84EB9EC
S214046D40000780384A406D1448790007ED0E486EF7
S214046D50FFF84EB9000780384A406F142F390007F1
S214046D60EA06487800CB4EB900073660508F603884
S214046D7028AEFFF8296EFFFC00042F0C6100F548CE
S214046D8008F90006001061DF48790010582A2F39E8
S214046D900007E96670001039001061E02F004EB954
S214046DA000073C5E4FEF0010285F4E5E4E754E5651
S214046DB0000048E70108286E00082F39001058E242
S214046DC04EB9000074CC588F4A80675E2F39001085
S214046DD058E24EB90007708A588F2E004A876D060F
S214046DE0700CBE806F142F390007EA0A487800CC6E
S214046DF04EB900073660508F603028872F0C61002C
S214046E00F50E08F90006001061DF48790010582ACC
S214046E102F390007E96A70001039001061E02F006E
S214046E204EB900073C5E4FEF00104CDF10804E5EFC
S214046E304E754E56000048E70308286E00082F39A2
S214046E40001058E24EB9000074CC588F4A80670090
S214046E5000A62F39001058E24EB90007708A588FE2
S214046E602E002007D0802C007032BE806D080C8760
S214046E70000003E86F142F390007EA0E487800CDA7
S214046E804EB900073660508F606CBCAE000C6F368F
S214046E90202E000C72024EB9000779202F00487984
S214046EA000085A6248790010582A4EB900074770FD
S214046EB048790010582A487800F84EB9000736601A
S214046EC04FEF0014603028872F0C6100F48608F911
S214046ED00006001061DF48790010582A2F39000791
S214046EE0E97E70001039001061E02F004EB90007EB
S214046EF03C5E4FEF00104CDF10C04E5E4E754E5693
S214046F00000048E70108286E00082F39001058E2F0
S214046F104EB9000074CC588F4A80675E2F39001033
S214046F2058E24EB90007708A588F2E0070D8BE807B
S214046F306D044A876F142F390007EA12487800CE8A
S214046F404EB900073660508F603028872F0C6100DA
S214046F50F44608F90006001061DF48790010582A44
S214046F602F390007E98270001039001061E02F0005
S214046F704EB900073C5E4FEF00104CDF10804E5EAB
S214046F804E754E56000048E70108286E00082F3953
S214046F90001058E24EB9000074CC588F4A80675EE1
S214046FA02F39001058E24EB90007708A588F2E0009
S214046FB070BABE806D044A876F142F390007EA162C
S214046FC0487800CF4EB900073660508F6030288767
S214046FD02F0C6100F3C208F90006001061DF48793F
S214046FE00010582A2F390007E9867000103900105F
S214046FF061E02F004EB900073C5E4FEF00104CDFF7
S21404700010804E5E4E754E56000048E70108286E06
S21404701000082F39001058E24EB9000074CC588F7F
S2140470204A8067602F39001058E24EB90007708A0C
S214047030588F2E0070ECBE806D067014BE806F14E0
S2140470402F390007EA1A487800D04EB90007366090
S214047050508F603028872F0C6100F2B408F90006C0
S214047060001061DF48790010582A2F390007E98A92
S21404707070001039001061E02F004EB900073C5E26
S2140470804FEF00104CDF10804E5E4E754E560000DB
S21404709048E70108286E00082F39001058E24EB958
S2140470A0000074CC588F4A80675E2F39001058E26F
S2140470B04EB90007708A588F2E004A876D06706492
S2140470C0BE806F142F390007EA1E487800D14EB9E7
S2140470D000073660508F603028872F0C6100F33E1F
S2140470E008F90006001061DF48790010582A2F3985
S2140470F00007E98E70001039001061E02F004EB9C9
S21404710000073C5E4FEF00104CDF10804E5E4E755D
S2140471104E56000048E70108286E00082F39001074
S21404712058E24EB9000074CC588F4A8067602F39F5
S214047130001058E24EB90007708A588F2E00703837
S214047140BE8067067040BE80663218872F0C6100CA
S214047150F31608F90006001061DF48790010582A73
S2140471602F390007E99270001039001061E02F00F3
S2140471704EB900073C5E4FEF001060122F3900072F
S214047180EA22487800D24EB900073660508F4CDFAA
S21404719010804E5E4E754E56FFFC2F39001058E296
S2140471A04EB9000074CC588F4A8067442F390010BB
S2140471B058E24EB90007708A2D40FFFC33EEFFFEFE
S2140471C00010537C6100F31808F90006001061DF14
S2140471D048790010582A2F390007E99A70001039A8
S2140471E0001061E02F004EB900073C5E4FEF001020
S2140471F04E5E4E754E56000048E707182F390010AD
S21404720058E24EB9000074CC588F4A806700010CCF
S2140472102679001058E24878002F2F0B4EB9000745
S2140472207A04508F2840200C6702528C200B670487
S214047230200C66162F390007EA2A487800D54EB97E
S21404724000073660508F600000D22F0B4EB900073F
S214047250708A1A002F0C4EB90007708A508F1E00D1
S2140472607C00100553000C00000B62524880D0408E
S214047270303B00064EFB00020018002800180038B9
S21404728000180038001800180038001800380018D5
S2140472900C07000165280C07001F62227C01601E93
S2140472A00C07000165180C07001D62127C01600EB5
S2140472B00C07000165080C07001E62027C014A8662
S2140472C0674613C50010537A13C70010537961003C
S2140472D0F28C08F90006001061DF48790010582A7D
S2140472E02F390007E99E70001039001061E02F0066
S2140472F04EB900073C5E2F390007E9F24EB9000785
S214047300384C4FEF001060122F390007EA2A4878ED
S21404731000D54EB900073660508F4CDF18E04E5E3D
S2140473204E754E56000048E707382F39001058E2CD
S2140473304EB9000074CC588F2E00670000F62479EE
S214047340001058E24878003A2F0A4EB900077A042B
S214047350508F2840200C671A528C4878003A2F0C1D
S2140473604EB900077A04508F2640200B6706528BCE
S214047370600297CB200A66162F390007EA2E487853
S21404738000D64EB900073660508F600000A62F0A5C
S2140473904EB90007708A588F1A00200C670E2F0CFF
S2140473A04EB90007708A588F1C0060024206200BF4
S2140473B0670E2F0B4EB90007708A588F1E006002A6
S2140473C042070C050017620C0C06003B62060C070D
S2140473D0003B63142F390007EA2E487800D64EB9CE
S2140473E000073660508F604A13C50010537813C6E2
S2140473F00010537713C7001053766100F1BE08F9E6
S2140474000006001061DF48790010582A2F3900075B
S214047410E9A270001039001061E02F004EB9000791
S2140474203C5E2F390007E9F24EB90007384C4FEF9F
S21404743000104CDF1CE04E5E4E754E5600002F07C3
S2140474402F39001058E24EB9000074CC588F4A8089
S21404745067682F39001058E24EB90007708A588FB3
S2140474602E0070E9BE806D067017BE806F142F392B
S2140474700007EA32487800D74EB900073660508FC6
S214047480603813C70010537E48790010537E61009D
S214047490F1C408F90006001061DF48790010582A84
S2140474A02F390007E9A670001039001061E02F009C
S2140474B04EB900073C5E4FEF00102E1F4E5E4E7511
S2140474C04E56000048E70108286E00082F390010C1
S2140474D058E24EB9000074CC588F4A806700009674
S2140474E02F39001058E24EB90007708A588F2E00C4
S2140474F04A876D080C8700000FFF6F142F390007AA
S214047500EA36487800D84EB900073660508F606473
S2140475103887700030142F002F006100F166508FFA
S21404752008F90006001061DF0C390043001061E022
S214047530662248790010582A2F390007E9AA7000F5
S2140475401039001061E02F004EB900073C5E4FEF83
S214047550000C602048790010582A2F390007E9AE3D
S21404756070001039001061E02F004EB900073C5E31
S2140475704FEF000C4CDF10804E5E4E754E560000EA
S21404758048E70108286E00082F39001058E24EB963
S214047590000074CC588F4A8067582079001058E24F
S2140475A01E100C070041671A0C07004267142F3997
S2140475B00007EA62487800D94EB900073660508F53
S2140475C0603018872F0C6100F13808F900060010A7
S2140475D061DF48790010582A2F390007E9B2700095
S2140475E01039001061E02F004EB900073C5E4FEFE3
S2140475F000104CDF10804E5E4E754E5600002F076E
S2140476002F39001058E24EB9000074CC588F4A80C7
S214047610676A2079001058E21E100C070059671A92
S2140476200C07004E67142F390007EA66487800F7FF
S2140476304EB900073660508F60420C070059660A40
S21404764013FC000100105384600642390010538472
S2140476506100F0D608F90006001061DF48790010D2
S214047660582A2F390007E9B670001039001061E077
S2140476702F004EB900073C5E4FEF000C2E1F4E5EE7
S2140476804E754E56000048E70308286E00087C0531
S2140476902F39001058E24EB9000074CC588F4A8037
S2140476A067662F39001058E24EB90007708A588F63
S2140476B02E004A390010484667027C01BE866D06D5
S2140476C07032BE806F142F390007EA6A487800DAF1
S2140476D04EB900073660508F602E1007D000188011
S2140476E02F0C6100F0D608F90006001061DF487917
S2140476F00010582A2F390007E9BA4878003E4EB9D8
S21404770000073C5E4FEF00104CDF10C04E5E4E7517
S2140477104E56000048E70F004A3900104AAD661C72
S21404772008390001001046DC660A0839000100101A
S21404773046E46704784560067844600278554A391A
S21404774000104AAE661208390001001046DD6704D0
S2140477507A4560067A4460027A554A3900104AAF80
S214047760661208390001001046DE67047C45600690
S2140477707C4460027C554A3900104AB066120839C7
S2140477800001001046DF67047E4560067E44600202
S2140477907E551007488048C02F001006488048C011
S2140477A02F001005488048C02F001004488048C0A9
S2140477B02F00487900085A9548790010582A4EB97F
S2140477C0000747704FEF00184CDF00F04E5E4E7512
S2140477D04E56FFE848E73F002E390010499C4A39C8
S2140477E0001049A8670E2039001025AA90B9001089
S2140477F049A0DE802007223C0A4CB8004EB9000798
S21404780079722A00C1414EB900078C96C1419E8107
S2140478102007223C006DDD004EB900077972260071
S214047820C1414EB900078C96C1419E812007223C77
S2140478300001D4C04EB9000779722800C1414EB980
S21404784000078C96C1419E812007223C000007D089
S2140478504EB9000779722C0020072D40FFE8200659
S214047860C1414EB900078C96C14193AEFFE8202E65
S214047870FFE872024EB90007792024004879000810
S2140478805ADC48790010582A4EB9000071C2508F4D
S2140478904A8567262F05487900085AFB486EFFEC90
S2140478A04EB900074770486EFFEC48790010582A16
S2140478B04EB9000071A04FEF00142F022F062F04BC
S2140478C02F03487900085B03486EFFEC4EB90007A7
S2140478D04770486EFFEC48790010582A4EB90000ED
S2140478E071A04FEF00204CDF00FC4E5E4E754E56E6
S2140478F000004A390010484666302F39001048B058
S2140479002F39001048AC2F39001048A82F39001022
S21404791048A4487900085B1748790010582A4EB9DD
S214047920000747704FEF0018602E2F3900104910DB
S2140479302F390010490C2F39001049082F39001030
S2140479404904487900085B5B48790010582A4EB908
S214047950000747704FEF00184E5E4E754E560000F7
S214047960487900085B9B48790010582A4EB90007EE
S2140479704770508F0C39000100104D6A66162F3977
S2140479800007ECE248790010582A4EB9000071A0AE
S214047990508F60142F390007ECE648790010582AF7
S2140479A04EB9000071A0508F4E5E4E754E560000C4
S2140479B0487900085BBA48790010582A4EB900077F
S2140479C04770508F0C39000100104D6B66162F3926
S2140479D00007ECE248790010582A4EB9000071A05E
S2140479E0508F60142F390007ECE648790010582AA7
S2140479F04EB9000071A0508F4E5E4E754E56FFE293
S214047A00487900085BD948790010582A4EB900070F
S214047A104770508F0C39000100104D6B664870009B
S214047A20303900104D6C723C4EB9000779B02F0007
S214047A307000303900104D6C4EB9000779202F00C5
S214047A40487900085BF8486EFFE24EB900074770B5
S214047A50486EFFE248790010582A4EB9000071A01B
S214047A604FEF00186014487900085C02487900104B
S214047A70582A4EB9000071A0508F4E5E4E754E5671
S214047A80FFF848E707004A3900104D6B670000927C
S214047A904A7900104D6C67000088486EFFF94EB9AD
S214047AA0000703A4588F7E001E2EFFFA4240102EB5
S214047AB0FFFB3200C2FC003CDE814240102EFFFC7D
S214047AC03200C2FC0E10DE81DEB900104D5A0C875F
S214047AD00001518063060487000151802007223C80
S214047AE000000E104EB9000779722C00C1414EB941
S214047AF000078C96C1419E812007723C4EB9000750
S214047B0079722A002F052F06487900085C06487902
S214047B100010582A4EB9000747704FEF0010601443
S214047B202F390007E90A48790010582A4EB9000090
S214047B3071C2508F4CDF00E04E5E4E754E5600000C
S214047B40487900085C1048790010587B4EB9000745
S214047B5047706100FF2A48790010582A48790010B7
S214047B60587B4EB9000071A04FEF00104E5E4E7564
S214047B704E5600002F3900104D5E487900085C2FE1
S214047B8048790010582A4EB9000747704FEF000C8A
S214047B904E5E4E754E5600002F3900104D624879E1
S214047BA000085C5148790010582A4EB900074770FF
S214047BB04FEF000C4E5E4E754E5600002F390010E7
S214047BC04D66487900085C7348790010582A4EB907
S214047BD0000747704FEF000C4E5E4E754E56FFB0D2
S214047BE048E70138287C00104D73247C0007366073
S214047BF04A3900104D74670000D00C39000D00108F
S214047C0061E0670C0C39000E001061E0660000BAF3
S214047C10487900085C95487800E94E92508F4A39B6
S214047C200010472A6700009A7000103900104D753E
S214047C302F00700010142F007000103900104D76BD
S214047C402F007000103900104D742F00700010398A
S214047C50001061E02F00487900085CAC486EFFB065
S214047C604EB900074770486EFFB04EB9000737A0FC
S214047C707000103900104D842F0070001039001069
S214047C804D7F2F007000103900104D832F007000B8
S214047C90103900104D7E2F007000103900104D7CF6
S214047CA02F00487900085CE1486EFFB04EB9000723
S214047CB04770486EFFB04EB9000737A04FEF00403C
S214047CC042147E0C6000031A267C001058EA103911
S214047CD0001061E00C00000A65080C00000C622A23
S214047CE060640C00000465080C000005621A605607
S214047CF00C00000262000116670000E80C00000198
S214047D00660002CC6000009460520C0000106528E7
S214047D10670001780C00006165080C000062620EC2
S214047D20604A0C000011660002A6600001280C00E0
S214047D3000636600029A60240C00000E650001F0E1
S214047D406700017460162F390007EA3A487800E99C
S214047D504E92508F42147E0C6000028618BC0003BC
S214047D604213610002861E00600002764A39001043
S214047D70472A671018BC000342136100026E1E00F7
S214047D806000025E487900085D20487800E24E9262
S214047D90508F42147E0C600002484A39001025F2C7
S214047DA06716487900085D37487800E94E92508F88
S214047DB042147E0C6000022A4A39001048456710B7
S214047DC0421318BC0003610002221E006000021267
S214047DD02F390007EA76487800014E92508F6000EB
S214047DE002004A39001048456710421318BC0003C5
S214047DF0610001F81E00600001E82F390007EA76EA
S214047E00487800014E92508F600001D64A3900101F
S214047E1025F26716487900085D68487800E94E92AE
S214047E20508F42147E0C600001B84A390010484650
S214047E306710421318BC0003610001B01E00600006
S214047E4001A02F390007EA76487800014E92508F39
S214047E506000018E0C39000900104821670A0C39AD
S214047E60000B001048216610421318BC0003610082
S214047E70017A1E006000016A2F390007EA76487806
S214047E8000014E92508F600001580C39000B001010
S214047E9048216610421318BC00036100014E1E0000
S214047EA06000013E2F390007EA76487800014E92BA
S214047EB0508F6000012C700CC039001061BA671630
S214047EC0487900085D99487800E24E92508F421433
S214047ED07E0C6000010C0C39000200104D956708FA
S214047EE04A3900104846671018BC00064213610061
S214047EF000FA1E00600000EA0C39000300104D95DD
S214047F006616487900085DB8487800E24E92508FAD
S214047F1042147E0C600000CA487900085DDE48788A
S214047F2000E24E92508F42147E0C600000B4700C37
S214047F30C039001061BA6716487900085DF74878BA
S214047F4000E24E92508F42147E0C600000944A3930
S214047F5000104D6B66142F390007EA42487800F08B
S214047F604E92508F42147E0C60760C39000200103C
S214047F704D9567084A3900104846670C18BC00043B
S214047F80421361661E0060580C39000300104D95BC
S214047F9066284A39001025F26714487900085E16E8
S214047FA0487800E94E92508F42147E0C603218BC1A
S214047FB00008421361341E006026487900085E47B4
S214047FC0487800E24E92508F42147E0C6012487934
S214047FD000085E60487800E24E92508F42147E0C91
S214047FE010074CDF1C804E5E4E754E56000048E768
S214047FF003381E39001061DE287C001058EA267CFF
S21404800000104D73247C0010582A101353000C00E3
S214048010000962000E5A4880D040303B00064EFBF2
S21404802000020486091E04B00014001402C402C42C
S214048030017001700BC610140C0000056200014CA0
S2140480404880D040303B00064EFB0002000C002067
S214048050003C0080009C0122487900085E774EB9F7
S214048060000737A0588F521460000E084EB9000758
S21404807036320C0000016606521460000DF64EB946
S2140480800007199260000DEC0C39000200104D74C4
S214048090670C0C39000300104D7466000DD6700092
S2140480A030390010472E2F00487900085E8F2F0ABB
S2140480B04EB9000747702F0A4EB90007384C4FEFE9
S2140480C0001016BC0005521460000DA84EB9000737
S2140480D036320C0000016606521460000D964EB946
S2140480E00007199260000D8C0C39000300104D74C3
S2140480F0665070003039001047322F004879000867
S2140481005EA52F0A4EB9000747702F0A4EB900071E
S214048110384C4FEF00104A390010471C6710487956
S21404812000085EBB4EB90007384C588F600E48797D
S21404813000085ECF4EB90007384C588F52146000C2
S2140481400D320C39000800104D7466000D2648796F
S21404815000085EE74EB90007384C487900085F020D
S2140481604EB90007384C508F521460000D064EB9B5
S214048170000736320C0000016606521460000CF448
S2140481804EB90007199260000CEA42137E0C600098
S2140481900CE210144A00671E0C000001672C0C0049
S2140481A0000267420C00000367660C0000046700C8
S2140481B001126000012A487900085F164EB90007CC
S2140481C037A0588F521460000CAA4EB900073632F6
S2140481D00C0000016606521460000C984EB90007A5
S2140481E0199260000C8E0C39000600104D74671648
S2140481F00C39000700104D74670C0C39000A001087
S2140482004D7466000C6E16BC0009521460000C64B3
S2140482100C39000700104D74666A08390000001017
S2140482204D80670E487900085F334EB90007384C16
S214048230588F0839000100104D80670E48790008F1
S2140482405F534EB90007384C588F70003039001011
S2140482504D800280000003000C80000003006610BE
S214048260487900085F744EB90007384C588F600E82
S214048270487900085F8E4EB90007384C588F521460
S21404828060000BF00C39000A00104D74661448792F
S21404829000085FA44EB90007384C588F521460008B
S2140482A00BD20C39000800104D7466000BC64879D2
S2140482B000085FBD4EB90007384C588F5214600052
S2140482C00BB24EB9000736320C0000016606521493
S2140482D060000BA04EB90007199260000B9642137B
S2140482E07E0C60000B8E10140C000005620001B2B8
S2140482F04880D040303B00064EFB0002000C0020B5
S214048300003C006A00860188487900085FD54EB9AB
S214048310000737A0588F521460000B584EB9000758
S21404832036320C0000016606521460000B464EB945
S2140483300007199260000B3C0C39000400104D74C1
S214048340670C0C39000500104D7466000B2648793E
S21404835000085FED4EB90007384C588F16BC00076E
S214048360521460000B0E4EB9000736320C000001A2
S2140483706606521460000AFC4EB9000719926000A3
S2140483800AF2267C00104D940C39000500104D743A
S21404839066547C001C130286000000014A86671C93
S2140483A070001013E2802F00487900085FFF2F0A40
S2140483B04EB9000747704FEF000C601A7000101398
S2140483C0E2802F0048790008601D2F0A4EB9000786
S2140483D047704FEF000C2F0A4EB90007384C588FE1
S2140483E0521460000A8E0C39000800104D746600A2
S2140483F00A8248790008603B4EB90007384C700082
S2140484001013E2802F004879000860562F0A4EB9F0
S214048410000747702F0A4EB90007384C4FEF001478
S2140484204A390010472A67567000103900104D84E8
S2140484302F007000103900104D7F2F007000103987
S21404844000104D832F007000103900104D7E2F0051
S2140484507000303900104D802F0070001039001065
S2140484604D7C2F004879000860732F0A4EB9000728
S21404847047702F0A4EB9000737A04FEF0024521456
S214048480600009F04EB9000736320C00000166069B
S2140484905214600009DE4EB900071992600009D430
S2140484A042137E0C600009CC4EB9000736320C002D
S2140484B0000166140C39000100104D74660009B4FE
S2140484C042137E0C600009AC4EB900071992600096
S2140484D009A210140C0000056200045E4880D04017
S2140484E0303B00064EFB0002000C01260142023619
S2140484F0025204341039001061E00C000001674C8D
S2140485000C00000267580C00000367640C000006A9
S21404851067720C000007677C0C0000086700008682
S2140485200C0000096700008E0C00000F6700009A1C
S2140485300C000010670000B20C0000116700009ADF
S2140485400C000063670000B2600000BE2F3900070D
S214048550E9124EB9000737A0588F600000AC6100DE
S214048560F1B02F0A4EB9000737A0588F6000009A62
S2140485704EB9000559202F0A4EB9000737A0588F68
S214048580600000866100F3D62F0A4EB9000737A0B4
S214048590588F60746100F4162F0A4EB9000737A08E
S2140485A0588F60646100F4562F0A4EB9000737A04E
S2140485B0588F60546100F58648790010587B4EB990
S2140485C0000737A0588F60402F390007E91E4EB9C0
S2140485D0000737A0588F60304879000860BD4EB950
S2140485E0000737A0588F60204879000860CC4EB941
S2140485F0000737A0588F60104EB9000561562F0A41
S2140486004EB9000737A0588F5214600008664EB95A
S214048610000736320C000001660652146000085447
S2140486204EB9000719926000084A08F900040010C1
S21404863061DF1039001061E00C000009653867003E
S21404864000AA0C00001065080C000011620E607A87
S2140486500C00000F660000C2600000A00C00006161
S214048660650000B60C000062630000A00C00006306
S214048670660000A660540C0000036512673C0C00FC
S2140486800006650000940C000007624E603C0C0077
S214048690000165000084670260104879000860E203
S2140486A04EB9000737A0588F606E4879000860F30B
S2140486B04EB9000737A0588F605E487900086116E7
S2140486C04EB9000737A0588F604E48790008611EDF
S2140486D04EB9000737A0588F603E48790008612FCE
S2140486E04EB9000737A0588F602E48790008614CB1
S2140486F04EB9000737A0588F601E487900086154A9
S2140487004EB9000737A0588F600E48790008616B91
S2140487104EB9000737A0588F5214600007564EB95A
S214048720000736320C000001660652146000074447
S2140487304EB9000719926000073A4EB90007357E15
S2140487404A00660A4EB900071992600007264EB919
S2140487500007347623C0001058E24A8066222F3978
S2140487600007E9F6487800E34EB900073660508FF4
S21404877008B90005001061DF42137E0C600006F4A1
S2140487801039001061E00C0000096540670000E045
S2140487900C0000116526670000F00C0000626510EE
S2140487A0670001160C00006366000154600000FABE
S2140487B00C00006166000148600001260C00000FF2
S2140487C06500013C670000BA600000CE0C000003A0
S2140487D06516674A0C00000762000082676C0C008E
S2140487E000066600011A60500C00000165000110C6
S2140487F067026018610006864A80670816BC000295
S2140488006000010E42137E0C6000010661000874CD
S2140488104A80660000FC42137E0C600000F44EB9E9
S21404882000055B1A4A80670816BC0002600000E276
S21404883042137E0C600000DA61000A6E4A8066000D
S21404884000D042137E0C600000C861000B0A4A8008
S214048850660000BE42137E0C600000B661000BA6E4
S2140488604A80660000AC42137E0C600000A46100DF
S2140488700C4E4A806600009A42137E0C60000092FA
S21404888061000DD86000008A4EB900055FB24A80C8
S214048890667E42137E0C60784EB9000560744A808A
S2140488A0666E42137E0C60684EB9000561A44A8069
S2140488B0665E42137E0C60584879001058FE4EB926
S2140488C000056330588F4A00660642137E0C6040EB
S2140488D02F39001058FE4EB900056382588F603059
S2140488E04879001058FE4EB900056330588F4A0088
S2140488F0660642137E0C601816BC000A601248799D
S2140489000008617A4EB9000737A0588F42137E0CD0
S2140489104EB9000738725214600005584EB9000765
S21404892036320C00000166065214600005464EB945
S214048930000719926000053C42137E0C6000053463
S21404894010140C00000567160C000006672C0C00BB
S214048950000767480C000008675E600002844EB992
S214048960000736320C000001660652146000050447
S2140489704EB900071992600004FA4EB90000717AE5
S21404898008F90004001061DF4879000861914EB9C7
S2140489900007384C588F5214600004D84EB90007AC
S2140489A036320C00000166065214600004C64EB946
S2140489B000071992600004BC287C00100008247C80
S2140489C000104D954EB90006D00E0C00000166004E
S2140489D001044EB90006D1284879000861A84EB9AA
S2140489E00007384C588F16BC00014239001025F297
S2140489F04A3900104AAD66140C12000167060C12C0
S214048A000005660808F90000001046DC4A39001024
S214048A104AAE66120C39000100104D96660808F935
S214048A200000001046DD4A3900104AAF66120C39C1
S214048A30000100104D97660808F90000001046DE95
S214048A404A3900104AB066120C39000100104D98DD
S214048A50660808F90000001046DF08B90000001098
S214048A6046E408B90000001046E508B90000001006
S214048A7046E608B90000001046E74A3900104AB135
S214048A80662A13F9001046E2001046E013F90010B7
S214048A9046E3001046E113F9001046EA001046E8E3
S214048AA013F9001046EB001046E96018423900102E
S214048AB046E04239001046E14239001046E84239A1
S214048AC0001046E908AC0002000133D40040000060
S214048AD0600003A04EB90000718C0C800000012CCD
S214048AE0650003904879000861AA4EB90007384C1F
S214048AF0588F16BC00014239001025F24A3900107E
S214048B004AAD66140C12000167060C1200056608CE
S214048B1008F90000001046DC4A3900104AAE661216
S214048B200C39000100104D96660808F90000001084
S214048B3046DD4A3900104AAF66120C3900010010AF
S214048B404D97660808F90000001046DE4A39001002
S214048B504AB066120C39000100104D98660808F9F0
S214048B600000001046DF08B90000001046E408B90B
S214048B700000001046E508B90000001046E608B9F3
S214048B800000001046E74A3900104AB1662A13F975
S214048B90001046E2001046E013F9001046E3001009
S214048BA046E113F9001046EA001046E813F90010EF
S214048BB046EB001046E960184239001046E0423998
S214048BC0001046E14239001046E84239001046E9F2
S214048BD008AC0002000133D4004000006000029498
S214048BE042137E0C6000028C10140C000005672CE7
S214048BF00C000006670000BA0C000007670000CEF1
S214048C000C0000086700017C0C0000096700019056
S214048C100C00000A6700023A6000024E2F3900106A
S214048C2058FE4879000861B92F0A4EB90007477004
S214048C302F0A4EB9000737A04FEF00100CB90011E9
S214048C400000001058FE63242079001058FE3C10E3
S214048C50700010062F002F004879000861C92F0AFB
S214048C604EB9000747704FEF0010602020790010BF
S214048C7058FE700010102F002F004879000861E598
S214048C802F0A4EB9000747704FEF00102F0A4EB94F
S214048C90000737A008F90004001061DF48790008CF
S214048CA062014EB9000737A0508F5214600001C409
S214048CB04EB9000736320C000001660652146000F6
S214048CC001B24EB900071992600001A84EB9000718
S214048CD0357E4A00660A4EB9000719926000019470
S214048CE04EB90007347623C0001058E24A80662046
S214048CF0487900086212487800E34EB900073660E7
S214048D00508F08B90005001061DF42137E0C6066C0
S214048D104879001059024EB900056354588F4A002A
S214048D20662048790008621C487800014EB900079E
S214048D303660508F08B90005001061DF42137E0CC0
S214048D40603470001039001059022F002F002F399C
S214048D50001058FE48790008622D2F0A4EB9000705
S214048D60477008F90004001061DF2F0A4EB90007A7
S214048D7037A04FEF00184EB900073872521460003F
S214048D8000F24EB9000736320C0000016606521493
S214048D90600000E04EB900071992600000D64EB994
S214048DA00007357E4A00660A4EB90007199260002D
S214048DB000C24EB90007347623C0001058E22040A3
S214048DC00C10007967060C100059666C0CB900117B
S214048DD00000001058FE633042401039001059025B
S214048DE02079001058FE30803C00700010062F00DA
S214048DF02F002F084879000862562F0A4EB900073C
S214048E0047704FEF0014603E2079001058FE10B9EA
S214048E10001059022079001058FE700010102F0020
S214048E202F002F0848790008627E2F0A4EB90007E3
S214048E3047704FEF0014600E4879000862A64EB9DA
S214048E40000737A0588F4EB90007387252146022B4
S214048E504EB9000736320C00000166045214601244
S214048E604EB900071992600A42137E0C600442133E
S214048E707E0C10074CDF1CC04E5E4E754E5600002E
S214048E8048E703387C012F39001058E24EB9000039
S214048E9074CC588F2E0066067C00600001DC2679B0
S214048EA0001058E24878002C2F0B4EB900077A04BD
S214048EB0508F2840200C670E528C0C14002067F844
S214048EC00C14000967F2200B6704200C66182F396F
S214048ED00007EA46487800EA4EB900073660508F25
S214048EE07C00600001942F0B4EB90007708A588FDF
S214048EF02E007001BE806D127004BE806E0C0C14C1
S214048F000048671E0C14004C67182F390007EA4601
S214048F10487800EA4EB900073660508F7C0060003F
S214048F200158267C0007EA3E7001BE8066364A3940
S214048F3000104AAD660A0C39000100104D956714FE
S214048F402F13487800E94EB900073660508F7C002E
S214048F5060000094247C001046DC267C001046E466
S214048F60600000847002BE8066284A3900104AAE4B
S214048F7067122F13487800E94EB900073660508F01
S214048F807C006062247C001046DD267C001046E5EA
S214048F9060547003BE8066284A3900104AAF6712D0
S214048FA02F13487800E94EB900073660508F7C00CE
S214048FB06034247C001046DE267C001046E66026DC
S214048FC04A3900104AB067122F13487800E94EB9A0
S214048FD000073660508F7C00600C247C001046DF4F
S214048FE0267C001046E77001BC806600008C0C14DA
S214048FF00048663C13FC0001001025F208D300006C
S21404900008D2000008B900020010000933F9001065
S2140490100008004000002F074879000862B048792D
S2140490200010582A4EB9000747704FEF000C603AFC
S21404903013FC0001001025F20893000008920000BB
S21404904008B900020010000933F9001000080040B7
S21404905000002F074879000862C748790010582A8C
S2140490604EB9000747704FEF000C48790010582A95
S2140490704EB9000737A0588F20064CDF1CC04E5E42
S2140490804E754E56FFF848E703387E012F39001018
S21404909058E24EB9000074CC588F2C0067000200CA
S2140490A0307C0001487068004EB9000072C42D4040
S2140490B0FFFC2F39001058E22F004EB9000071C291
S2140490C02F390007ECEA2F2EFFFC4EB9000759167D
S2140490D028402F390007ECEA42A74EB90007591674
S2140490E024402F390007ECEA42A74EB90007591668
S2140490F02D40FFF82F390007E8FA42A74EB90007BB
S21404910059164FEF002C2640200C670E200A670ADB
S2140491104AAEFFF86704200B66182F390007EA4AA0
S214049120487800EB4EB900073660508F7E0060002A
S21404913001620C14004567060C14004466280C12E1
S214049140004567060C120044661C206EFFF80C10DF
S214049150004567060C100044660C0C130045671E99
S2140491600C13004467182F390007EA4A487800EBC6
S2140491704EB900073660508F7E00600001164A39EB
S21404918000104AAD66660C14004566280C390002C9
S21404919000104D95670A0C39000300104D95660AB9
S2140491A008F90001001046E4603008F900010010D8
S2140491B046DC60260C39000200104D95670A0C390F
S2140491C0000300104D95660A08B90001001046E435
S2140491D0600808B90001001046DC08B90002001057
S2140491E0000933F900100008004000004A39001056
S2140491F04AAE6628287C001046DD0C12004566063A
S21404920008D4000160040894000108B900020010A4
S214049210000933F900100008004000004A39001025
S2140492204AAF662C287C001046DE206EFFF80C1031
S2140492300045660608D4000160040894000108B9D5
S21404924000020010000933F9001000080040000076
S2140492504A3900104AB06628287C001046DF0C13F2
S2140492600045660608D4000160040894000108B9A5
S21404927000020010000933F9001000080040000046
S2140492806100E48E48790010582A4EB9000737A0CA
S214049290588F2F2EFFFC4EB9000071DE588F200722
S2140492A04CDF1CC04E5E4E754E56000048E7010863
S2140492B07E012F39001058E24EB9000074CC588F46
S2140492C04A8067000088287C00104D6A20790010C8
S2140492D058E210100C00004467080C000045672C88
S2140492E060564214487800012F0C48790080081E06
S2140492F04EB90006A09E6100E66448790010582A1C
S2140493004EB9000737A04FEF0010604018BC0001AC
S214049310487800012F0C48790080081E4EB90006D4
S214049320A09E6100E63848790010582A4EB9000716
S21404933037A04FEF001060142F390007EA4E487824
S21404934000EC4EB900073660508F7E0020074CDFD5
S21404935010804E5E4E754E56000048E701087E01AA
S2140493602F39001058E24EB9000074CC588F4A804A
S21404937067000088287C00104D6B2079001058E2A6
S21404938010100C00004467080C000045672C60565B
S2140493904214487800012F0C4879008008204EB902
S2140493A00006A09E6100E60648790010582A4EB9C9
S2140493B0000737A04FEF0010604018BC0001487843
S2140493C000012F0C4879008008204EB90006A09EA4
S2140493D06100E5DA48790010582A4EB9000737A02C
S2140493E04FEF001060142F390007EA56487800ED56
S2140493F04EB900073660508F7E0020074CDF108081
S2140494004E5E4E754E56000048E707187C012F390D
S214049410001058E24EB9000074CC588F4A8067009A
S21404942000942679001058E22F0B4EB90007708A74
S2140494303A004878003A2F0B4EB900077A044FEFEB
S214049440000C2840200C6710528C2F0C4EB90007D5
S214049450708A588F3E00600242470C4500186240EE
S2140494600C47003B623A3005C0FC003CD04733C092
S21404947000104D6C48780002487900104D6C48790D
S21404948000800DF04EB90006A09E6100E570487994
S2140494900010582A4EB9000737A04FEF001060148A
S2140494A02F390007EA5A487800EE4EB900073660AE
S2140494B0508F7C0020064CDF18E04E5E4E754E56EC
S2140494C0FFF248E723387C012F39001058E24EB9E2
S2140494D0000074CC588F2E0067000176307C0001A3
S2140494E0487078004EB9000072C424402F3900102A
S2140494F058E22F0A4EB9000071C24879000862DDAE
S2140495002F0A4EB90007591626404879000862DF2C
S21404951042A74EB9000759164FEF001C2840200BEF
S2140495206704200C66182F390007EA2E487800D600
S2140495304EB900073660508F7C006000010A2F0B7E
S2140495404EB90007708A1D40FFFF2F0C4EB9000766
S214049550708A508F1D40FFFE0C2E0017FFFF620618
S2140495600C00003B63182F390007EA5E487800EFCA
S2140495704EB900073660508F7C00600000CA4878F9
S2140495800001486EFFFF4879008008244EB90006A3
S214049590A09E48780001486EFFFE487900800826A1
S2140495A04EB90006A09E287C00104D6E7000102E4A
S2140495B0FFFF223C00000E10C1414EB900078C96F6
S2140495C0C1417000102EFFFE743C2D41FFF22202B2
S2140495D0C1414EB900078C96C141D2AEFFF2288134
S2140495E0486EFFF74EB9000703A44FEF001C7E0039
S2140495F01E2EFFF87000102EFFF922024EB9000747
S2140496008C96DE807000102EFFFA223C00000E10AE
S214049610C1414EB900078C96C141DE812014B08743
S214049620640806800001518028802014908723C097
S21404963000104D5A6100E50648790010587B4EB973
S214049640000737A0588F2F0A4EB9000071DE588FD6
S21404965020064CDF1CC44E5E4E754E5600002F3955
S214049660001058E24EB9000074CC588F4A80672226
S2140496702079001058E210100C00005967026004AC
S2140496806114600E4879000862E14EB9000737A0FD
S214049690588F4E5E4E754E56FFFC48E7001847EE50
S2140496A0FFFC429342B900104864287C0006A24C92
S2140496B0487800044879001048644879006020F02F
S2140496C04E9442B90010486848780004487900105F
S2140496D048684879006020F84E9442B90010486CF7
S2140496E04878000448790010486C487900602100E6
S2140496F04E9442B900104870487800044879001027
S21404970048704879006021084E9442B900104874A5
S214049710487800044879001048744879006021109D
S2140497204E9442B9001048784878000448790010EE
S21404973048784879006021184E944FEF004842B9A3
S2140497400010487C4878000448790010487C487922
S214049750006021204E9442B90010488048780004E6
S2140497604879001048804879006021284E9442B910
S21404977000104884487800044879001048844879E2
S214049780006021304E9442B900104888487800049E
S2140497904879001048884879006021384E9442B9C8
S2140497A00010488C4878000448790010488C4879A2
S2140497B0006021404E9442B9001048904878000456
S2140497C04879001048904879006021484E944FEF3D
S2140497D0004842B9001048944878000448790010BC
S2140497E048944879006021504E9442B90010489835
S2140497F04878000448790010489848790060215851
S2140498004E9442B90010489C4878000448790010E9
S214049810489C4879006021604E9442B9001048A0E4
S214049820487800044879001048A048790060216808
S2140498304E9442B9001048A44878000448790010B1
S21404984048A44879006021704E9442B9001048A894
S214049850487800044879001048A8487900602178C0
S2140498604E944FEF004842B9001048AC48780004C4
S2140498704879001048AC4879006021804E9442B97B
S214049880001048B0487800044879001048B0487979
S214049890006021884E9442B9001048B44878000409
S2140498A04879001048B44879006021904E9442B933
S2140498B0001048B8487800044879001048B8487939
S2140498C0006021984E9442B9001048BC48780004C1
S2140498D04879001048BC4879006021A04E9442B9EB
S2140498E0001048C0487800044879001048C04879F9
S2140498F0006021A84E944FEF004842B9001048C4B7
S214049900487800044879001048C44879006021B0BB
S2140499104E9442B9001048C84878000448790010AC
S21404992048C84879006021B84E9442B9001048CC23
S214049930487800044879001048CC4879006021C073
S2140499404E9442B9001048D0487800044879001074
S21404995048D04879006021C84E9442B9001048D4D3
S214049960487800044879001048D44879006021D02B
S2140499704E9442B9001048D848780004487900103C
S21404998048D84879006021D84E944FEF004842B931
S214049990001048DC487800044879001048DC487910
S2140499A0006021E04E9442B9001048E04878000474
S2140499B04879001048E04879006021E84E9442B99E
S2140499C0001048E4487800044879001048E44879D0
S2140499D0006021F04E9442B9001048E8487800042C
S2140499E04879001048E84879006021F84E9442B956
S2140499F0001048EC487800044879001048EC487990
S214049A00006022004E9442B9001048F048780004E2
S214049A104879001048F04879006022084E944FEFC9
S214049A20004842B9001048F4487800044879001009
S214049A3048F44879006022104E9442B9001048F861
S214049A40487800044879001048F8487900602218DD
S214049A504E9442B9001048FC487800044879001037
S214049A6048FC4879006022204E9442B90010490010
S214049A704878000448790010490048790060222894
S214049A804E9442B900104D5E4878000448790010A0
S214049A904D5E4879006020D84E9442B900104D625D
S214049AA048780004487900104D624879006020E048
S214049AB04E944FEF004842B900104D6648780004B3
S214049AC0487900104D664879006020E84E944FEFC0
S214049AD0000C42B90010499C4AB9001049A0670A14
S214049AE023F9001025AA001049A0487800044879F4
S214049AF00010499C4879006022904E9442B90010A8
S214049B00496C4878000448790010496C487900602C
S214049B1022304E9442B900104970487800044879BF
S214049B20001049704879006022384E9442B90010FB
S214049B3049744878000448790010497448790060EC
S214049B4022404E9442B90010497848780004487977
S214049B50001049784879006022484E9442B90010B3
S214049B60497C4878000448790010497C48790060AC
S214049B7022504E944FEF004842B90010498048786E
S214049B8000044879001049804879006022584E94B1
S214049B9042B9001049844878000448790010498482
S214049BA04879006022604E9442B90010498848788B
S214049BB000044879001049884879006022684E9469
S214049BC042B90010498C4878000448790010498C42
S214049BD04879006022704E9442B900104990487843
S214049BE000044879001049904879006022784E9421
S214049BF042B9001049944878000448790010499402
S214049C004879006022804E944FEF004842B9001015
S214049C1049984878000448790010499848790060C3
S214049C2022884E9442B900104904487800042F0B49
S214049C304879006022A64E9442B900104908487834
S214049C4000042F0B4879006022AE4E9442B90010EF
S214049C50490C487800042F0B4879006022B64E94CD
S214049C6042B900104910487800042F0B4879006068
S214049C7022BE4E9442B900104914487800042F0BB3
S214049C804879006022C64E944FEF004842B900104F
S214049C904918487800042F0B4879006022CE4E9469
S214049CA042B90010491C487800042F0B487900601C
S214049CB022D64E9442B900104920487800042F0B4F
S214049CC04879006022DE4E9442B900104924487850
S214049CD000042F0B4879006022E64E9442B9001027
S214049CE04928487800042F0B4879006022EE4E94E9
S214049CF042B90010492C487800042F0B48790060BC
S214049D0022F64E944FEF004842B900104930487886
S214049D1000042F0B4879006022FE4E9442B90010CE
S214049D204934487800042F0B4879006023064E9483
S214049D3042B900104938487800042F0B487900606F
S214049D40230E4E9442B90010493C487800042F0B69
S214049D504879006023164E9442B90010494048786A
S214049D6000042F0B48790060231E4E9442B900105D
S214049D704944487800042F0B4879006023264E9403
S214049D804FEF004842B900104948487800042F0BAA
S214049D9048790060232E4E9442B90010494C487806
S214049DA000042F0B4879006023364E9442B9001005
S214049DB04950487800042F0B48790060233E4E949F
S214049DC042B900104954487800042F0B48790060C3
S214049DD023464E9442B900104958487800042F0B85
S214049DE048790060234E4E9442B90010495C487886
S214049DF000042F0B4879006023564E944FEF00481A
S214049E0042B900104960487800042F0B4879006076
S214049E10235E4E9442B900104964487800042F0B20
S214049E204879006023664E9442B900104968487821
S214049E3000042F0B48790060236E4E9442B900103C
S214049E40472642B900104834487800042F0B487956
S214049E50006023764E944879001049AA4EB900074C
S214049E6003A4487800074879001049AA4879006096
S214049E7022984E944FEF00404CDF18004E5E4E750D
S214049E804E56000023FC006000000010256248784F
S214049E9000044879001025624879006020D04EB945
S214049EA00006A24C4279001049B24878000248796C
S214049EB0001049B248790060237E4EB90006A24CD1
S214049EC04FEF00184E5E4E754E56000048E70F00E2
S214049ED04A3900105385671A1839001053861A3900
S214049EE0001053871C39001053881E3900105389FC
S214049EF060181839001047CA1A39001047CB1C39A5
S214049F00001047CC1E39001047CD700010072F00F4
S214049F10700010062F00700010052F00700010044B
S214049F202F004879000862F548790010582A4EB97F
S214049F30000747704FEF00184CDF00F04E5E4E757A
S214049F404E56FFFC48E70F382F39001058E24EB93A
S214049F50000074CC588F4A806700010C2D790010DD
S214049F6058E2FFFC4878002E2F2EFFFC4EB900075F
S214049F707A04508F2640200B6702528B4878002EB6
S214049F802F0B4EB900077A04508F2840200C670226
S214049F90528C4878002E2F0C4EB900077A04508F46
S214049FA02440200A6702528A2F2EFFFC4EB900076F
S214049FB0708A28002F0B4EB90007708A2A002F0CCF
S214049FC04EB90007708A2C002F0A4EB90007708A13
S214049FD04FEF00102E004A846D2C0C84000000FF06
S214049FE06E244A856D200C85000000FF6E184A8694
S214049FF06D140C86000000FF6E0C4A876D080C87F3
S21404A000000000FF6F142F390007EA36487800D89E
S21404A0104EB900073660508F604C13C40010538648
S21404A02013C50010538713C60010538813C70010B7
S21404A030538913FC0001001053856100FE8C08F957
S21404A0400006001061DF48790010582A2F390007EF
S21404A050E9E670001039001061E02F004EB90007E1
S21404A0603C5E4FEF000C4CDF1CF04E5E4E754E56B9
S21404A070000048E70138267C001061DE0C1300104F
S21404A08066086100152A60000400287C00106AB087
S21404A090247C00106ABD0C13000A670001680C13C8
S21404A0A00007670001600C130008670001580C13D2
S21404A0B0000B670001500C13001166400C390010A9
S21404A0C000105904660E4239001052A24EB9000719
S21404A0D0254060064EB9000723DC0C390013001037
S21404A0E05904670A0C3900090010590466040892DA
S21404A0F000010C130011660416BC000108390007A1
S21404A100001061DF6704420760144EB90006D00EE3
S21404A1101E00670A4EB90006D128205410804A074C
S21404A120670000E20812000466280812000066228F
S21404A13008120005661C20540C10001167140C103D
S21404A1400013670E700010102F004EB900071F1E74
S21404A150588F20540C10006165140C10007A620E9F
S21404A16008390000001061DF660404100020700047
S21404A17010120280000000107210B081660C205489
S21404A1804210089200045394607020540C10000D82
S21404A190660A4210610002FA5394605E0C10000ACC
S21404A1A066064210539460520C10000867060C10A2
S21404A1B0007F660C0C94001061E8673E5594603A84
S21404A1C00C100013660E4210539408F90001001098
S21404A1D06ABE60260C100011660E4210539408B92D
S21404A1E0000100106ABE60124A106606538828886A
S21404A1F060084A13660416BC00010C9400106246FC
S21404A200640252940C9400106239653408390000D4
S21404A210001061BA672A0839000000106ABE66207A
S21404A2204EB90006D2460C000001661448780013A6
S21404A2304EB90006D270588F08F9000000106ABEA6
S21404A2400C9400106239644408390000001061BAA6
S21404A250673A7000103900106ABE028000000001E0
S21404A2607201B08166264EB90006D2460C00000183
S21404A270660000F0487800114EB90006D270588F78
S21404A28008B9000000106ABE600000D80839000152
S21404A29000106ABE660000C4081200046710203965
S21404A2A000106AB4B0B900106AB8640000AE207931
S21404A2B000106AB44A10670000AA4EB90006D246D7
S21404A2C00C000001661A207900106AB470001010A1
S21404A2D02F004EB90006D270588F52B900106AB4D7
S21404A2E0203900106AB4538023C0001061E220793C
S21404A2F000106AB44A10662020404A10671A70009C
S21404A3001039001061DF0280000000207220B08146
S21404A31066064EB9000723DC4A13660E2079001041
S21404A3206AB44A10670416BC0001207900106AB4A7
S21404A3304A10661C23FC001062B000106AB4207930
S21404A34000106AB4421008B90007001061DF6012FA
S21404A35008F90007001061DF600808B9000700105C
S21404A36061DF0C130001661220544A10660C207933
S21404A37000106AB44A10660242134A136600010AC1
S21404A3800812000466000102700010120280000029
S21404A39000027202B081660000BA10390010590437
S21404A3A053000C000014620000A44880D040303BE8
S21404A3B000064EFB0002002A0032003A0042004A21
S21404A3C00062009600960068009600960096009636
S21404A3D000960096009600840096008A00960090E8
S21404A3E0610005EA600000A216BC00026000009A44
S21404A3F016BC00036000009216BC00046000008ACD
S21404A400700010120280000000087208B08166080E
S21404A4104EB90007458E607016BC0005606A700071
S21404A42010120280000000087208B08166066100FF
S21404A43012FC605416BC000D604E16BC000E60483C
S21404A44016BC000D604216BC0012603C0892000167
S21404A4506036700010120280000000207220B08166
S21404A46066124EB90000718C7201B081651A6100E3
S21404A47008806014700010120280000000407240D1
S21404A480B081660461000BF84CDF1C804E5E4E758E
S21404A4904E56000048E70338247C001061E82F0A73
S21404A4A04EB9000074CC588F1C00267C001059044A
S21404A4B00C1300076608610010F6600004980C137D
S21404A4C0000B6608610008786000048A0C13000D0F
S21404A4D0660861000CE46000047C0C13000F660838
S21404A4E061000B1C6000046E4A0666104EB9000735
S21404A4F023DC23CA00106AB06000045A0C12004120
S21404A50065060C12005A63080C12003F6600041419
S21404A510287C00106ABD0C060001660003640C1358
S21404A5200009664C10120C00005667140C00003F1D
S21404A53067160C00004867140C0000516716602666
S21404A540610013326000040E08940000610011B428
S21404A5506000040223F90007ED1600106AD26100B9
S21404A560044C600003F04EB90007243E600003E686
S21404A5701012060000C10C000015620002FA4880A2
S21404A580D040303B00064EFB000202A202EC002C38
S21404A59002EC0034003C00440274029202A602EC70
S21404A5A002EC02EC02AE029A02EC02EC02EC02BCF2
S21404A5B002C402CC02DC6100071460000398610048
S21404A5C0077E600003906100072860000388700C13
S21404A5D0C039001061BA6600020A42A74EB90006E6
S21404A5E0D4B408B90002001046DF70001039001019
S21404A5F046D9E880C039001046DF13C0001046EF85
S21404A6004878000270001039001046EF2F00487892
S21404A61000684EB900065F56287C001046DC089495
S21404A6200002700FC039001046D9C039001046DE4B
S21404A63013C0001046EE4878000170001039001070
S21404A64046EE2F00487800484EB900065F56089438
S21404A6500002700FC039001046D8C01413C0001092
S21404A66046EC4878000370001039001046EC2F00C2
S21404A670487800084EB900065F56267C001046DD72
S21404A6800893000270001039001046D8E880C01302
S21404A69013C0001046ED487800047000103900100E
S21404A6A046ED2F00487800284EB900065F564FEF57
S21404A6B000343E3C0FA060104EB900056B384EB90E
S21404A6C0000070505347670A08390006002000014E
S21404A6D066E613FC00010010209E4EB9000404DA5E
S21404A6E04EB900061A3A3E3C0FA0600A4EB9000066
S21404A6F070505347670A083900050020000166ECCD
S21404A7004EB9000057D242390010209E08F90002C4
S21404A710001046DF70001039001046D9E880C039B2
S21404A720001046DF13C0001046EF487800027000A1
S21404A7301039001046EF2F00487800684EB900061E
S21404A7405F5608D40002700FC039001046D9C039CD
S21404A750001046DE13C0001046EE48780001700074
S21404A7601039001046EE2F00487800484EB900060F
S21404A7705F5608D40002700FC039001046D8C014C3
S21404A78013C0001046EC487800037000103900101F
S21404A79046EC2F00487800084EB900065F5608D3EA
S21404A7A0000270001039001046D8E880C01313C0A9
S21404A7B0001046ED4878000470001039001046ED8D
S21404A7C02F00487800284EB900065F5648780001E6
S21404A7D04EB90006D4B44FEF00344EB90006D490F8
S21404A7E0601248790008631A487800E24EB90007F8
S21404A7F03660508F4EB9000723DC6000015813FC06
S21404A8000059001061E016BC000F13FC000900108C
S21404A81061DE423900106AC86000013A610007F838
S21404A82060000132610008246000012A08940000D8
S21404A8306100017A6000011E089400004EB900070A
S21404A84023DC6000011061000672600001086100EC
S21404A85004C46000010013FC00AA001052A36100A7
S21404A8600EA2600000F013FC0055001052A3610015
S21404A8700E92600000E04EB90007243E600000D649
S21404A8800C060002666E0C12005366160C3900564F
S21404A890001061E9660C13FC000A001061DE60001B
S21404A8A000B4700010140280000000017201B08130
S21404A8B066240C12005566160C390041001061E936
S21404A8C0660C16BC0001610007B6600000884EB92D
S21404A8D00007243E607E0C12005366100C390046B6
S21404A8E0001061E9660608D4000060684EB90007E7
S21404A8F0243E6060700010140280000000017201A3
S21404A900B08166160C12004466100C390044001020
S21404A91061E96606610007AC603A4EB90007243E5A
S21404A92060320C12003065260C12003962200C06C8
S21404A930000363084EB90007243E60180C13000990
S21404A940660661000F5C600C610005B460064EB9D3
S21404A9500007243E0C390007001061DE67464207F4
S21404A960287C001061E2267C001061E660207000FE
S21404A970100772001206D081D08A288020401690D4
S21404A98070001007D08A28802040109352071006C3
S21404A990440006000060BE0065D47000100691B93D
S21404A9A000106AB04CDF1CC04E5E4E754E5600005A
S21404A9B013FC00010010590408F9000100106ABDD8
S21404A9C04239001061E061044E5E4E754E5600003A
S21404A9D048E70038287C00106ABD267C001061E039
S21404A9E0247C000737A010130C00000E620002AE91
S21404A9F04880D040303B00064EFB0002001E003666
S21404AA000064009200C000EE011C014A017801A611
S21404AA1001D402020230025C027E081400006612B0
S21404AA204879000863384E92588F16BC00016000BF
S21404AA30028C700010140280000000017201B081C4
S21404AA40660C48790008634F4E92588F600A48791E
S21404AA50000863514E92588F16BC00026000025ED6
S21404AA60700010140280000000017201B081660CB0
S21404AA7048790008636D4E92588F600A487900083A
S21404AA80636F4E92588F16BC00036000023070004D
S21404AA9010140280000000017201B081660C48792F
S21404AAA0000863914E92588F600A487900086393B1
S21404AAB04E92588F16BC00046000020270001014F8
S21404AAC00280000000017201B081660C487900081B
S21404AAD063CA4E92588F600A4879000863CC4E9237
S21404AAE0588F16BC0005600001D470001014028054
S21404AAF0000000017201B081660C4879000863EB1F
S21404AB004E92588F600A4879000863ED4E92588F2B
S21404AB1016BC0006600001A6700010140280000037
S21404AB2000017201B081660C48790008640B4E92ED
S21404AB30588F600A48790008640D4E92588F16BCE8
S21404AB400007600001787000101402800000000105
S21404AB507201B081660C4879000864274E92588FBB
S21404AB60600A4879000864294E92588F16BC00087B
S21404AB706000014A70001014028000000001720197
S21404AB80B081660C48790008644A4E92588F600A71
S21404AB9048790008644C4E92588F16BC0009600031
S21404ABA0011C700010140280000000017201B081C4
S21404ABB0660C4879000864694E92588F600A487992
S21404ABC00008646B4E92588F16BC000A600000EEB4
S21404ABD0700010140280000000017201B081660C3F
S21404ABE048790008648C4E92588F600A48790008A9
S21404ABF0648E4E92588F16BC000B600000C0700026
S21404AC0010140280000000017201B081660C4879BD
S21404AC10000864B94E92588F600A4879000864BBED
S21404AC204E92588F16BC000C6000009270001014F0
S21404AC300280000000017201B081660C48790008A9
S21404AC4064E44E92588F600A4879000864E64E928F
S21404AC50588F16BC000D606408140000670C487911
S21404AC60000865014E92588F600A4879000865040A
S21404AC704E92588F16BC000E604208140000670CF3
S21404AC8048790008652D4E92588F600A4879000866
S21404AC9065304E92588F16BC000F602008F90004E9
S21404ACA0001061DF4879000865584E92588F08F9FD
S21404ACB00005001061DF08940001421313FC000134
S21404ACC0001061DE4CDF1C004E5E4E754E560000D2
S21404ACD013FC00020010590408F9000100106ABDB4
S21404ACE04239001061E0423900106AC84E5E4E7563
S21404ACF04E56000013FC00030010590408F9000126
S21404AD0000106ABD4239001061E0423900106AC87A
S21404AD104E5E4E754E56000013FC00060010590495
S21404AD2008F9000100106ABD4239001061E042399A
S21404AD3000106ABF423900106AC84E5E4E754E5601
S21404AD40000048E70038287C001061DF267C0010ED
S21404AD506AC7247C001059040C12000B660000EE2F
S21404AD604879001061E84EB9000074CC588F4A80C8
S21404AD70661A14BC000148790008655A487800072A
S21404AD804EB900073660508F600000FE2F39000869
S21404AD9024E44879001061E84EB9000758B0508F93
S21404ADA04A80664C08D400047000103900106ABD4E
S21404ADB00280000000017201B08166104879000824
S21404ADC065724EB9000737A0588F600E48790008A0
S21404ADD065744EB9000737A0588F487900106AD6B4
S21404ADE04EB9000737A0588F610003CE6000009A62
S21404ADF052130C130003661C14BC000148790008A7
S21404AE006589487800054EB900073660508F08D427
S21404AE100005607408D400047000103900106ABD80
S21404AE200280000000017201B08166102F3900080C
S21404AE3024F84EB9000737A0588F604C2F39000805
S21404AE4024EC4EB9000737A0588F603C08D40004A1
S21404AE507000103900106ABD028000000001720103
S21404AE60B08166102F39000824F84EB9000737A0C1
S21404AE70588F600E2F39000824EC4EB9000737A00F
S21404AE80588F421314BC000B4CDF1C004E5E4E75EC
S21404AE904E5600000C39000500105904670A0C3998
S21404AEA000070010590466084EB90007456E600690
S21404AEB04EB90007243E4E5E4E754E56000013FCF7
S21404AEC0000B001061DE13FC00100010590423F977
S21404AED0000824D400106AD24E5E4E754E5600000A
S21404AEE008F9000100106ABD4239001061E04239D9
S21404AEF000106ABF423900106AC84E5E4E754E5640
S21404AF00000048E70018287C001061E228BC001006
S21404AF1061E8267C001061E04213602A20540C107D
S21404AF20003065060C100039630616BC00FF60206E
S21404AF3042401013323C000AC2C0103C00D0D0106D
S21404AF40D200168152942014B0B900106AB065CCB1
S21404AF50612A4A0066084EB900072472601013FC82
S21404AF60000F0010590413FC0009001061DE42397A
S21404AF7000106AC84CDF18004E5E4E754E56000030
S21404AF80227C001061E00C110001650A0C110050CF
S21404AF906204720160620C110078650A0C11008369
S21404AFA06204720160520C11005B650A0C11006D9C
S21404AFB06204720160420C11008C650A0C11009345
S21404AFC06204720160320C110096650A0C11009D31
S21404AFD06204720160220C1100A0650A0C1100A81C
S21404AFE06204720160120C1100AB650A0C1100BFFA
S21404AFF0620472016002420110014E5E4E754E56A6
S21404B000000013FC0007001061DE13FC00050010AE
S21404B01059044E5E4E754E56000013FC0013001085
S21404B020590413FC000D001061DE13FC00AA001086
S21404B03052A308F9000100106ABD4239001061E00D
S21404B040423900106AC84E5E4E754E56000013FC18
S21404B05000130010590413FC000D001061DE13FCED
S21404B0600055001052A308F9000100106ABD4239C9
S21404B070001061E0423900106AC84E5E4E754E56A6
S21404B08000001039001059040C000001670E0C0073
S21404B090000267160C0000036716601A08F900061B
S21404B0A000106ABD6100FC2660146100FC44600E5A
S21404B0B06100FC62600808B9000600106ABD4E5EB6
S21404B0C04E754E56000048E700380C39002C001028
S21404B0D061EA660000DC287C001061E228BC0010EF
S21404B0E061EB267C001061E016BC00FF247C001097
S21404B0F06AB0605E20540C10002C660652882888BD
S21404B10060560C10002067060C100009660A0C1323
S21404B11000FF66045294603A20540C100030650612
S21404B1200C100039630616BC00FF602C0C1300FFDD
S21404B130660A103C00D0D0101680601442401013EB
S21404B140323C000AC2C0103C00D0D010D200168197
S21404B15052942014B092659C6100FE224A00660850
S21404B1604EB9000724726048267C001061E642133C
S21404B170601A22545213103C00FFD01372001200BF
S21404B1800681001061E82041109928892014B092A5
S21404B19063E07000101353800680001061E824807A
S21404B1A013FC0007001061DE13FC000500105904B0
S21404B1B04CDF1C004E5E4E754E56000048E70038C5
S21404B1C0247C00106AC00C39000D00105904660077
S21404B1D001444239001061EE4879001061E84EB926
S21404B1E0000074CC588F4A80661E13FC00010010C1
S21404B1F0590448790008659A487800074EB900074C
S21404B2003660508F600001540C12002A665048794C
S21404B210001061E82F0A4EB9000071C2508F08F979
S21404B2200004001061DF7000103900106ABD02804F
S21404B230000000017201B08166122F39000824F85C
S21404B2404EB9000737A0588F600001102F39000848
S21404B25024F44EB9000737A0588F600000FE4879E2
S21404B260001061E82F0A4EB9000758B0508F4A8084
S21404B270667C2F0A487900106AD64EB9000071C25F
S21404B280487800072F0A4879008000004EB9000667
S21404B290A09E4FEF0014267C001061E74213287C22
S21404B2A0001061E642146012720012140681001047
S21404B2B06AD620411010D11352140C14000765E806
S21404B2C013D300106ADD48780001487900106ADD5F
S21404B2D048790080000E4EB90006A09E4879000802
S21404B2E065B24EB90007384C4FEF0010601248792B
S21404B2F0000865C4487800064EB900073660508FCB
S21404B30013FC00010010590408F90005001061DF61
S21404B3104212604608F90004001061DF700010391C
S21404B32000106ABD0280000000017201B081661040
S21404B3302F39000824F84EB9000737A0588F600E3E
S21404B3402F39000824F04EB9000737A0588F14BCD4
S21404B350002A13FC000D001059044CDF1C004E5E3E
S21404B3604E754E56000048E70038287C001061E20F
S21404B370246E000828B900106AB46002529420545F
S21404B3804A1066F8267C001061E616B9001061E0E3
S21404B3907000101372644EB900077920060000305E
S21404B3A0205410C02888700010134EB9000779B0D6
S21404B3B0168070001013720A4EB900077920060032
S21404B3C00030205410C02888700010134EB90007AF
S21404B3D079B0168006000030205410C0288808393A
S21404B3E0000000106ABD664410FC0020288810FC8B
S21404B3F00020288842136008205410DA2888521344
S21404B4004A1267120C13001065EE600A205410FCF2
S21404B4100020288852130C13001065F0205410FCEA
S21404B4200020288810FC00202888600610FC002CC9
S21404B430288842136010226E000C205410D92888E5
S21404B4402D49000C5213206E000C4A1067060C138C
S21404B450003765E2205410FC000D288810FC000A12
S21404B4602888600E226E0010205410D928882D4992
S21404B4700010206E00104A1067080C9400106AAA88
S21404B48065E2205410FC003E288842105239001011
S21404B4906AC813FC000F0010590413FC00010010C6
S21404B4A061DE4CDF1C004E5E4E754E56000048E7CB
S21404B4B00108287C001061E21E2E000B226E000C90
S21404B4C028B900106AB46002529420544A1066F8F0
S21404B4D07000100772644EB9000779200600003029
S21404B4E0205410C02888700010074EB9000779B0A1
S21404B4F01E0070001007720A4EB900077920060075
S21404B5000030205410C02888700010074EB9000779
S21404B51079B01E007030D007205410C0288808392F
S21404B520000000106ABD662A10FC0020288810FC63
S21404B530002028886006205410D928884A1166F608
S21404B5400C39000A00106ABC670808F900050010E8
S21404B55061DF205410FC000D288810FC000A28889F
S21404B5604210523900106AC8287C001059040C1482
S21404B570000F670C0C14000B67060C14000D660411
S21404B58018BC0005287C001061DE0C140007671642
S21404B5900C14000867100C14000A670A0C14000B3D
S21404B5A0670418BC00014CDF10804E5E4E754E5684
S21404B5B000000C39000700105904660000FA4879A8
S21404B5C0001061E84EB9000074CC588F4A80662497
S21404B5D013FC000100106ABC423900105904487973
S21404B5E0000865DA487800074EB900073660508FC1
S21404B5F06000010C487900106AD64879001061E8AA
S21404B6004EB9000758B0508F4A8067182F39000883
S21404B61024E44879001061E84EB9000758B0508F0A
S21404B6204A80661A23F90007ED1600106AD213FC46
S21404B6300001001052A26100F374600000C2523987
S21404B64000106AC70C39000300106AC7662C4EB98E
S21404B6500000717A13FC000A00106ABC13FC000F89
S21404B660001061DE4879000865F1487800034EB999
S21404B67000073660508F6000008608F9000400104A
S21404B68061DF7000103900106ABD028000000001FE
S21404B6907201B08166102F39000824F84EB90007ED
S21404B6A037A0588F60582F39000824E84EB9000791
S21404B6B037A0588F604808F90004001061DF700056
S21404B6C0103900106ABD0280000000017201B081CA
S21404B6D066102F39000824F84EB9000737A0588F93
S21404B6E0600E2F39000824E84EB9000737A0588F9B
S21404B6F0423900106AC713FC0007001059044E5E56
S21404B7004E754E56000013FC00090010590400390B
S21404B710000A00106ABD4239001061E023F90007F0
S21404B720ED1A00106AD261044E5E4E754E56000045
S21404B73048E70038287C00106ABD267C000737A03E
S21404B740247C001061E010120C0000056200010465
S21404B7504880D040303B00064EFB0002000C0050F0
S21404B7600074009600B800DA08140000663E0C392F
S21404B77000AA001052A366104879000865F94EB96D
S21404B7800007384C588F600E4879000866234EB977
S21404B7900007384C588F4879000866494EB90007A8
S21404B7A0384C588F14BC0001600000BA081400001E
S21404B7B0670C48790008664B4E93588F600A4879A0
S21404B7C00008664D4E93588F14BC00026000009625
S21404B7D008140000670C4879000866614E93588F79
S21404B7E0600A4879000866634E93588F14BC0003B9
S21404B7F0607208140000670C4879000866724E935D
S21404B800588F600A4879000866744E93588F14BCA3
S21404B8100004605008140000670C48790008668528
S21404B8204E93588F600A4879000866884E93588F5E
S21404B83014BC0005602E08140000670C4879000844
S21404B840669E4E93588F600A4879000866A14E9308
S21404B850588F08F90005001061DF421208940001B1
S21404B8600894000313FC0001001061DE4CDF1C008A
S21404B8704E5E4E754E56000013FC00090010590427
S21404B88013FC000D001061DE423900106AC808F986
S21404B890000100106ABD4239001061E04E5E4E752C
S21404B8A04E56000048E70018287C001061E228BCC9
S21404B8B0001061E8267C001061E04213602A2054E0
S21404B8C00C10003065060C100039630616BC00FF29
S21404B8D0602042401013323C000AC2C0103C00D024
S21404B8E0D010D200168152942014B0B900106AB059
S21404B8F065CC0C13000165120C1300C8620C5313BC
S21404B90013FC0008001061DE60064EB900072472BE
S21404B9104CDF18004E5E4E754E5600000C2E00018D
S21404B920000B66162F390007EBEA48790010582AF0
S21404B9304EB9000071A0508F60142F390007EBEE4B
S21404B94048790010582A4EB9000071A0508F4E5EF8
S21404B9504E754E56000048E70018287C0010582AFA
S21404B960267C000071A0102E000B0C00000762005D
S21404B970008E4880D040303B00064EFB000200722A
S21404B9800010001E002C003A0048005600642F39B0
S21404B9900007EBF22F0C4E93508F606E2F39000782
S21404B9A0EBF62F0C4E93508F60602F390007EBFA9E
S21404B9B02F0C4E93508F60522F390007EBFE2F0C3E
S21404B9C04E93508F60442F390007EC022F0C4E9391
S21404B9D0508F60362F390007EC062F0C4E93508F8D
S21404B9E060282F390007EC0A2F0C4E93508F601AEC
S21404B9F02F390007EC0E2F0C4E93508F600C4879AD
S21404BA00000866CA2F0C4E93508F4CDF18004E5E0B
S21404BA104E754E5600000C2E0001000B66162F398C
S21404BA200007E8FE48790010582A4EB9000071A0B5
S21404BA30508F60142F390007E90248790010582AFD
S21404BA404EB9000071A0508F4E5E4E754E560000E3
S21404BA504AB9001052A4662C487806404EB9000035
S21404BA6072C4588F23C0001052A44A8067164878C0
S21404BA7006402F390007F01E2F004EB9000752F477
S21404BA804FEF000C4E5E4E754E5600004AB900103D
S21404BA9052A8662C487806404EB9000072C4588FE7
S21404BAA023C0001052A84A806716487806402F39EB
S21404BAB00007F0222F004EB9000752F44FEF000C97
S21404BAC04E5E4E754E5600004AB9001052AC662CB7
S21404BAD048780B404EB9000072C4588F23C000103B
S21404BAE052AC4A80671648780B4048790002030037
S21404BAF02F004EB9000752F44FEF000C4E5E4E7501
S21404BB004E56000048E707087C887000102E000B8D
S21404BB10DC80287C0010582A701122064EB90007D3
S21404BB208C960680001053E220400C1000FF6762DB
S21404BB3070114EB900078C960680001053E22F0051
S21404BB402F0C4EB9000071C22F0C4EB9000074CCF5
S21404BB504FEF000C2A002E05600819BC0020780060
S21404BB6052877010BE806DF213FC007C0010583AA9
S21404BB70701122064EB900078C960680001054AE4B
S21404BB802F0048790010583B4EB9000071C2508F00
S21404BB90606C487800112F0C702222064EB90007FC
S21404BBA08C9606800080004E2F004EB90006A1DE5B
S21404BBB02F0C4EB9000074CC4FEF00102A002E054F
S21404BBC0600819BC0020780052877010BE806DF2A1
S21404BBD013FC007C0010583A48780011487900108D
S21404BBE0583B702222064EB900078C9606800080C9
S21404BBF001E62F004EB90006A1DE4FEF000C4CDF25
S21404BC0010E04E5E4E754E5600002F077EF870000C
S21404BC10102E000BDE80701122074EB900078C969A
S21404BC2006800010557A20400C1000FF6720701123
S21404BC304EB900078C9606800010557A2F00487976
S21404BC400010582A4EB9000071C2508F60264878FA
S21404BC50001148790010582A702222074EB90007AE
S21404BC608C9606800080037E2F004EB90006A1DE67
S21404BC704FEF000C2E1F4E5E4E754E5600002F07DB
S21404BC807EF87000102E000BDE80701122074EB96D
S21404BC9000078C9606800010560220400C1000FF09
S21404BCA0672070114EB900078C9606800010560265
S21404BCB02F0048790010582A4EB9000071C2508FE0
S21404BCC060264878001148790010582A7022220706
S21404BCD04EB900078C9606800080048E2F004EB95D
S21404BCE00006A1DE4FEF000C2E1F4E5E4E754E561C
S21404BCF0000048E70308287C0010264D1E2E000B83
S21404BD000C0700A066060814000466540C0700A27C
S21404BD1066060814000566480C0700A466060814A0
S21404BD200006663C0C0700A6660608140007663084
S21404BD300C0700A166060814000066240C0700A37E
S21404BD4066060814000166180C0700A566060814A3
S21404BD500002660C0C0700A7661C0814000367168E
S21404BD604879000866D048790010582A4EB9000071
S21404BD7071C2508F60582C3CFFFFFF6070001007A4
S21404BD80DC80207C0010568A0C3000FF68006706B2
S21404BD901E306800600A207C0010263D1E306800B5
S21404BDA04A0767164879000866DA48790010582A60
S21404BDB04EB9000071C2508F60144879000866DFDF
S21404BDC048790010582A4EB9000071C2508F4CDFD3
S21404BDD010C04E5E4E754E5600002F070C3900FFFD
S21404BDE00010569267081E390010569260061E39D7
S21404BDF0001026454A0767162F390007E8FE4879DB
S21404BE000010582A4EB9000071C2508F60142F39A2
S21404BE100007E90248790010582A4EB9000071C29A
S21404BE20508F2E1F4E5E4E754E56FFFC7000102E21
S21404BE30000B0680FFFFFF882D40FFFC48780011AA
S21404BE4048790010582A7222C1414EB900078C96D0
S21404BE50C14106810080004E20012F004EB9000625
S21404BE60A1DE4FEF000C4E5E4E754E56000048E7BE
S21404BE7003382F39001058E24EB9000074CC588F9E
S21404BE802E006700014E7C887000102E000BDC80AC
S21404BE90307C0001487078004EB9000072C4264019
S21404BEA02F39001058E22F0B4EB9000071C24879A2
S21404BEB0000866E32F0B4EB9000759162840487948
S21404BEC0000866E542A74EB9000759164FEF001C56
S21404BED02440200C673A487800102F0C7011220674
S21404BEE04EB900078C960680001053E22F004EB918
S21404BEF0000758DA4FEF000C701122064EB90007FF
S21404BF008C960680001053E22040422800106020E1
S21404BF104879000866E6701122064EB900078C962A
S21404BF200680001053E22F004EB9000071C2508FF5
S21404BF30200A673A487800102F0A701122064EB974
S21404BF4000078C960680001054AE2F004EB90007EA
S21404BF5058DA4FEF000C701122064EB900078C9683
S21404BF600680001054AE2040422800106020487915
S21404BF70000866E8701122064EB900078C96068003
S21404BF80001054AE2F004EB9000071C2508F7000DE
S21404BF90102E000B2F006100FB6808F90006001045
S21404BFA061DF48790010582A2006E58806800007D5
S21404BFB0EAEE20402F1070001039001061E02F00C8
S21404BFC04EB900073C5E2F0B4EB9000071DE4FEFF2
S21404BFD000144CDF1CC04E5E4E754E56000048E7FB
S21404BFE003002F39001058E24EB9000074CC588F65
S21404BFF04A80670000AE7EF87000102E000BDE80CC
S21404C0002C3CFFFFFF7470001039001061E0DC80E8
S21404C010487800102F39001058E2701122074EB9E4
S21404C02000078C9606800010557A2F004EB900073C
S21404C03058DA701122074EB900078C960680001055
S21404C040557A2040422800107000102E000B2F0056
S21404C0506100FBB408F90006001061DF2006E588DD
S21404C06006800007EB2220402F102F390007EB92A2
S21404C0702F390007EB1E4879001058CC4EB900073C
S21404C080477048790010582A4879001058CC700038
S21404C0901039001061E02F004EB900073C5E4FEFE8
S21404C0A0002C4CDF00C04E5E4E754E56000048E72E
S21404C0B003002F39001058E24EB9000074CC588F94
S21404C0C04A80670000AE7EF87000102E000BDE80FB
S21404C0D02C3CFFFFFF6A70001039001061E0DC8022
S21404C0E0487800102F39001058E2701122074EB914
S21404C0F000078C960680001056022F004EB90007E3
S21404C10058DA701122074EB900078C960680001084
S21404C11056022040422800107000102E000B2F00FC
S21404C1206100FB5808F90006001061DF2006E58868
S21404C13006800007EB2220402F102F390007EB96CD
S21404C1402F390007EB1E4879001058CC4EB900076B
S21404C150477048790010582A4879001058CC700067
S21404C1601039001061E02F004EB900073C5E4FEF17
S21404C170002C4CDF00C04E5E4E754E56000048E75D
S21404C1800318267C001058E21E2E000B2F134EB9FF
S21404C190000074CC588F4A8067000106287C001083
S21404C1A0264D0C0700A066060814000466540C0707
S21404C1B000A266060814000566480C0700A4660676
S21404C1C008140006663C0C0700A66606081400075A
S21404C1D066300C0700A166060814000066240C07E7
S21404C1E000A366060814000166180C0700A5660678
S21404C1F008140002660C0C0700A7661C081400034B
S21404C20067164879000866EA487800F14EB90004D3
S21404C210B4AA508F6000008A20530C1000486706AA
S21404C2200C10004C66682C3CFFFFFF607000100783
S21404C230DC8020530C100048660E207C0010568AC2
S21404C24011BC00016800600A207C0010568A423047
S21404C2506800700010072F006100FA9408F90006C1
S21404C260001061DF48790010582A2006E588068009
S21404C2700007EBA220402F1070001039001061E078
S21404C2802F004EB900073C5E4FEF001060122F39A6
S21404C2900007EC96487800F14EB90004B4AA508F13
S21404C2A04CDF18C04E5E4E754E5600002F390010F7
S21404C2B058E24EB9000074CC588F4A80676E2079D5
S21404C2C0001058E20C10005967060C10004E664A1F
S21404C2D02079001058E20C100059660A13FC00017D
S21404C2E00010569260064239001056926100FAE831
S21404C2F008F90006001061DF48790010582A2F3923
S21404C3000007EBC270001039001061E02F004EB930
S21404C31000073C5E4FEF000C60122F390007EC9AC2
S21404C320487800F24EB90004B4AA508F4E5E4E759B
S21404C3304E56FFE448E703081C2E000B7E001E063C
S21404C34053872007D08006800010569420400C5057
S21404C350FFFF67222007D0800680001056942040F6
S21404C3603D50FFFE2007D080068000105734204042
S21404C3703D50FFFC60700C060029643A48780002C1
S21404C380486EFFFE2007E58806800080059E2F0085
S21404C3904EB90006A1DE48780002486EFFFC20076E
S21404C3A0E5880680008006DE2F004EB90006A1DE72
S21404C3B04FEF00186030700010060680FFFFFFD7AE
S21404C3C0D08006800010230020403D50FFFE700001
S21404C3D010060680FFFFFFD7D080068000102400DA
S21404C3E020403D50FFFC4AB9001052AC672020396B
S21404C3F0001052AC72242D40FFE42007C1414EB910
S21404C40000078C96C141D2AEFFE428416012702426
S21404C41022074EB900078C960680000203002840C7
S21404C4204A14670000C60C1400FF670000BE7E01B5
S21404C4307000302EFFFEE2802F0048790008670562
S21404C440486EFFF24EB9000747704FEF000C082EF7
S21404C4500000FFFF6714487900086709486EFFF27A
S21404C4604EB9000071A0508F601248790008670C1E
S21404C470486EFFF24EB9000071A0508F7000302E47
S21404C480FFFCE2802F0048790008670F486EFFE83B
S21404C4904EB9000747704FEF000C082E0000FFFD52
S21404C4A06714487900086713486EFFE84EB9000021
S21404C4B071A0508F6012487900086716486EFFE82E
S21404C4C04EB9000071A0508F2F0C486EFFE8486EDE
S21404C4D0FFF248790008671948790010582A4EB9BF
S21404C4E0000747704FEF00146002420710074CDF46
S21404C4F010C04E5E4E754E5600002F070C2E0029B7
S21404C500000B64207E001E2E000B2F0748790008BF
S21404C51067274879001058EC4EB9000747704FEF6C
S21404C520000C60227ED87000102E000BDE802F07D1
S21404C5304879000867354879001058EC4EB900076A
S21404C54047704FEF000C2E1F4E5E4E754E56FFE89A
S21404C55048E707382F39001058E24EB9000074CC6B
S21404C560588F2E00670001907C001C2E000B53860B
S21404C570307C0001487078004EB9000072C4244034
S21404C5802F39001058E22F0A4EB9000071C24879BC
S21404C590000867442F0A4EB9000759162640487902
S21404C5A00008674642A74EB9000759164FEF001C0D
S21404C5B02840200B6704200C66162F390007EC8EE3
S21404C5C0487800E54EB90004B4AA508F6000011EF6
S21404C5D02F0B43EEFFF84EB900074EBA2F0C43EE6E
S21404C5E0FFF04EB900074EBA508F48790007ED1E8B
S21404C5F0486EFFF84EB9000780384A406D3C4879CB
S21404C6000007ED26486EFFF84EB9000780384A400A
S21404C6106E2848790007ED1E486EFFF04EB90007F5
S21404C62080384A406D1448790007ED26486EFFF0BE
S21404C6304EB9000780384A406F162F390007EC8E33
S21404C640487800E54EB90004B4AA508F6000009EF6
S21404C65048790007ED2E486EFFF8486EFFE84EB99D
S21404C66000078170486EFFE84EB900077C8E3A00DA
S21404C67048790007ED2E486EFFF0486EFFE84EB985
S21404C68000078170486EFFE84EB900077C8E3E00B6
S21404C6902006D08006800010569420403085200660
S21404C6A0D080068000105734204030877000102E4B
S21404C6B0000B2F006100FC7A7000102E000B2F0078
S21404C6C06100FE3408F90006001061DF48790010A6
S21404C6D0582A4879001058EC70001039001061E0B0
S21404C6E02F004EB900073C5E4FEF00142F0A4EB9D8
S21404C6F0000071DE588F4CDF1CE04E5E4E754E56C1
S21404C70000000C3900FF001057D4670812390010D7
S21404C71057D4600612390010265210014E5E4E752C
S21404C7204E5600000C3900FF001057D56708123922
S21404C730001057D5600612390010263810014E5ED8
S21404C7404E754E56000048E7011861B21E00287C5C
S21404C7500010582A4879000867472F0C4EB9000085
S21404C76071C2508F267C000071A010070C00000ACE
S21404C770672E0C00000B67360C00000C67140C00C8
S21404C780000D67460C00000E67320C000011674867
S21404C79060544879000867532F0C4E93508F6052AC
S21404C7A048790008676D2F0C4E93508F6044487983
S21404C7B0000867872F0C4E93508F60364879000820
S21404C7C067A12F0C4E93508F60284879000867BBEA
S21404C7D02F0C4E93508F601A4879000867D52F0C9B
S21404C7E04E93508F600C4879000867EF2F0C4E93D9
S21404C7F0508F0C3900FF001057D567081E390010FB
S21404C80057D560061E390010263810070C000001A4
S21404C81067360C00000267220C000003670E0C004B
S21404C820000D67320C000011673A6046487900082C
S21404C83068092F0C4E93508F604448790008681797
S21404C8402F0C4E93508F60364879000868252F0CBD
S21404C8504E93508F60284879000868352F0C4E9305
S21404C860508F601A4879000868402F0C4E93508FFA
S21404C870600C48790008684F2F0C4E93508F4CDF9D
S21404C88018804E5E4E754E56000048E70338420642
S21404C8902F39001058E24EB9000074CC588F4A80E5
S21404C8A06700043C287C001052A4267C001052AC7E
S21404C8B0247C001057D42079001058E210100C0085
S21404C8C0004167140C000039670001C80C000036EC
S21404C8D06700034C600003CA6100F1AE6100F1E634
S21404C8E0287C001052A84A39001048516700008A74
S21404C8F04A94671E13FC0002001057D54878013886
S21404C900487900079EAA2F144EB9000752F44FEF39
S21404C910000C4A93671A487805A0487900079FE2F6
S21404C9202053486805A04EB9000752F44FEF000C98
S21404C9307E00603A2007D08006800007A582224049
S21404C9407028D087D08006800010569420403091FE
S21404C9502007D08006800007A5D222407028D08702
S21404C960D0800680001057342040309152877028BB
S21404C970BE806DC06000033E4A390010484667001A
S21404C980008A4A94671E13FC0001001057D54878A5
S21404C99001384879000796722F144EB9000752F4EE
S21404C9A04FEF000C4A93671A487805A048790007A9
S21404C9B097AA2053486805A04EB9000752F44FEFD3
S21404C9C0000C7E00603A2007D080068000079D4A4F
S21404C9D022407028D087D0800680001056942040CD
S21404C9E030912007D080068000079D9A2240702848
S21404C9F0D087D0800680001057342040309152876C
S21404CA007028BE806DC0600002AC4A94671E13FC9A
S21404CA100003001057D548780108487900078E6A45
S21404CA202F144EB9000752F44FEF000C4A93671ABE
S21404CA30487805A0487900078F722053486805A0F7
S21404CA404EB9000752F44FEF000C7E00603A200700
S21404CA50D08006800007951222407028D087D080A8
S21404CA60068000105694204030912007D08006801F
S21404CA700007956222407028D087D0800680001078
S21404CA8057342040309152877028BE806DC06000B5
S21404CA9002246100EFB86100F02C4A3900104851B6
S21404CAA0677C4A94671A14BC000B48780640487999
S21404CAB00007AED22F144EB9000752F44FEF000C05
S21404CAC04A936716487805A048790007C6922F133C
S21404CAD04EB9000752F44FEF000C7E006036200774
S21404CAE0D08006800007CD7222402007D0800680C2
S21404CAF000105694204030912007D080068000070E
S21404CB00CDC222402007D080068000105734204033
S21404CB10309152877028BE806DC4600001984A39EF
S21404CB2000104846677C4A94671A14BC000A487882
S21404CB30064048790007B5122F144EB9000752F480
S21404CB404FEF000C4A936716487805A0487900070B
S21404CB50C0F22F134EB9000752F44FEF000C7E00BC
S21404CB6060362007D08006800007CCD222402007FB
S21404CB70D080068000105694204030912007D08044
S21404CB8006800007CD2222402007D08006800010B1
S21404CB9057342040309152877028BE806DC46000A0
S21404CBA001144A94671A14BC000C48780640487965
S21404CBB00007A8922F144EB9000752F44FEF000C4A
S21404CBC04A936716487805A048790007BB522F1386
S21404CBD04EB9000752F44FEF000C7E006036200773
S21404CBE0D08006800007CC3222402007D080068002
S21404CBF000105694204030912007D080068000070D
S21404CC00CC8222402007D080068000105734204073
S21404CC10309152877028BE806DC460000098610011
S21404CC20EE2C6100EEA04A94671A14BC000E4878F5
S21404CC30064048790007D0522F144EB9000752F424
S21404CC404FEF000C4A936716487805A0487900070A
S21404CC50D6922F134EB9000752F44FEF000C7E0005
S21404CC6060362007D08006800007DC32224020078A
S21404CC70D080068000105694204030912007D08043
S21404CC8006800007DC8222402007D0800680001041
S21404CC9057342040309152877028BE806DC460148B
S21404CCA02F390007EC92487800E84EB90004B4AA7D
S21404CCB0508F7C014A0666266100FA8808F9000649
S21404CCC0001061DF48790010582A2F390007EBD28C
S21404CCD0487800594EB900073C5E4FEF000C4CDF15
S21404CCE01CC04E5E4E754E5600002F074EB9000708
S21404CCF036324A006604700160244AB9001052A411
S21404CD00670E2F39001052A46158588F1E00600C0D
S21404CD102F390007F01E614A588F1E0010072E1F79
S21404CD204E5E4E754E5600002F074EB9000736323B
S21404CD304A0066047E0160224AB9001052A8670EB3
S21404CD402F39001052A8611A588F1E00600C2F3914
S21404CD500007F022610C588F1E0010072E1F4E5E2F
S21404CD604E754E56FFE248E70138267C001061E017
S21404CD70286E00084A13660E48790008685E4EB9A5
S21404CD800007343E588F0C1300C865064200600046
S21404CD9000E470001013E788D9C052134A5466069C
S21404CDA04207600000CE0C54000165060C540007D0
S21404CDB063064207600000BC7E02247C0010582AEA
S21404CDC0700010132F0048790008688F2F0A4EB998
S21404CDD0000747707000102C00012F006100EB74F0
S21404CDE04879000868962F0A4EB9000071A07000B2
S21404CDF0302C00022F006100008448790008689CEB
S21404CE002F0A4EB9000071A04FEF00240C54000600
S21404CE10662E7000302C00042040486800014879D3
S21404CE20000868A2486EFFE24EB900074770486ED5
S21404CE30FFE22F0A4EB9000071A04FEF0014600CF9
S21404CE407000302C00042F006132588F4879000897
S21404CE5068AC2F0A4EB9000071A07000302C000692
S21404CE602F00610001842F0A4EB90007343E4FEFAD
S21404CE70001010074CDF1C804E5E4E754E56FFE2C7
S21404CE8048E701183E2E000A4A3900104851670840
S21404CE90287C0007E05460164A39001048466708A4
S21404CEA0287C0007DF946006287C0007DED447EE63
S21404CEB0FFE20C4700C86520700030072040486831
S21404CEC0FF394879000868B22F0B4EB9000747703F
S21404CED04FEF000C600000FA4A4765260C47002F07
S21404CEE0622070003007E5882F340800487900086F
S21404CEF068BB2F0B4EB9000747704FEF000C60005D
S21404CF0000D00C47004065320C47005F622C70006E
S21404CF1030070680FFFFFFC0E58806800007E1149F
S21404CF2020402F104879000868C02F0B4EB9000720
S21404CF3047704FEF000C600000980C470080655067
S21404CF400C47009F624A4A39001048516708287CFB
S21404CF500007E29460164A39001048466708287CA1
S21404CF600007E2146006287C0007E194700030078E
S21404CF700680FFFFFF80E5882F3408004879000804
S21404CF8068C52F0B4EB9000747704FEF000C604082
S21404CF900C4700C666124879000868CA2F0B4EB9BB
S21404CFA000074770508F60280C4700C76612487900
S21404CFB0000868D32F0B4EB900074770508F6010D7
S21404CFC04879000868DC2F0B4EB900074770508F6D
S21404CFD02F0B48790010582A4EB9000071A0508FC4
S21404CFE04CDF18804E5E4E754E56FFE248E7010849
S21404CFF03E2E000A4A39001048516708287C00076C
S21404D000E29460164A39001048466708287C0007F0
S21404D010E2146006287C0007E1940C4700FF6606CD
S21404D020422EFFE260744A4765260C47001F6220C2
S21404D03070003007E5882F3408004879000868E453
S21404D040486EFFE24EB9000747704FEF000C604A87
S21404D0500C47003065320C470049622C70003007DC
S21404D0600680FFFFFFD0E58806800007E314204013
S21404D0702F104879000868E9486EFFE24EB90007A9
S21404D08047704FEF000C60124879000868EE486E4F
S21404D090FFE24EB900074770508F486EFFE24879AA
S21404D0A00010582A4EB9000071A0508F4CDF108033
S21404D0B04E5E4E754E560000227C00104854102ECC
S21404D0C0000B060000AB0C00002E620001DE488058
S21404D0D0D040303B00064EFB0002009600A000BE87
S21404D0E000C800D201D000DC00E600F001D001D078
S21404D0F001D001D001D001D001D0005E007A01D069
S21404D10001D001D001D001D001D001D001D000AAB5
S21404D11000B400FA0104010E0122011801D001D066
S21404D120012C01360140014A0154015C0164017678
S21404D1300188019A01AC01BE123900102017823909
S21404D1400010201F82390010202782390010202F5B
S21404D1506000015C12390010201682390010201E6F
S21404D16082390010202682390010202E60000140EB
S21404D17012390010209760000136123900102094EE
S21404D1806000012C123900102017600001221239A9
S21404D190001020166000011812390010209160005B
S21404D1A0010E12390010209260000104123900109A
S21404D1B02093600000FA12390010471C600000F04B
S21404D1C0123900102095600000E6123900102096EF
S21404D1D0600000DC123900102002600000D2123910
S21404D1E000102014600000C81239001020156000DA
S21404D1F000BE123900102098600000B412390010E6
S21404D2002018600000AA123900102100600000A057
S21404D2101239001021016000009612390010210214
S21404D2206000008C1239001021036000008212395D
S21404D23000102104607812390010210560704A112C
S21404D24067081239001021066064123C00FF605E15
S21404D2504A1167081239001021076052123C00FF79
S21404D260604C4A1167081239001021086040123CCD
S21404D27000FF603A4A116708123900102109602E2F
S21404D280123C00FF60284A11670812390010210A70
S21404D290601C123C00FF60164A1167081239001021
S21404D2A0210B600A123C00FF6004123C00FF1001D0
S21404D2B04E5E4E754E56000048E723003E2E000A8A
S21404D2C04206227C0010582A0C472710652470005A
S21404D2D03007223C000027104EB9000779200600CC
S21404D2E000301280700030074EB9000779B03E0057
S21404D2F052060C4703E864044A0667387000300791
S21404D300223C000003E84EB90007792006000030EE
S21404D3105206123C00FFD206740014012202138047
S21404D320180070003007223C000003E84EB90007DE
S21404D33079B03E000C47006464044A066730700007
S21404D340300772644EB90007792006000030520692
S21404D350123C00FFD2067400140122021380180047
S21404D3607000300772644EB9000779B03E000C476F
S21404D370000A64044A06673070003007720A4EB921
S21404D38000077920060000305206123C00FFD20641
S21404D3907400140122021380180070003007720A09
S21404D3A04EB9000779B03E0030070600003052063A
S21404D3B0123C00FFD20674001401220213801800E7
S21404D3C070001006423108004CDF00C44E5E4E75F5
S21404D3D04E560000610C61000372610004B44E5E98
S21404D3E04E754E56000013FC00FF001052B013FC9E
S21404D3F000FF001052B113FC00FF001052B213FCE1
S21404D40000FF001052B323FCFFFFFC18001052B4B8
S21404D41023FCFFFFFC18001052B823FCFFFFFC1887
S21404D420001052BC23FCFFFFFC18001052C023FC63
S21404D430FFFFFC18001052C423FCFFFFFC1800106A
S21404D44052C823FCFFFFFC18001052CC23FCFFFF3D
S21404D450FC18001052D023FCC08F4000001052D499
S21404D46023FC00000000001052D823FCC08F4000AC
S21404D470001052DC23FC00000000001052E023FCE5
S21404D480C08F4000001052E423FC0000000000108F
S21404D49052E823FCC08F4000001052EC23FC00002E
S21404D4A00000001052F023FCFFFFFC18001052F49A
S21404D4B023FCFFFFFC18001052F823FCFFFFFC18A7
S21404D4C0001052FC23FCFFFFFC180010530023FC42
S21404D4D0FFFFFC180010530423FCFFFFFC18001089
S21404D4E0530823FCFFFFFC180010530C23FCFFFF1B
S21404D4F0FC180010531023FCFFFFFC1800105314F4
S21404D50023FCFFFFFC180010531823FCFFFFFC1835
S21404D5100010531C23FCFFFFFC180010532023FCB0
S21404D520FFFFFC180010532423FCFFFFFC18001018
S21404D530532823FCFFFFFC180010532C23FCFFFF8A
S21404D540FC180010533023FCFFFFFC180010533463
S21404D55023FCFFFFFC180010533823FCFFFFFC18C5
S21404D5600010533C23FCFFFFFC180010534023FC20
S21404D570FFFFFC180010534423FCFFFFFC180010A8
S21404D580534823FCFFFFFC180010534C23FCFFFFFA
S21404D590FC180010535023FCFFFFFC1800105354D3
S21404D5A023FCFFFFFC180010535823FCFFFFFC1855
S21404D5B00010535C23FCFFFFFC180010536023FC90
S21404D5C0FFFFFC180010536423FCFFFFFC18001038
S21404D5D0536823FCFFFFFC180010536C23FCFFFF6A
S21404D5E0FC180010537070FF23C00010539223C021
S21404D5F00010539623C00010539A23C00010539E65
S21404D60023FCC08F40000010538A23FC0000000057
S21404D6100010538E23C0001053A223C0001053A63C
S21404D62013FC00FF001053AA23FCC08F4000001018
S21404D63053AC23FC00000000001053B013FC00FFA2
S21404D640001053B413FC00FF001053B513FC00FF86
S21404D650001053B613FC00FF001053B713FC00FF72
S21404D660001053B833FCFFFF001053BA33FCFFFF1F
S21404D670001053BC13FC00FF0010537613FC00FF8D
S21404D6800010537713FC00FF0010537813FC00FFC0
S21404D6900010537913FC00FF0010537A33FCFFFF8D
S21404D6A00010537C13FC00550010537E13FC00FF3F
S21404D6B00010537413FC00FF0010537533FCFFFF77
S21404D6C00010538033FCFFFF0010538213FC00FF4E
S21404D6D00010538442390010538523FCC08F400049
S21404D6E0001053BE23FC00000000001053C223FCAD
S21404D6F0C08F4000001053C623FC0000000000103A
S21404D70053CA23FCFFFFFC18001053CE23FCFFFF74
S21404D710FC18001053D233FCFFFF001053D633FC22
S21404D720FFFF001053D833FCFFFF001053DA33FC1E
S21404D730FFFF001053DC33FCFFFF001053DE33FC06
S21404D740FFFF001053E04E5E4E754E5600002F0746
S21404D75013FC00FF001057D413FC00FF001057D52D
S21404D7604AB9001052A467142F39001052A44EB9B7
S21404D770000071DE588F42B9001052A44AB9001056
S21404D78052A867342F39001052A84EB9000071DE33
S21404D790588F42B9001052A87E30601670001007E9
S21404D7A00680FFFFFFD006800010210020404210B4
S21404D7B052070C07004963E44AB9001052AC6714D8
S21404D7C02F39001052AC4EB9000071DE588F42B9A2
S21404D7D0001052AC4207602A424010073200C2FCD6
S21404D7E000110681001053E2204110BC00FF3200F5
S21404D7F0C2FC00110681001054AE204110BC00FF8C
S21404D80052070C07000C65D04207603A42401007E6
S21404D8103200C2FC001106810010557A204110BC6B
S21404D82000FF3200C2FC001106810010560220419F
S21404D83010BC00FF7000100706800010568A2040B7
S21404D84010BC00FF52070C07000865C013FC00FF5D
S21404D850001056924207602670001007D08006809B
S21404D86000105694204030BCFFFF70001007D08094
S21404D870068000105734204030BCFFFF52070C07C8
S21404D880005065D44239001058EB2E1F4E5E4E757C
S21404D8904E5600002F0C4239001025F24A3900106B
S21404D8A0484666000142287C001046E4207C0010AE
S21404D8B046DC4A3900104AAD664E227C00104D956F
S21404D8C00C11000167060C110005660A001000031F
S21404D8D0021400FC60360C1100026608421008D4DC
S21404D8E0000160280C110003660842100894000129
S21404D8F0601A0C110006660A10BC000618BC0080EC
S21404D900600A42104214600442104214287C00103C
S21404D91046DD207C001046E54A3900104AAE6614FF
S21404D9200C39000100104D96660A0014000302101C
S21404D93000FC60204A3900104AAE66140C39000612
S21404D94000104D96660A18BC000610BC00806004E1
S21404D95042144210287C001046DE207C001046E666
S21404D9604A3900104AAF66140C39000100104D976E
S21404D970660A00140003021000FC60204A390010F6
S21404D9804AAF66140C39000600104D97660A18BC98
S21404D990000610BC0080600442144210287C00106C
S21404D9A046DF207C001046E74A3900104AB0661469
S21404D9B00C39000100104D98660A0014000302108A
S21404D9C000FC606C4A3900104AB066140C39000634
S21404D9D000104D98660A18BC000610BC0080605003
S21404D9E042144210604A4A3900104AB1662A13F9B2
S21404D9F0001046E2001046E013F9001046E300105B
S21404DA0046E113F9001046EA001046E813F9001040
S21404DA1046EB001046E960184239001046E04239E9
S21404DA20001046E14239001046E84239001046E943
S21404DA3008B900020010000933F90010000800407D
S21404DA400000285F4E5E4E754E56FFF848E70318F2
S21404DA504A390010486267081E3C00FF7C016004D7
S21404DA6042074206267C0006A09E0C3900FF0010E2
S21404DA705374672413F90010537400104E5D4878ED
S21404DA800001487900104E5D487900800DE24E93FF
S21404DA904FEF000C0007000F0C3900FF001052B0C7
S21404DAA0672413F9001052B000104D954878000111
S21404DAB0487900104D9548790080082A4E934FEF18
S21404DAC0000C0007001F0C3900FF001052B1672439
S21404DAD013F9001052B100104D96487800014879A9
S21404DAE000104D9648790080082C4E934FEF000C9A
S21404DAF00007000F0C3900FF001052B2672413F918
S21404DB00001052B200104D97487800014879001072
S21404DB104D9748790080082E4E934FEF000C00076F
S21404DB20000F0C3900FF001052B3672413F90010DD
S21404DB3052B300104D9848780001487900104D986B
S21404DB404879008008304E934FEF000C0007000F12
S21404DB500CB9FFFFFC18001052B4674023F90010FC
S21404DB6052B400104D9A23F9001052C400104DAA66
S21404DB7048780004487900104D9A487900800832A5
S21404DB804E9348780004487900104DAA48790080DE
S21404DB9008524E934FEF0018000700130CB9FFFF0E
S21404DBA0FC18001052B8674023F9001052B8001051
S21404DBB04D9E23F9001052C800104DAE487800045C
S21404DBC0487900104D9E48790080083A4E9348786C
S21404DBD00004487900104DAE48790080085A4E93E8
S21404DBE04FEF0018000700030CB9FFFFFC180010E5
S21404DBF052BC674023F9001052BC00104DA223F912
S21404DC00001052CC00104DB2487800044879001039
S21404DC104DA24879008008424E934878000448791B
S21404DC2000104DB24879008008624E934FEF0018FA
S21404DC300007000C0CB9FFFFFC18001052C0674028
S21404DC4023F9001052C000104DA623F9001052D03C
S21404DC5000104DB648780004487900104DA648795F
S21404DC600080084A4E9348780004487900104DB660
S21404DC7048790080086A4E934FEF00180007000C9E
S21404DC8048790007ED4E4879001052D44EB9000783
S21404DC9080384A40672E23F9001052D400104DBA3B
S21404DCA023F9001052D800104DBE48780008487971
S21404DCB000104DBA4879008008724E934FEF000C5E
S21404DCC00007000348790007ED4E4879001052DC3F
S21404DCD04EB9000780384A40672E23F9001052DCFC
S21404DCE000104DC223F9001052E000104DC64878CB
S21404DCF00008487900104DC24879008008824E9387
S21404DD004FEF000C0007000348790007ED4E4879F2
S21404DD10001052E44EB9000780384A40672E23F9B3
S21404DD20001052E400104DCA23F9001052E8001007
S21404DD304DCE48780008487900104DCA48790080CE
S21404DD4008924E934FEF000C0007000C487900072A
S21404DD50ED4E4879001052EC4EB9000780384A4020
S21404DD60672E23F9001052EC00104DD223F9001050
S21404DD7052F000104DD648780008487900104DD26D
S21404DD804879008008A24E934FEF000C0007000C61
S21404DD900CB9FFFFFC18001052F4672423F9001096
S21404DDA052F400104DDA48780004487900104DDA31
S21404DDB04879008008B24E934FEF000C000700032A
S21404DDC00CB9FFFFFC18001052F8672423F9001062
S21404DDD052F800104DDE48780004487900104DDEF5
S21404DDE04879008008BA4E934FEF000C00070003F2
S21404DDF00CB9FFFFFC18001052FC672423F900102E
S21404DE0052FC00104DE248780004487900104DE2B8
S21404DE104879008008C24E934FEF000C0007000CB0
S21404DE200CB9FFFFFC1800105300672423F90010F8
S21404DE30530000104DE648780004487900104DE67B
S21404DE404879008008CA4E934FEF000C0007000C78
S21404DE500CB9FFFFFC1800105304674023F90010A8
S21404DE60530400104DEA23F90010531400104DFA21
S21404DE7048780004487900104DEA4879008008D2B2
S21404DE804E9348780004487900104DFA487900808B
S21404DE9008F24E934FEF0018000700110CB9FFFF6D
S21404DEA0FC1800105308674023F9001053080010AC
S21404DEB04DEE23F90010531800104DFE4878000468
S21404DEC0487900104DEE4879008008DA4E93487879
S21404DED00004487900104DFE4879008008FA4E93F5
S21404DEE04FEF0018000700220CB9FFFFFC180010C3
S21404DEF0530C674023F90010530C00104DF223F91D
S21404DF000010531C00104E02487800044879001094
S21404DF104DF24879008008E24E9348780004487928
S21404DF2000104E024879008009024E934FEF001805
S21404DF30000700440CB9FFFFFC180010531067409C
S21404DF4023F90010531000104DF623F90010532047
S21404DF5000104E0648780004487900104DF64879BB
S21404DF60008008EA4E9348780004487900104E066C
S21404DF7048790080090A4E934FEF0018000700887E
S21404DF800CB9FFFFFC1800105324672423F9001073
S21404DF90532400104E0A48780004487900104E0AAC
S21404DFA04879008009124E934FEF000C00070011C9
S21404DFB00CB9FFFFFC1800105328672423F900103F
S21404DFC0532800104E0E48780004487900104E0E70
S21404DFD048790080091A4E934FEF000C0007002280
S21404DFE00CB9FFFFFC180010532C672423F900100B
S21404DFF0532C00104E1248780004487900104E1234
S21404E0004879008009224E934FEF000C0007004425
S21404E0100CB9FFFFFC1800105330672423F90010D6
S21404E020533000104E1648780004487900104E16F7
S21404E03048790080092A4E934FEF000C00070088A9
S21404E0400CB9FFFFFC1800105334672423F90010A2
S21404E050533400104E1A48780004487900104E1ABB
S21404E0604879008009324E934FEF000C0007000FEA
S21404E0700CB9FFFFFC1800105338672423F900106E
S21404E080533800104E1E48780004487900104E1E7F
S21404E09048790080093A4E934FEF000C0007000FB2
S21404E0A00CB9FFFFFC180010533C672423F900103A
S21404E0B0533C00104E2248780004487900104E2243
S21404E0C04879008009424E934FEF000C0007000F7A
S21404E0D00CB9FFFFFC1800105340672423F9001006
S21404E0E0534000104E2648780004487900104E2607
S21404E0F048790080094A4E934FEF000C0007000F42
S21404E1000CB9FFFFFC1800105344672423F90010D1
S21404E110534400104E2A48780004487900104E2ACA
S21404E1204879008009524E934FEF000C08C7000050
S21404E1300CB9FFFFFC1800105348672423F900109D
S21404E140534800104E2E48780004487900104E2E8E
S21404E15048790080095A4E934FEF000C08C7000117
S21404E1600CB9FFFFFC180010534C672423F9001069
S21404E170534C00104E3248780004487900104E3252
S21404E1804879008009624E934FEF000C08C70002DE
S21404E1900CB9FFFFFC1800105350672423F9001035
S21404E1A0535000104E3648780004487900104E3616
S21404E1B048790080096A4E934FEF000C08C70003A5
S21404E1C00CB9FFFFFC1800105354672423F9001001
S21404E1D0535400104E3A48780004487900104E3ADA
S21404E1E04879008009724E934FEF000C08C7000070
S21404E1F00CB9FFFFFC1800105358672423F90010CD
S21404E200535800104E3E48780004487900104E3E9D
S21404E21048790080097A4E934FEF000C08C7000136
S21404E2200CB9FFFFFC180010535C672423F9001098
S21404E230535C00104E4248780004487900104E4261
S21404E2404879008009824E934FEF000C08C70002FD
S21404E2500CB9FFFFFC1800105360672423F9001064
S21404E260536000104E4648780004487900104E4625
S21404E27048790080098A4E934FEF000C08C70003C4
S21404E2800CB9FFFFFC1800105364672423F9001030
S21404E290536400104E4A48780004487900104E4AE9
S21404E2A04879008009924E934FEF000C08C700008F
S21404E2B00CB9FFFFFC1800105368672423F90010FC
S21404E2C0536800104E4E48780004487900104E4EAD
S21404E2D048790080099A4E934FEF000C08C7000156
S21404E2E00CB9FFFFFC180010536C672423F90010C8
S21404E2F0536C00104E5248780004487900104E5271
S21404E3004879008009A24E934FEF000C08C700021C
S21404E3100CB9FFFFFC1800105370672423F9001093
S21404E320537000104E5648780004487900104E5634
S21404E3304879008009AA4E934FEF000C08C70003E3
S21404E34048790007ED4E4879001053BE4EB90007D1
S21404E35080384A40672E23F9001053BE00102590DB
S21404E36023F9001053C20010259448780008487911
S21404E37000102590487900800EA04E934FEF000CB5
S21404E3800007000F48790007ED4E4879001053C681
S21404E3904EB9000780384A40672E23F9001053C64A
S21404E3A00010259823F9001053CA0010259C4878BD
S21404E3B00008487900102598487900800EB04E93DE
S21404E3C04FEF000C0007000F0CB9FFFFFC180010FD
S21404E3D053CE672423F9001053CE001025A04878A6
S21404E3E000044879001025A0487900800EC04E939A
S21404E3F04FEF000C0007000F0CB9FFFFFC180010CD
S21404E40053D2672423F9001053D2001025A4487869
S21404E41000044879001025A4487900800EC84E935D
S21404E4204FEF000C0007000F0C79FFFF001053D6C7
S21404E430672433F9001053D600104E8A4878000239
S21404E440487900104E8A487900800D304E934FEF7D
S21404E450000C000700030C79FFFF001053D8672454
S21404E46033F9001053D800104E8C487800024879CF
S21404E47000104E8C487900800D344E934FEF000CFC
S21404E480000700030C79FFFF001053DA672433F902
S21404E490001053DA00104E8E4878000248790010B7
S21404E4A04E8E487900800D384E934FEF000C0007CF
S21404E4B000030C79FFFF001053DC672433F90010C7
S21404E4C053DC00104E9048780002487900104E90B5
S21404E4D0487900800D3C4E934FEF000C0007000C6B
S21404E4E00C79FFFF001053DE672433F9001053DE67
S21404E4F000104E9248780002487900104E924879EF
S21404E50000800D404E934FEF000C0007000C0C7972
S21404E510FFFF001053E0672433F9001053E00010A7
S21404E5204E9448780002487900104E94487900804A
S21404E5300D444E934FEF000C0007000C0CB9FFFF80
S21404E540FFFF00105392672223F900105392001025
S21404E5504E5E48780004487900104E5E4879008084
S21404E5600E3A4E934FEF000C7C010CB9FFFFFFFFF1
S21404E57000105396672223F90010539600104E623B
S21404E58048780004487900104E62487900800E42AC
S21404E5904E934FEF000C7C010CB9FFFFFFFF0010F9
S21404E5A0539A672223F90010539A00104E6648784F
S21404E5B00004487900104E66487900800E4A4E934F
S21404E5C04FEF000C7C010CB9FFFFFFFF0010539EB9
S21404E5D0672223F90010539E00104E6A4878000400
S21404E5E0487900104E6A487900800E524E934FEFD9
S21404E5F0000C7C0148790007ED4E48790010538AD8
S21404E6004EB9000780384A40672A23F90010538A17
S21404E610001047FE23F90010538E00104802487875
S21404E62000084879001047FE487900800E904E9303
S21404E6304FEF000C0CB9FFFFFFFF001053A2672238
S21404E64023F9001053A200104E6E4878000448794F
S21404E65000104E6E487900800E5A4E934FEF000C11
S21404E6607C010CB9FFFFFFFF001053A6672223F9B5
S21404E670001053A600104E72487800044879001023
S21404E6804E72487900800E884E934FEF000C7C0142
S21404E6900C3900FF001053AA672213F9001053AA7E
S21404E6A000104E7648780001487900104E76487976
S21404E6B000800E624E934FEF000C7C0148790007F1
S21404E6C0ED4E4879001053AC4EB9000780384A40E6
S21404E6D0672C23F9001053AC00104E7823F9001071
S21404E6E053B000104E7C48780008487900104E78E5
S21404E6F0487900800E784E934FEF000C7C010C395D
S21404E70000FF001053B4672213F9001053B400102E
S21404E7104E8048780001487900104E804879008081
S21404E7200E664E934FEF000C7C010C3900FF001070
S21404E73053B5672213F9001053B500104E8148787C
S21404E7400001487900104E81487900800E684E9387
S21404E7504FEF000C7C010C3900FF001053B6672203
S21404E76013F9001053B600104E8248780001487919
S21404E77000104E82487900800E6A4E934FEF000CCC
S21404E7807C010C3900FF001053B7672213F9001000
S21404E79053B700104E8348780001487900104E8322
S21404E7A0487900800E6C4E934FEF000C7C010C39B8
S21404E7B000FF001053B8672213F9001053B8001076
S21404E7C04E8448780001487900104E8448790080C9
S21404E7D00E6E4E934FEF000C7C010C79FFFF001079
S21404E7E053BA672233F9001053BA00104E8648789D
S21404E7F00002487900104E86487900800E704E93C9
S21404E8004FEF000C7C010C79FFFF001053BC67220D
S21404E81033F9001053BC00104E884878000248793B
S21404E82000104E88487900800E744E934FEF000C0B
S21404E8307C014A3900104846670A4A0667064EB9FC
S21404E84000057C1E4A390010484567124A07670EC1
S21404E850700010072F004EB900057178588F0C39D8
S21404E86000FF00105375672013F90010537500104D
S21404E870471A4878000148790010471A48790080FA
S21404E8800DF64E934FEF000C287C0010537C0C3989
S21404E89000FF0010537666100C3900FF0010537901
S21404E8A066060C54FFFF6770486EFFF94EB9000702
S21404E8B003A4588F0C3900FF0010537667181D798F
S21404E8C000105376FFFA1D7900105377FFFB1D796D
S21404E8D000105378FFFC0C3900FF001053796710C2
S21404E8E01D7900105379FFFD1D790010537AFFFE41
S21404E8F00C54FFFF671633D4001047EC7000301436
S21404E90072644EB9000779B01D40FFFF486EFFF9E8
S21404E9104EB90007043C588F0C3900550010537E3E
S21404E920672013F90010537E001047EE4878000164
S21404E9304879001047EE487900800E384E934FEF22
S21404E940000C0C79FFFF00105380672033F9001089
S21404E95053800010472C4878000248790010472C52
S21404E960487900800DE44E934FEF000C0C79FFFFBE
S21404E97000105382672033F9001053820010472E8C
S21404E9804878000248790010472E487900800DE840
S21404E9904E934FEF000C0C3900FF00105384672091
S21404E9A013F900105384001048544878000148793D
S21404E9B000104854487900800DF84E934FEF000C31
S21404E9C04A3900105385677413F9001053860010F3
S21404E9D047CA13F900105387001047CB13F90010E9
S21404E9E05388001047CC13F900105389001047CD04
S21404E9F0487800014879001047CA487900800FF823
S21404EA004E93487800014879001047CB4879008037
S21404EA100FFA4E93487800014879001047CC48799D
S21404EA2000800FFC4E93487800014879001047CDCB
S21404EA30487900800FFE4E934FEF00304CDF18C02D
S21404EA404E5E4E754E56FFFE48E703384206426E4B
S21404EA50FFFE0C3900FF001057D4670A13F90010A4
S21404EA6057D4001026520C3900FF001057D5670AF9
S21404EA7013F9001057D5001026384AB9001052A4CE
S21404EA80660A4AB9001052A8670005FA4EB900048F
S21404EA90BA4C4EB90004BA884EB90004BAC44EB98A
S21404EAA000007050487800014879000200004EB912
S21404EAB0000067204EB900007050267C00006848AD
S21404EAC0487803202F39001052A448790002180011
S21404EAD04E93487803202F39001052A84879000234
S21404EAE010004E93487805A02F39001052AC487990
S21404EAF0000203004E934FEF002C4EB900007050F6
S21404EB00287C00078E3A247C000200604EB900067A
S21404EB10EEA60C4000016600024E10390010265284
S21404EB200C00000A67760C00000B670000BC0C00A3
S21404EB30000C671C0C00000D670001460C00000E5C
S21404EB40670000F20C00001167000182600001C833
S21404EB504878001848790007CE122F0A4E93487852
S21404EB60001848790007CE424879000200904E9378
S21404EB704878001848790007CE7248790002018068
S21404EB804E934878001848790007CEA248790002C8
S21404EB9001B04E934FEF0030600001B4487800187F
S21404EBA048790007CED22F0A4E9348780018487941
S21404EBB00007CF024879000200904E934878001868
S21404EBC048790007CF324879000201804E9348788E
S21404EBD0001848790007CF624879000201B04E93C6
S21404EBE04FEF003060000168487800184879000745
S21404EBF0CF922F0A4E934878001848790007CFC260
S21404EC004879000200904E93487800184879000727
S21404EC10CFF24879000201804E934878001848796C
S21404EC200007D0224879000201B04E934FEF00301F
S21404EC306000011C4878001848790007DCD22F0AC7
S21404EC404E934878001848790007DD024879000298
S21404EC5000904E934878001848790007DD324879CA
S21404EC60000201804E934878001848790007DD6258
S21404EC704879000201B04E934FEF0030600000D098
S21404EC8048780018487900078CBA2F0A4E934878BB
S21404EC900018487900078CEA4879000200904E93E1
S21404ECA048780018487900078D1A487900020180D0
S21404ECB04E9348780018487900078D4A4879000230
S21404ECC001B04E934FEF003060000084487800187F
S21404ECD0487900078D7A2F0A4E93487800184879A9
S21404ECE000078DAA4879000200904E9348780018D1
S21404ECF0487900078DDA4879000201804E934878F7
S21404ED000018487900078E0A4879000201B04E932D
S21404ED104FEF00306038487800182F0C2F0A4E93B7
S21404ED20487800182F0C4879000200904E934878D3
S21404ED3000182F0C4879000201804E93487800187A
S21404ED402F0C4879000201B04E934FEF003023FC9D
S21404ED50000240000010264E4EB90006B9184EB9FF
S21404ED600006B968603E487800182F0C2F0A4E93A8
S21404ED70487800182F0C4879000200904E93487883
S21404ED8000182F0C4879000201804E93487800182A
S21404ED902F0C4879000201B04E934FEF003042B971
S21404EDA00010264E4EB900007050287C0010264DE8
S21404EDB0247C0007A8624EB90006C9EA4A406700E8
S21404EDC002801039001026380C000001670000C2CB
S21404EDD00C000002676A0C00000367140C00000DA8
S21404EDE0670000FE0C0000116700014660000190F9
S21404EDF0487800184879000795B248790002000060
S21404EE004E93487800184879000795E2487900023E
S21404EE1000304E93487800184879000796124879CF
S21404EE20000201204E93487800184879000796425D
S21404EE304879000201504E934FEF00306000017C89
S21404EE404878001848790007A6224879000200008E
S21404EE504E934878001848790007A652487900026D
S21404EE6000304E934878001848790007A6824879FF
S21404EE70000201204E934878001848790007A6B28D
S21404EE804879000201504E934FEF00306000012C89
S21404EE9048780018487900079DEA4879000200007F
S21404EEA04E9348780018487900079E1A487900025D
S21404EEB000304E9348780018487900079E4A4879EF
S21404EEC0000201204E9348780018487900079E7A7D
S21404EED04879000201504E934FEF0030600000DC8A
S21404EEE04878001848790007A6E24879000200002E
S21404EEF04E934878001848790007A712487900020C
S21404EF0000304E934878001848790007A74248799D
S21404EF10000201204E934878001848790007A7722B
S21404EF204879000201504E934FEF00306000008C89
S21404EF304878001848790007A7A24879000200001C
S21404EF404E934878001848790007A7D248790002FB
S21404EF5000304E934878001848790007A80248798C
S21404EF60000201204E934878001848790007A8321A
S21404EF704879000201504E934FEF0030603C4878C9
S21404EF8000182F0A4879000200004E9348780018AB
S21404EF902F0A4879000200304E93487800182F0A4A
S21404EFA04879000201204E93487800182F0A4879C1
S21404EFB0000201504E934FEF003023FC0002200065
S21404EFC00010003E48780001486EFFFE2F390010FE
S21404EFD000364E934FEF000C421426790007F022B9
S21404EFE06058302B00060640FFBE0C4000076248FF
S21404EFF0D040303B00064EFB000200100016001CFA
S21404F00000220028002E0034003A08D400006028AD
S21404F01008D40001602208D40002601C08D400034F
S21404F020601608D40004601008D40005600A08D4EA
S21404F0300006600408D40007508B4A5366A4604454
S21404F040487800182F0A4879000200004E93487842
S21404F05000182F0A4879000200304E9348780018AA
S21404F0602F0A4879000201204E93487800182F0A88
S21404F0704879000201504E934FEF003042B9001019
S21404F080003E42144207287C0006A09E267C001000
S21404F09053E26066424010073200C2FC00112001B1
S21404F0A00C3300FF080067504878001148730800C6
S21404F0B0424010073200C2FC002206810080004E47
S21404F0C020012F004E944878001142401007320069
S21404F0D0C2FC00110681001054AE20012F004240ED
S21404F0E010073200C2FC00220681008001E62001DF
S21404F0F02F004E944FEF001852070C07000C65942F
S21404F1004207267C0010568A247C001056026000B3
S21404F11000BC424010073200C2FC001106810010F9
S21404F120557A20410C1000FF67324878001142409F
S21404F13010073200C2FC001106810010557A200127
S21404F1402F00424010073200C2FC002206810080D5
S21404F150037E20012F004E944FEF000C4240100710
S21404F1603200C2FC001120010C3200FF08006722A6
S21404F1704878001148720800424010073200C2FC6A
S21404F180002206810080048E20012F004E944FEF4B
S21404F190000C700010070C3300FF0800672C720088
S21404F1A0120706810010263D204110B30800487857
S21404F1B000014873080070001007D08006800080A5
S21404F1C00DD02F004E944FEF000C52070C0700088A
S21404F1D06500FF400C3900FF00105692672013F9B3
S21404F1E00010569200102645487800014879001011
S21404F1F02645487900800DF44E944FEF000C4207E4
S21404F200247C00105694600000A270001007D08082
S21404F2100C72FFFF08006700009048780002700038
S21404F2201007D0804872080070001007E588068032
S21404F2300080059E2F004E94487800027000100748
S21404F240D0800680001057342F0070001007E58821
S21404F2500680008006DE2F004E944FEF00180C0741
S21404F2600028654270001007D080720012070681DD
S21404F270FFFFFFD8D281068100102300204130B260
S21404F280080070001007D080068000105734224013
S21404F290700010070680FFFFFFD8D080068000109D
S21404F2A02400204030917C0152070C070050650072
S21404F2B0FF5A4A06677A4AB90010264E6772267CB9
S21404F2C00010000808AB0001000108AB00030001B1
S21404F2D033D3004000004207604670001007D08019
S21404F2E00C72FFFF0800673670001007D080068097
S21404F2F000B01E60284070001007D08038B20800A6
S21404F30070001007D080068000B01EC02840700031
S21404F3101007D080068000105734204038905207DB
S21404F3200C07002865B40053000A33D300400000DD
S21404F3304CDF1CC04E5E4E754E56000023F900107E
S21404F3400042001058E64E5E4E754E5600002039B8
S21404F3500010004290B9001058E60C8000000258D5
S21404F360652223F900100042001058E642390010C6
S21404F3704D73423900104D744EB90006CFDC4EB9B9
S21404F380000734B04E5E4E754E5600002F0C287C97
S21404F390001049B81039001049B50C000010671861
S21404F3A00C00003067120C00002067480C00004078
S21404F3B0670000A0600000A04878002A4879001082
S21404F3C025667000301453807254C1414EB900074C
S21404F3D08C96C14106810060000020012F004EB9C2
S21404F3E00006A1DE4FEF000C33FC0001001049B606
S21404F3F06174606C4878002A4879001025663014D9
S21404F400C0FC00540680006000002F004EB90006C1
S21404F410A1DE4FEF000C61001F9A53540C54FFFFFB
S21404F420661A0C790064001049B2640C42A74EB9FF
S21404F430000731A0588F600438BC00633014B079DC
S21404F440001049BA661A42A74EB9000731A0588F71
S21404F450600E6112600A42A74EB9000731A0588FA9
S21404F460285F4E5E4E754E56000048E70018287C0E
S21404F470001049B61039001049B50C000010671288
S21404F4800C000030674A0C000040670000CC6000A7
S21404F49001D60C540030660E42A74EB9000731A0C0
S21404F4A0588F600001CC082C00000001670861003A
S21404F4B001C8600001BC4EB9000736324A00670630
S21404F4C05254600001AC4EB900071992600001A2C4
S21404F4D00C54002E6650267C001049B853534254F0
S21404F4E048790008690B4EB9000737A0588F4A536D
S21404F4F0661A0C790064001049B2640C42A74EB92F
S21404F500000731A0588F600436BC00643013B0790D
S21404F510001049BA6600015A42A74EB9000731A046
S21404F520588F6000014C082C00000001670E4EB98D
S21404F5300007346861000142600001364EB90007D6
S21404F54036320C00000166065254600001244EB99F
S21404F550000719926000011A30144A4067100C40E4
S21404F560000167260C400002673C600000EE08F9C4
S21404F5700004001061DF48790008690D4EB90007E1
S21404F58037A0588F5254600000E84EB90007363250
S21404F5900C00000166065254600000D64EB90007FF
S21404F5A01992600000CC4EB90007357E4A00660A00
S21404F5B04EB900071992600000B84EB900073476B9
S21404F5C023C0001058E24A8066142F390007E9F673
S21404F5D0487800E34EB900073660508F60702040CC
S21404F5E00C100059665423FC0060000000102562CD
S21404F5F0487800044879001025624879006020D0D5
S21404F6004EB90006A24C4279001049B2487800026E
S21404F6104879001049B248790060237E4EB9000646
S21404F620A24C4EB9000738724879000869244EB9CE
S21404F630000737A04FEF001C60144EB9000738725D
S21404F64048790008693B4EB9000737A0588F42A78F
S21404F6504EB9000731A0588F601642A74EB900076E
S21404F66031A0588F600A42A74EB9000731A0588FC0
S21404F6704CDF18004E5E4E754E56000048E70038C4
S21404F680287C001061DF267C000737A0247C00104D
S21404F690582A3039001049B65340E2580C40001737
S21404F6A062001CF8D040303B00064EFB00020030DF
S21404F6B000A80118029C0414058C0704086609C8EF
S21404F6C00B2A0C8C0DEC0F40109E11FC12D013A6C6
S21404F6D014861612179E192A1A981B6C1C3E700064
S21404F6E03039001049B82F004879000869542F0AA9
S21404F6F04EB90007477008D400042F0A4EB9000715
S21404F700343E08D400044879000869604E9308D44F
S21404F71000044878001470003039001025662F0065
S21404F72061001D6808D400042F0A4E934FEF002092
S21404F7300C39000100102568660E487900086984B3
S21404F7404E93588F60001C5E48790008698B4E9370
S21404F750588F60001C5008D4000448790008699447
S21404F7604EB90007343E20390010256AE2882F007F
S21404F770700010390010256F2F007000103900102B
S21404F78025702F0070001039001025712F007000AE
S21404F7901039001025742F007000103900102572DF
S21404F7A02F0070001039001025732F0048790008C8
S21404F7B069C22F0A4EB9000747702F0A4E934FEFBF
S21404F7C0002C60001BE04879000869E74EB9000782
S21404F7D0343E487800144878000861001CAE08D40B
S21404F7E000042F0A4EB90007343E4FEF001008D429
S21404F7F000040839000000102575670C2F3900072F
S21404F800EC9E4E93588F600A2F390007ECA24E9355
S21404F810588F08D400042F390007ED364E934878E5
S21404F820001448790000800861001C6008D40004B5
S21404F8302F0A4E934FEF001008D400040839000036
S21404F8400010257667220839000000102588670C0A
S21404F8502F390007ED3E4E93588F602C2F39000742
S21404F860EC9E4E93588F60200839000000102589BE
S21404F870670C2F390007ED424E93588F600A2F39D4
S21404F8800007ECA24E93588F08D400042F390007C3
S21404F890ED364E93588F4A390010484667564878D6
S21404F8A000144878001061001BE208D400042F0AF4
S21404F8B04E934FEF000C083900000010257C660EAE
S21404F8C02F390007ECA64E93588F60001AD80839D3
S21404F8D0000000102581670E2F390007EC9E4E931A
S21404F8E0588F60001AC02F390007ECA24E93588F29
S21404F8F060001AB2487800144878001061001B8C27
S21404F90008D400042F0A4E934FEF000C0839000267
S21404F91000102577660E2F390007ECA64E93588FF5
S21404F92060001A82083900000010257D670E2F3902
S21404F9300007EC9E4E93588F60001A6A2F39000712
S21404F940ECA24E93588F60001A5C487800144878EE
S21404F950000961001B3608D400042F0A4EB90007BC
S21404F960343E4FEF000C08D40004083900010010A0
S21404F9702575670C2F390007EC9E4E93588F600A46
S21404F9802F390007ECA24E93588F08D400042F3961
S21404F9900007ED364E934878001448790000800935
S21404F9A061001AE808D400042F0A4E934FEF0010A3
S21404F9B008D40004083900010010257667220839A7
S21404F9C0000100102588670C2F390007ED3E4E9382
S21404F9D0588F602C2F390007EC9E4E93588F60206A
S21404F9E00839000100102589670C2F390007ED42FD
S21404F9F04E93588F600A2F390007ECA24E93588F07
S21404FA0008D400042F390007ED364E93588F4A3930
S21404FA10001048466756487800144878001161007C
S21404FA201A6A08D400042F0A4E934FEF000C0839C4
S21404FA3000010010257C660E2F390007ECA64E93B5
S21404FA40588F600019600839000100102581670E80
S21404FA502F390007EC9E4E93588F600019482F39B3
S21404FA600007ECA24E93588F6000193A48780014A9
S21404FA704878001861001A1408D400042F0A4E931C
S21404FA804FEF000C0839000200102578660E2F3957
S21404FA900007ECA64E93588F6000190A0839000038
S21404FAA00010257E670E2F390007EC9E4E93588F64
S21404FAB0600018F22F390007ECA24E93588F6000AE
S21404FAC018E4487800144878000A610019BE08D47F
S21404FAD000042F0A4EB90007343E4FEF000C08D43A
S21404FAE000040839000200102575670C2F3900073A
S21404FAF0EC9E4E93588F600A2F390007ECA24E9363
S21404FB00588F08D400042F390007ED364E934878F2
S21404FB10001448790000800A6100197008D40004B3
S21404FB202F0A4E934FEF001008D400040839000241
S21404FB300010257667220839000200102588670C15
S21404FB402F390007ED3E4E93588F602C2F3900074F
S21404FB50EC9E4E93588F60200839000200102589C9
S21404FB60670C2F390007ED424E93588F600A2F39E1
S21404FB700007ECA24E93588F08D400042F390007D0
S21404FB80ED364E93588F4A390010484667564878E3
S21404FB90001448780012610018F208D400042F0AF2
S21404FBA04E934FEF000C083900020010257C660EB9
S21404FBB02F390007ECA64E93588F600017E80839D3
S21404FBC0000200102581670E2F390007EC9E4E9325
S21404FBD0588F600017D02F390007ECA24E93588F29
S21404FBE0600017C248780014487800206100189C0A
S21404FBF008D400042F0A4E934FEF000C0839000275
S21404FC0000102579660E2F390007ECA64E93588F00
S21404FC1060001792083900000010257F670E2F3900
S21404FC200007EC9E4E93588F6000177A2F39000712
S21404FC30ECA24E93588F6000176C487800144878EE
S21404FC40000B6100184608D400042F0A4EB90007BA
S21404FC50343E4FEF000C08D40004083900030010AB
S21404FC602575670C2F390007EC9E4E93588F600A53
S21404FC702F390007ECA24E93588F08D400042F396E
S21404FC800007ED364E934878001448790000800B40
S21404FC90610017F808D400042F0A4E934FEF0010A3
S21404FCA008D40004083900030010257667220839B2
S21404FCB0000300102588670C2F390007ED3E4E938D
S21404FCC0588F602C2F390007EC9E4E93588F602077
S21404FCD00839000300102589670C2F390007ED4208
S21404FCE04E93588F600A2F390007ECA24E93588F14
S21404FCF008D400042F390007ED364E93588F4A393E
S21404FD000010484667564878001448780013610087
S21404FD10177A08D400042F0A4E934FEF000C0839C4
S21404FD2000030010257C660E2F390007ECA64E93C0
S21404FD30588F600016700839000300102581670E7E
S21404FD402F390007EC9E4E93588F600016582F39B3
S21404FD500007ECA24E93588F6000164A48780014A9
S21404FD60487800286100172408D400042F0A4E930C
S21404FD704FEF000C083900020010257A660E2F3962
S21404FD800007ECA64E93588F6000161A0839000038
S21404FD9000102580670E2F390007EC9E4E93588F6F
S21404FDA0600016022F390007ECA24E93588F6000AD
S21404FDB015F4487800144878000C610016CE08D470
S21404FDC000042F0A4EB90007343E4FEF000C08D447
S21404FDD000040839000400102575670C2F39000745
S21404FDE0EC9E4E93588F600A2F390007ECA24E9370
S21404FDF0588F08D400042F390007ED364E93487800
S21404FE00001448790000800C6100168008D40004B1
S21404FE102F0A4E934FEF001008D40004083900044C
S21404FE200010257667220839000400102588670C20
S21404FE302F390007ED3E4E93588F602C2F3900075C
S21404FE40EC9E4E93588F60200839000400102589D4
S21404FE50670C2F390007ED424E93588F600A2F39EE
S21404FE600007ECA24E93588F08D400042F390007DD
S21404FE70ED364E93588F4A39001048466740487806
S21404FE8000144879000080106100160008D40004AD
S21404FE902F0A4E934FEF000C083900000010257B04
S21404FEA0670E2F390007EC9E4E93588F600014F6A9
S21404FEB02F390007ECA24E93588F600014E8487858
S21404FEC0001448780011610015C208D400042F0AF3
S21404FED04E934FEF000C0839000200102577660E8B
S21404FEE02F390007ECA64E93588F600014B80839D3
S21404FEF000010010257D670E2F390007EC9E4E93F7
S21404FF00588F600014A02F390007ECA24E93588F28
S21404FF1060001492487800144878000D6100156C4F
S21404FF2008D400042F0A4EB90007343E4FEF000CE5
S21404FF3008D400040839000500102575670C2F390D
S21404FF400007EC9E4E93588F600A2F390007ECA2E8
S21404FF504E93588F08D400042F390007ED364E937D
S21404FF604878001448790000800D6100151E08D4F6
S21404FF7000042F0A4E934FEF001008D400040839EB
S21404FF80000500102576672208390005001025882C
S21404FF90670C2F390007ED3E4E93588F602C2F398F
S21404FFA00007EC9E4E93588F602008390005001019
S21404FFB02589670C2F390007ED424E93588F600A47
S21404FFC02F390007ECA24E93588F08D400042F391B
S21404FFD00007ED364E93588F4A390010484667405E
S21404FFE0487800144879000080116100149E08D4F3
S21404FFF000042F0A4E934FEF000C0839000100103E
S214050000257B670E2F390007EC9E4E93588F6000B0
S21405001013942F390007ECA24E93588F6000138671
S21405002048780014487800196100146008D4000464
S2140500302F0A4E934FEF000C083900020010257862
S214050040660E2F390007ECA64E93588F60001356A0
S214050050083900010010257E670E2F390007EC9E33
S2140500604E93588F6000133E2F390007ECA24E932F
S214050070588F60001330487800144878000E6100E9
S214050080140A08D400042F0A4EB90007343E4FEF71
S214050090000C08D400040839000600102575670C06
S2140500A02F390007EC9E4E93588F600A2F390007AC
S2140500B0ECA24E93588F08D400042F390007ED366E
S2140500C04E934878001448790000800E610013BCF2
S2140500D008D400042F0A4E934FEF001008D40004EE
S2140500E00839000600102576672208390006001034
S2140500F02588670C2F390007ED3E4E93588F602CE8
S2140501002F390007EC9E4E93588F6020083900065D
S21405011000102589670C2F390007ED424E93588F3E
S214050120600A2F390007ECA24E93588F08D40004B6
S2140501302F390007ED364E93588F4A39001048463A
S2140501406740487800144879000080126100133C27
S21405015008D400042F0A4E934FEF000C083900020E
S2140501600010257B670E2F390007EC9E4E93588F9F
S214050170600012322F390007ECA24E93588F6000AC
S21405018012244878001448780021610012FE08D42D
S21405019000042F0A4E934FEF000C0839000200109A
S2140501A02579660E2F390007ECA64E93588F60000A
S2140501B011F4083900010010257F670E2F39000756
S2140501C0EC9E4E93588F600011DC2F390007ECA289
S2140501D04E93588F600011CE487800144878000F6B
S2140501E0610012A808D400042F0A4EB90007343E51
S2140501F04FEF000C08D400040839000700102575D9
S214050200670C2F390007EC9E4E93588F600A2F39DE
S2140502100007ECA24E93588F08D400042F39000728
S214050220ED364E934878001448790000800F61003B
S214050230125A08D400042F0A4E934FEF001008D424
S21405024000040839000700102576672208390007DC
S21405025000102588670C2F390007ED3E4E93588F02
S214050260602C2F390007EC9E4E93588F6020083976
S214050270000700102589670C2F390007ED424E93BD
S214050280588F600A2F390007ECA24E93588F08D472
S21405029000042F390007ED364E93588F4A39001063
S2140502A04846674048780014487900008013610086
S2140502B011DA08D400042F0A4E934FEF000C0839C4
S2140502C000030010257B670E2F390007EC9E4E9322
S2140502D0588F600010D02F390007ECA24E93588F28
S2140502E0600010C248780014487800296100119C07
S2140502F008D400042F0A4E934FEF000C083900026D
S2140503000010257A660E2F390007ECA64E93588FF7
S214050310600010920839000100102580670E2F39FD
S2140503200007EC9E4E93588F6000107A2F39000711
S214050330ECA24E93588F6000106C4879000869E966
S2140503404EB90007343E48780014487900008030DE
S2140503506100113808D400042F0A4EB90007343E50
S2140503604FEF001008D40004083900000010258A55
S214050370670C2F390007EC9E4E93588F600A2F396D
S2140503800007ECA24E93588F08D400042F390007B7
S214050390ED364E93487800144879000080366100A3
S2140503A010EA08D400042F0A4E934FEF001008D425
S2140503B00004083900000010258B670C2F3900074C
S2140503C0EC9E4E93588F600A2F390007ECA24E9389
S2140503D0588F08D400042F390007ED364E93588FF2
S2140503E04A3900104846674248780014487800178E
S2140503F06100109808D400042F0A4EB90007343E51
S2140504004FEF000C0839000700102581670E2F39BD
S2140504100007EC9E4E93588F60000F8A2F39000711
S214050420ECA24E93588F60000F7C487800144879EC
S214050430000080106100105408D400042F0A4E9363
S2140504404FEF000C0839000100102577660E2F398E
S2140504500007ECA64E93588F60000F4A0839000037
S2140504600010257767260839000300102577670EE4
S2140504702F390007ED464E93588F60000F282F3909
S2140504800007EC9E4E93588F60000F1A2F39000711
S214050490ECA24E93588F60000F0C487800144879EC
S2140504A00000803161000FE408D400042F0A4EB91D
S2140504B00007343E4FEF000C08D40004083900014D
S2140504C00010258A670C2F390007EC9E4E93588F2F
S2140504D0600A2F390007ECA24E93588F08D4000403
S2140504E02F390007ED364E934878001448790000FA
S2140504F0803761000F9608D400042F0A4E934FEFFD
S214050500001008D40004083900010010258B670C7C
S2140505102F390007EC9E4E93588F600A2F39000737
S214050520ECA24E93588F08D400042F390007ED36F9
S2140505304E93588F4A39001048466742487800144B
S2140505404878001661000F4408D400042F0A4EB9F7
S2140505500007343E4FEF000C0839000600102581D1
S214050560670E2F390007EC9E4E93588F60000E36A7
S2140505702F390007ECA24E93588F60000E28487856
S214050580001448790000801461000F0008D40004A8
S2140505902F0A4E934FEF000C0839000100102578FE
S2140505A0660E2F390007ECA64E93588F60000DF6A1
S2140505B00839000000102578672608390003001062
S2140505C02578670E2F390007ED464E93588F600045
S2140505D00DD42F390007EC9E4E93588F60000DC63C
S2140505E02F390007ECA24E93588F60000DB8487857
S2140505F0001448790000803261000E9008D400048B
S2140506002F0A4EB90007343E4FEF000C08D40004FD
S214050610083900020010258A670C2F390007EC9E62
S2140506204E93588F600A2F390007ECA24E93588FC9
S21405063008D400042F390007ED364E934878001489
S21405064048790000803861000E4208D400042F0A5D
S2140506504E934FEF001008D400040839000200102E
S214050660258B670C2F390007EC9E4E93588F600A32
S2140506702F390007ECA24E93588F4A39001048468A
S214050680674E08D400042F390007ED364E93487898
S21405069000144878000261000DF208D400042F0A01
S2140506A04EB90007343E4FEF001008390001001020
S2140506B02584670E2F390007EC9E4E93588F6000F1
S2140506C00CE42F390007ECA24E93588F60000CD629
S2140506D008D400042F390007ED364E9348780014E9
S2140506E048790000801861000DA208D400042F0A7E
S2140506F04E934FEF00100839000100102579660E5D
S2140507002F390007ECA64E93588F60000C980839D1
S21405071000000010257967260839000300102579A2
S214050720670E2F390007ED464E93588F60000C76FE
S2140507302F390007EC9E4E93588F60000C682F39B2
S2140507400007ECA24E93588F60000C5A48780014A8
S21405075048790000803361000D3208D400042F0A62
S2140507604EB90007343E4FEF000C08D40004083994
S21405077000030010258A670C2F390007EC9E4E9360
S214050780588F600A2F390007ECA24E93588F08D46D
S21405079000042F390007ED364E9348780014487943
S2140507A00000803961000CE408D400042F0A4E933B
S2140507B04FEF001008D40004083900030010258BFD
S2140507C0670C2F390007EC9E4E93588F600A2F3919
S2140507D00007ECA24E93588F4A3900104846674EDC
S2140507E008D400042F390007ED364E9348780014D8
S2140507F04878005861000C9408D400042F0A4EB9B6
S2140508000007343E4FEF001008390002001025841B
S214050810670E2F390007EC9E4E93588F60000B86A7
S2140508202F390007ECA24E93588F60000B7808D43A
S21405083000042F390007ED364E93487800144879A2
S2140508400000801C61000C4408D400042F0A4E9357
S2140508504FEF0010083900010010257A660E2F3973
S2140508600007ECA64E93588F60000B3A0839000037
S2140508700010257A6726083900030010257A670ECA
S2140508802F390007ED464E93588F60000B182F3909
S2140508900007EC9E4E93588F60000B0A2F39000711
S2140508A0ECA24E93588F60000AFC487800144879ED
S2140508B00000803461000BD408D400042F0A4EB91A
S2140508C00007343E4FEF000C08D400040839000436
S2140508D00010258A670C2F390007EC9E4E93588F1B
S2140508E0600A2F390007ECA24E93588F08D40004EF
S2140508F02F390007ED364E934878001448790000E6
S214050900803A61000B8608D400042F0A4E934FEFF9
S214050910001008D40004083900040010258B670C65
S2140509202F390007EC9E4E93588F600A2F39000723
S214050930ECA24E93588F08D400042F390007ED36E5
S2140509404E934878001442A761000B4008D4000473
S2140509502F0A4E934FEF0010083900050010258525
S214050960670E2F390007EC9E4E93588F60000A36A7
S2140509702F390007ECA24E93588F60000A28487856
S214050980001448790000803561000B0008D4000487
S2140509902F0A4EB90007343E4FEF000C08D400046A
S2140509A0083900050010258A670C2F390007EC9ECC
S2140509B04E93588F600A2F390007ECA24E93588F36
S2140509C008D400042F390007ED364E9348780014F6
S2140509D048790000803B61000AB208D400042F0A5B
S2140509E04E934FEF001008D4000408390005001098
S2140509F0258B670C2F390007EC9E4E93588F600A9F
S214050A002F390007ECA24E93588F08D400042F39CF
S214050A100007ED364E934878001448780055610077
S214050A200A6A08D400042F0A4E934FEF00100839BF
S214050A30000600102585670E2F390007EC9E4E939D
S214050A40588F600009602F390007ECA24E93588F27
S214050A50600009524879000869EB4EB90007343E34
S214050A604878001448790000803C61000A1E08D4C6
S214050A7000042F0A4EB90007343E4FEF001008D485
S214050A8000040839000000102587670C2F39000779
S214050A90EC9E4E93588F600A2F390007ECA24E93B2
S214050AA0588F08D400042F390007ED364E93487842
S214050AB0001448780056610009D208D400042F0AAD
S214050AC04E934FEF001008D40004083900070010B5
S214050AD02585670C2F390007EC9E4E93588F600AC4
S214050AE02F390007ECA24E93588F08D400042F39EF
S214050AF00007ED364E934878001448780054610098
S214050B00098A08D400042F0A4E934FEF00100839BF
S214050B10000000102585670E2F390007EC9E4E93C2
S214050B20588F600008802F390007ECA24E93588F27
S214050B30600008724A3900104846670000B24878D7
S214050B4000144878001C6100094208D400042F0AE6
S214050B504E934FEF000C08D400040839000400102B
S214050B60257C66182F390007ECA64E9308D400049A
S214050B702F390007ED3A4E93508F602E0839000442
S214050B8000102582670C2F390007EC9E4E93588F70
S214050B90600A2F390007ECA24E93588F08D400043C
S214050BA02F390007ED364E93588F4878001448794C
S214050BB000008014610008D408D400042F0A4E9360
S214050BC04FEF000C08D40004083900040010257BFC
S214050BD0670E2F390007EC9E4E93588F60000098DD
S214050BE02F390007ECA24E93588F6000008A48788C
S214050BF00014487800166100089208D400042F0AED
S214050C004EB90007343E4FEF000C08D400040839EF
S214050C1000060010257D670C2F390007EC9E4E93C5
S214050C20588F600A2F390007ECA24E93588F08D4C8
S214050C3000042F390007ED364E934878001448789F
S214050C4000176100084608D400042F0A4E934FEF9C
S214050C50001008D40004083900070010257D670C2D
S214050C602F390007EC9E4E93588F600A2F390007E0
S214050C70ECA24E93588F08D400042F390007ED36A2
S214050C804E934878001448780051610007FE08D452
S214050C9000042F0A4E934FEF00100839000100108C
S214050CA02585670E2F390007EC9E4E93588F6000FA
S214050CB006F42F390007ECA24E93588F600006E61F
S214050CC04A3900104846670000B24878001448784C
S214050CD0001D610007B608D400042F0A4E934FEF97
S214050CE0000C08D40004083900050010257C661899
S214050CF02F390007ECA64E9308D400042F390007B9
S214050D00ED3A4E93508F602E083900050010258267
S214050D10670C2F390007EC9E4E93588F600A2F39C3
S214050D200007ECA24E93588F08D400042F3900070D
S214050D30ED364E93588F4878001448790000801594
S214050D406100074808D400042F0A4E934FEF000CA5
S214050D5008D40004083900050010257B670E2F39D6
S214050D600007EC9E4E93588F600000982F390007B9
S214050D70ECA24E93588F6000008A48780014487895
S214050D80001E6100070608D400042F0A4EB90007A6
S214050D90343E4FEF000C08D4000408390006001056
S214050DA0257E670C2F390007EC9E4E93588F600AF8
S214050DB02F390007ECA24E93588F08D400042F391C
S214050DC00007ED364E93487800144878001F6100FA
S214050DD006BA08D400042F0A4E934FEF001008D425
S214050DE00004083900070010257E670C2F39000718
S214050DF0EC9E4E93588F600A2F390007ECA24E934F
S214050E00588F08D400042F390007ED364E934878DE
S214050E100014487800526100067208D400042F0AB0
S214050E204E934FEF00100839000200102585670E17
S214050E302F390007EC9E4E93588F600005682F39B2
S214050E400007ECA24E93588F6000055A4A390010E9
S214050E504846670000B2487800144878001E6100CE
S214050E60062A08D400042F0A4E934FEF000C08D428
S214050E700004083900060010257C66182F3900077F
S214050E80ECA64E9308D400042F390007ED3A4E938E
S214050E90508F602E0839000600102582670C2F3902
S214050EA00007EC9E4E93588F600A2F390007ECA278
S214050EB04E93588F08D400042F390007ED364E930D
S214050EC0588F48780014487900008016610005BCE4
S214050ED008D400042F0A4E934FEF000C08D40004E4
S214050EE0083900060010257B670E2F390007EC9E93
S214050EF04E93588F600000982F390007ECA24E934A
S214050F00588F6000008A48780014487800266100EB
S214050F10057A08D400042F0A4EB90007343E4FEF71
S214050F20000C08D40004083900060010257F670C5D
S214050F302F390007EC9E4E93588F600A2F3900070D
S214050F40ECA24E93588F08D400042F390007ED36CF
S214050F504E9348780014487800276100052E08D47B
S214050F6000042F0A4E934FEF001008D400040839EA
S214050F7000070010257F670C2F390007EC9E4E935F
S214050F80588F600A2F390007ECA24E93588F08D465
S214050F9000042F390007ED364E934878001448783C
S214050FA00053610004E608D400042F0A4E934FEF61
S214050FB000100839000300102585670E2F39000735
S214050FC0EC9E4E93588F600003DC2F390007ECA289
S214050FD04E93588F600003CE4A3900104846670086
S214050FE0009448780014487800156100049E08D4DB
S214050FF000042F0A4EB90007343E4FEF000C08D404
S21405100000040839000500102581670C2F390007F4
S214051010EC9E4E93588F600A2F390007ECA24E932C
S214051020588F08D400042F390007ED364E934878BC
S2140510300014487800146100045208D400042F0AEE
S2140510404EB90007343E4FEF001008D400040839A7
S214051050000400102581670E2F390007EC9E4E937D
S214051060588F600000982F390007ECA24E93588FD2
S2140510706000008A487800144878002E6100040C49
S21405108008D400042F0A4EB90007343E4FEF000C73
S21405109008D400040839000600102580670C2F398F
S2140510A00007EC9E4E93588F600A2F390007ECA276
S2140510B04E93588F08D400042F390007ED364E930B
S2140510C0487800144878002F610003C008D400044F
S2140510D02F0A4E934FEF001008D400040839000776
S2140510E000102580670C2F390007EC9E4E93588F0D
S2140510F0600A2F390007ECA24E93588F08D40004D7
S2140511002F390007ED364E9348780014487800507E
S2140511106100037808D400042F0A4E934FEF0010A1
S2140511200839000400102585670E2F390007EC9E48
S2140511304E93588F6000026E2F390007ECA24E932F
S214051140588F6000026048780014487800576100A0
S214051150033A08D400042F0A4EB90007343E4FEF71
S214051160000C08D400040839000000102584670C1C
S2140511702F390007EC9E4E93588F600A2F390007CB
S214051180ECA24E93588F08D400042F390007ED368D
S2140511904E934878001448790000803D610002ECC3
S2140511A008D400042F0A4E934FEF001008D400040D
S2140511B00839000100102587670C2F390007EC9EBB
S2140511C04E93588F600A2F390007ECA24E93588F1E
S2140511D008D400042F390007ED364E9348780014DE
S2140511E048780001610002A408D400042F0A4E9333
S2140511F04FEF00100839000300102584670E2F39BD
S2140512000007EC9E4E93588F6000019A2F39000711
S214051210ECA24E93588F6000018C487800144878ED
S214051220005D6100026608D400042F0A4EB9000767
S214051230343E4FEF000C08D40004083900040010B3
S2140512402584670C2F390007EC9E4E93588F600A4D
S2140512502F390007ECA24E93588F08D400042F3977
S2140512600007ED364E93487800144878005E610016
S214051270021A08D400042F0A4E934FEF001008D424
S21405128000040839000500102584670C2F3900076F
S214051290EC9E4E93588F600A2F390007ECA24E93AA
S2140512A0588F08D400042F390007ED364E9348783A
S2140512B000144878005F610001D208D400042F0AA4
S2140512C04E934FEF00100839000600102584670E70
S2140512D02F390007EC9E4E93588F600000C82F39B3
S2140512E00007ECA24E93588F600000BA4A390010EA
S2140512F0484667464A3900104851673E08D40004F8
S21405130048780014487800186100018008D4000465
S2140513102F0A4E934FEF000C083900000010258267
S214051320670C2F390007EC9E4E93588F60762F3941
S2140513300007ECA24E93588F606A4A39001048455C
S214051340674C4A390010472A674408D400047000E1
S2140513501039001025802F00700010390010257FE9
S2140513602F00700010390010257E2F0070001039F0
S2140513700010257D2F004879000869ED2F0A4EB923
S214051380000747702F0A4E934FEF001C60162F3943
S2140513900007ED4A4E93588F600A42A74EB90007DC
S2140513A031A0588F5279001049B64CDF1C004E5EAE
S2140513B04E754E56FFFE20390010256AE2882F002E
S2140513C0700010390010256F2F00700010390010BE
S2140513D025702F0070001039001025712F00700041
S2140513E01039001025742F00700010390010257272
S2140513F02F0070001039001025732F00700030394B
S214051400001049B8204048680001487900086A1F5E
S21405141048790010582A4EB90007477008F90004A5
S214051420001061DF48790010582A4EB90007343E8F
S2140514303D7900102566FFFE487800147000302EB2
S214051440FFFE2F00614408F90004001061DF4879AB
S2140514500010582A4EB9000737A04FEF00380C3950
S2140514600001001025686610487900086A4B4EB9D9
S214051470000737A0588F600E487900086A524EB9A3
S214051480000737A0588F4E5E4E754E56FFEE48E75E
S21405149007183E2E000A2C2E000C0807000F6700C2
S2140514A000D60887000F4A4765320C470049622C6C
S2140514B04A3900104846671270003007E5880680EE
S2140514C00007E78420402850601870003007E5883C
S2140514D006800007E67C204028506006287C000829
S2140514E06A5B08390001001049B46700010C0C4717
S2140514F00008653A0C47000F623449EEFFEF48785E
S21405150000112F0C7000300751807222C1414EB970
S21405151000078C96C14106810080048E20012F00AD
S2140515204EB90006A1DE4FEF000C600000CC0C475C
S2140515300030650000C40C47003B620000BC49EE65
S214051540FFEF487800112F0C700030070680FFFF6C
S214051550FFD07222C1414EB900078C96C141068163
S2140515600080004E20012F004EB90006A1DE4FEF89
S214051570000C600000844A4765320C47005F622C09
S2140515804A3900104846671270003007E58806801D
S2140515900007E4FC20402850601870003007E588F6
S2140515A006800007E37C204028506006287C00085B
S2140515B06A6A08390001001049B4673C0C47000800
S2140515C065360C47000F623049EEFFEF487800118C
S2140515D02F0C7000300751807222C1414EB90007AA
S2140515E08C96C14106810080037E20012F004EB9EE
S2140515F00006A1DE4FEF000C2F0C4EB9000074CC90
S214051600588F2A00267C0010582ABA866D107E0050
S2140516106006179C78005287BE866DF6601C7E00B5
S2140516206006179C78005287BE856DF6600817BC65
S214051630002078005287BE866DF4423368004CDF82
S21405164018E04E5E4E754E56000048E701084AB94A
S214051650001052A467082879001052A4600628795D
S2140516600007F01E4EB90004C6FE0C00000C66040A
S2140516707E3260027E2242390010582A0C7400C859
S2140516807800660C42A74EB90004B918588F600C4E
S214051690487800014EB90004B918588F4CDF108001
S2140516A04E5E4E754E56000048E701084AB90010D2
S2140516B052A467082879001052A460062879000706
S2140516C0F01E4EB90004C6FE0C00000C66047E34FF
S2140516D060027E2442390010582A0C7400C978002E
S2140516E0660C42A74EB90004B918588F600C4878A6
S2140516F000014EB90004B918588F4CDF10804E5EB5
S2140517004E754E56000048E701084AB9001052A427
S21405171067082879001052A4600628790007F01E8D
